:020000040800F2
:1000000000200010051E03086D1E03080D5900088E
:100010006D1E03086D1E03086D1E0308000000001E
:100020000000000000000000000000006D1E03083A
:100030006D1E0308000000006D1E0308ED5500084A
:100040006D1E03086D1E03086D1E03086D1E030858
:100050006D1E03086D1E0308790D0008A50E00082B
:10006000690E00082D0E0008F10D00088D2A000809
:100070007D2A00086D2A00085D2A00084D2A000824
:10008000392A0008252A00086D1E03086D1E030882
:100090006D1E03086D1E03086D1E0308B50D0008D4
:1000A000214D0008614D0008114D0008894D0008E0
:1000B000514D0008414D0008314D00086D1E0308E8
:1000C0006D1E03086D1E03086D1E03086D1E0308D8
:1000D0006D1E030871570008F55600087956000890
:1000E0003D0D00086D1E03086D1E03086D1E0308FC
:1000F0006D1E03086D1E03086D1E03086D1E0308A8
:100100000000000000000000000000006D1E030859
:100110006D1E03086D1E03089D4A0108814A0108EF
:10012000112A0008FD290008E9290008D52900083E
:10013000C12900086D1E0308000000000000000037
:100140006D1E03086D1E03086D1E030800000000ED
:10015000000000000000000000000000000000009F
:1001600000000000000000006D1E03086D1E030863
:100170006D1E0308000000000000000000000000E9
:08018000000000006D1E0308E1
:100188002D2343702E2303712F23C371704700283A
:1001980070B51EDB0928044620DD012303EB830329
:1001A8005B00B0FBF3F2092AF8D87BB10D4EB4FB23
:1001B800F3F00928CCBF57223022A6FB03E50244FE
:1001C80003FB1044EB0801F8012BF0D100230B705E
:1001D80070BD2D230B7040420131DBE7303001F850
:1001E800010BF3E7CDCCCCCC884230B44FF00104FE
:1001F8002ED301FB04F4B0FBF4F58D42F9D284B19F
:10020800AAB901E0B0FBF4F5092DCCBF5722302282
:100218002A4404FB150003F8012BB4FBF1F4002C6D
:10022800F0D100221A7030BC7047B0FBF4F5092DEC
:10023800CCBF372230222A4404FB150003F8012BD7
:10024800B4FBF1F4002CF0D100221A7030BC7047D6
:100258000546002AEBD1D7E72DE9F04714461D469D
:10026800064600234FF47A722046294631F0F2FB05
:10027800DFF840814B4A4C4F88FB00310144C317DB
:1002880082FB002EC3EB611188FB012887FB002746
:100298008644464AC3EBEE2EC1EB011C82FB0E29B5
:1002A800A0EB8C0C0744424A86F806C0C3EB2747EC
:1002B8004FEAEE7C08EB010ACCEBA90C82FB078223
:1002C8004FEAE1780CEB4C0CC8EB6A18AEEBCC0E9D
:1002D800C8EB0818DFF8E0C086F804E0A1EB880155
:1002E80071718CFB0010F917C1EBE21240F2B551A5
:1002F80001FB1272C3EBE050B2F5896F4FEA800739
:100308003CDA40F2DA239A4242DCB2F5B77FB4BF56
:100318004FF0000C4FF0010C4FEA4C09DFF89C80BD
:1003280009EB0C0308EBC3031FFA8CFED88A09EB10
:100338000C0108EBC10116310B2301E031F8020D65
:10034800824218DA013BF9D1CC44012338F83C0049
:10035800B37007F2B2770132121ABE44F270A6F8EF
:1003680000E0204629464FF47A72002331F072FBF0
:100378003281BDE8F0870133DBB2E9E74FF0030EC5
:10038800F44640F29650DFF834804FF00609CEE785
:100398004FF0020EDFF82480F44640F229404FF077
:1003A8000409C4E7C5B3A29107452EC2ABAAAA2A7D
:1003B80073B06D1689888888792D0311B8320308BF
:1003C80003685A1C0260197070472DE9F047089CB1
:1003D8002578002B804689460CBF4FF0200A4FF045
:1003E800300A661C35B3002A29DD334601E002468F
:1003F80098B113F8011B501E0029F8D1971E60B15F
:100408003D46013D51464046C8476B1C002BF8DC71
:10041800257827EAE770013055B1041B2946404684
:10042800C847301916F8015B002DF7D1BDE8F087F1
:10043800BDE8F087002A04DC2846BDE8F0870020E4
:10044800EBE7571EDCE783684268D0ED037A00EBE0
:1004580083010133934281ED040A836004BF0023C2
:10046800836000EB830393ED047A036870EE277AC8
:100478009A42C0ED037A77EEC77AC0ED037A0CDAB8
:10048800013307EE103AF8EEC76AB7EE007A87EE46
:10049800A60A036030EE070A704707EE102AB8EE86
:1004A800C77A87EE870A704790ED057A90ED004A83
:1004B800D0ED066AD0ED014AD0ED047A90ED035AEA
:1004C800D0ED025AA4EE007AB0EE406AB0EE470AC8
:1004D800B0EE667AA6EE247A67EEC07AA0EE457A88
:1004E800E6EE257A80ED057AC0ED067A7047D0ED04
:1004F800057A90ED013AD0ED003AD0ED064A90ED3C
:10050800024A90ED077A90ED035A90ED086AD0ED13
:10051800045AC0ED067AF0EE406A27EE830AC0ED71
:10052800056AA3EEA60A80ED087AA4EE240AA5EED1
:10053800470AA5EEC60A80ED070A7047D0ED007A93
:1005480090ED017A30EE670AE7EE007AB0EE670ABE
:10055800C0ED007A704770470A44914214D030B415
:100568000139551E41F2210211F8014F082380EA92
:10057800042004044CBF82EA40004000013B80B2E2
:10058800F7D18D42F0D130BC7047012380F8453057
:10059800704790F8203033B1012B03D14FF400633A
:1005A8008382704770474FF48063838270472DE9D8
:1005B800F74F6A4CDFF8A8E123880091DEF80010B5
:1005C800B4F90480C3EB21125B00C3EBE103B4F977
:1005D800021052435943131308FB03F84FEAA83893
:1005E80008EBE12101EB8102B1F5FA3802F1800252
:1005F8004FEAE1794FEA222349F1FF39B4F908209B
:100608000193A8FB08AB08FB09F30BEB430BA161B3
:10061800D31702FB09F108FB0311A2FB08230B44C3
:100628001F03160347EA1257B4F90A2002FB0BF11D
:10063800D3170AFB03130546A2FB0A011944020A51
:1006480042EA016292194FEA2123E6887B4100328F
:1006580043F50043A2FB060106FB03114A10CB1722
:1006680052EA03016FD0B4F91060B4F90E00F7171D
:1006780006FB0BF10AFB0711A6FB0AAB8B4400FB38
:1006880009F6C11708FB0161A0FB08898944DEF857
:1006980004104FEA4846C1F5801E4FEA494747EA29
:1006A800D8371AEB060AB4F90C8076464BEB070BE1
:1006B800F71700264FEACE70F90716EB0A064FEA3D
:1006C800C80741EA5E0147EB0B0740F6354E861B2B
:1006D80061EB0707A6FB0E010EFB071131F0BAF913
:1006E800B4F916204E13470B47EAC14702FB06FE32
:1006F800D31707FB03EEA2FB07237344564307FBFC
:100708000366A2FB07233344560E46EAC316321883
:10071800B4F914604FEA636747EB01037143F717B5
:1007280000FB0717A6FB00013944C60C46EA413610
:1007380092194FEAE147B4F912607B41100A40EA86
:100748000360320112180DB1120A2A60009B13B11E
:100758001A46019B136003B0BDE8F08F1C480020C7
:10076800882200207047704707B5F7216A4628F0AD
:100778009BFB9DF801309DF800100C4A1B0143EAD1
:1007880001339DF8021043EA111353609DF80430B9
:100798009DF803101B0143EA01339DF8051043EA55
:1007A8001113136003B05DF804FB00BF882200201A
:1007B80070B40468037B2268022101FA03F31A4229
:1007C80013D042690A495C2000FB02124FF6FE76FC
:1007D80050685289C5680068296831402960C16835
:1007E800D24392B20A40C260636070BC704700BFD7
:1007F8005471002030B40A4B1D7875B1094B0020A4
:1008080003EBC5051A6899885062D4682143D16002
:10081800083323F8040CAB42F4D130BC704700BF56
:10082800347400203874002010B40268047B116806
:100838000223A340194209D00649406800240C70DD
:1008480001684FF6FE742140016053605DF8044B67
:10085800704700BF935100200023262203600270D6
:1008680027228270012243600271837170472DE94B
:10087800F341056906460F467DBBD0F80080C8F3F2
:100888000A0323B30023D6F80080019329F0F6FA6F
:10089800042819D1214C236943F001032361BBB219
:1008A800A8F8003029F0EAFA04282ED108F102034A
:1008B8000193019B3F0C1F8029F0E0FA236904286B
:1008C80023F00103236125D06FF0010505E029F02D
:1008D800D5FA042805D04FF0FF35284602B0BDE808
:1008E800F0810E4C236943F002032361C4F814809D
:1008F800236943F04003236129F0C0FA23690428DF
:1009080023F002032361BDD0E5E7236923F0010347
:100918002361D9E7336804333360DEE700200240FF
:10092800F8B504460D468E180027B54201D1206956
:10093800F8BDE368591CE160234415F8012B1A72CD
:100948000429F2D1A1682046FFF791FFE7602061F2
:10095800EBE7024B186804F0B5BF00BFE82200209F
:1009680010B490E80600047B40690223A3404B6062
:1009780013685DF8044B4FF6FE710B40136004F0EA
:1009880031BF002852D0036803F138422DE9F04FF7
:10099800920A514DAA5C02F01F0552090124022A4D
:1009A80004FA05F443D0032A00F09080012A43D0CA
:1009B80001F003077A1E012AC1F3810CC1F3001864
:1009C8008088C1F341113CD9C60700F189808507A9
:1009D80000F19580440700F1A380020700F1B1807F
:1009E800C60600F1BF80850600F1CD80440600F1FF
:1009F800DB80020600F1E980C60500F1F780850575
:100A080000F10581440500F11381020500F12181FF
:100A1800C60400F12F81850400F13D81440400F1F2
:100A28004B81020400F15981BDE8F08F70472B4AD1
:100A380095692C439461BBE7284A55692C43546156
:100A4800B6E7002422464FF0010E4FF0030904E0F8
:100A58000132102A04F10204E6D00EFA02F636EA50
:100A68000005F5D1D3F808A009FA04F5ED430AEA20
:100A7800050AC3F808A0D3F808B00CFA04FA4AEA41
:100A88000B0AC3F808A0B3F804A01FFA8AFA2AEAE6
:100A980006069E80B3F804A008FA02F646EA0A069B
:100AA800B6B29E801E682E401E60D3F800A007FADA
:100AB80004F646EA0A061E60D3F80CA001FA04F60A
:100AC80005EA0A0A46EA0A05DD60C1E7034AD5696C
:100AD8002C43D4616CE700BF9C61030800100240FE
:100AE8001A6822F003021A601A683A431A60DA6830
:100AF80022F003020A438507DA607FF56BAF1A68B4
:100B080022F00C021A601A6842EA87021A60DA6850
:100B180022F00C0242EA81024407DA607FF55DAFF9
:100B28001A6822F030021A601A6842EA07121A603C
:100B3800DA6822F0300242EA0112DA6002077FF531
:100B48004FAF1A6822F0C0021A601A6842EA871288
:100B58001A60DA6822F0C00242EA8112C606DA6038
:100B68007FF541AF1A6822F440721A601A6842EAA7
:100B780007221A60DA6822F4407242EA01228506E6
:100B8800DA607FF533AF1A6822F440621A601A6897
:100B980042EA87221A60DA6822F4406242EA812235
:100BA8004406DA607FF525AF1A6822F440521A60CD
:100BB8001A6842EA07321A60DA6822F4405242EAB6
:100BC8000132DA6002067FF517AF1A6822F4404254
:100BD8001A601A6842EA87321A60DA6822F44042D8
:100BE80042EA8132C605DA607FF509AF1A6822F455
:100BF80040321A601A6842EA07421A60DA6822F438
:100C0800403242EA01428505DA607FF5FBAE1A6898
:100C180022F440221A601A6842EA87421A60DA68A7
:100C280022F4402242EA81424405DA607FF5EDAEC3
:100C38001A6822F440121A601A6842EA07521A60C7
:100C4800DA6822F4401242EA0152DA6002057FF5BE
:100C5800DFAE1A6822F440021A601A6842EA875224
:100C68001A60DA6822F4400242EA8152C604DA6065
:100C78007FF5D1AE1A6822F040721A601A6842EA0B
:100C880007621A60DA6822F0407242EA016285045B
:100C9800DA607FF5C3AE1A6822F040621A601A68FB
:100CA80042EA87621A60DA6822F0406242EA8162A8
:100CB8004404DA607FF5B5AE1A6822F040521A6033
:100CC8001A6842EA07721A60DA6822F0405242EA69
:100CD8000172DA6002047FF5A7AE1A6822F040427A
:100CE8001A601A6842EA87771F60DA6822F0404281
:100CF80042EA8171D960BDE8F08F10B1036882883B
:100D08001A85704710B1036882889A61704738B1B4
:100D180000298388026814BF002110218B40936149
:100D2800704730B1036882881B8A1A4214BF0120B9
:100D3800002070472DE9F0410B4E356873691D405E
:100D480010D0DFF828800127B5FA85F4C4F11F0414
:100D580008EB840307FA04F4986803689847A543E6
:100D68007461F1D1BDE8F0810004014088220020BF
:100D78002DE9F0410B4E356873691D4010D0DFF83E
:100D880028800127B5FA85F4C4F11F0408EB840311
:100D980007FA04F4986803689847A5437461F1D189
:100DA800BDE8F08100040140882200202DE9F041CF
:100DB8000B4E356873691D4010D0DFF82880012775
:100DC800B5FA85F4C4F11F0408EB840307FA04F4A8
:100DD800986803689847A5437461F1D1BDE8F0812C
:100DE80000040140882200202DE9F0410B4E3568AF
:100DF80073691D4010D0DFF828800127B5FA85F403
:100E0800C4F11F0408EB840307FA04F49868036824
:100E18009847A5437461F1D1BDE8F0810004014011
:100E2800882200202DE9F0410B4E356873691D407A
:100E380010D0DFF828800127B5FA85F4C4F11F0423
:100E480008EB840307FA04F4986803689847A543F5
:100E58007461F1D1BDE8F0810004014088220020CE
:100E68002DE9F0410B4E356873691D4010D0DFF84D
:100E780028800127B5FA85F4C4F11F0408EB840320
:100E880007FA04F4986803689847A5437461F1D198
:100E9800BDE8F08100040140882200202DE9F041DE
:100EA8000B4E356873691D4010D0DFF82880012784
:100EB800B5FA85F4C4F11F0408EB840307FA04F4B7
:100EC800986803689847A5437461F1D1BDE8F0813B
:100ED80000040140882200200B490C4A8B6943F02A
:100EE800010310B58B611368094C43F480531360F8
:100EF80004F108004022002132F06BF94FF0FF3373
:100F0800A364C4F84B3010BD00100240000001403B
:100F18008822002003685B6A184703681B6A184721
:100F280070B44E1C0568C2728672AC69A44670BC67
:100F380060472DE9F041044618460D461646984686
:100F480030F0BEF82768E6722844A07229467D6909
:100F5800434632462046AC46BDE8F0416047036848
:100F680010B504461B689847236820469B68984735
:100F7800A37B0133A37310BD03681B69184710B521
:100F8800036804469B689847FF2301226373227312
:100F980010BD074B984202D04FF0FF307047054A0A
:100FA800538B01339BB25383508B80B2704700BF81
:100FB800003800408875002008B540F2E93300E0A9
:100FC8009BB10289013B12F0020F9BB2F8D001736A
:100FD80040F2E93300E043B10289013B12F0010F0E
:100FE8009BB2F8D0007BC0B208BDFFF7D2FFC0B2F9
:100FF80008BD38B583680446154601F07F0113B172
:101008001A689B881385606840F2E93300E07BB377
:101018000289013B12F0020F9BB2F8D0017340F233
:10102800E93300E023B30289013B12F0010F9BB2C0
:10103800F8D0037B606840F2E93300E0DBB1028955
:10104800013B12F0020F9BB2F8D0057340F2E9336E
:1010580000E083B10289013B12F0010F9BB2F8D086
:10106800037BA36813B11A689B889361012038BD7C
:10107800FFF78FFFDEE7FFF78CFFF2E7427A02B94E
:10108800704710B504460368406804F10A019847A0
:101098000023637210BD437A5A1C0344D2B24272D1
:1010A8009972037A934200D802B9704710B5044682
:1010B8000368406804F10A0198470023637210BD71
:1010C80098B10B4B012210B402FA01F103F1750437
:1010D80002E00333A34209D01A788242F9D15A7840
:1010E8000A42F6D001205DF8044B70470020FAE769
:1010F8001833030830B40A4D002305F1600401E0F9
:10110800272B0AD003EB43020133A15C8142F7D1BC
:101118002A4430BC92F862007047002030BC704707
:10112800B832030870B5448806460D46C4F30B046C
:1011380022460021284632F04CF83369094A934286
:1011480009D3094A934206D2224628461946BDE8E1
:10115800704030F0ADBE23B121462846BDE870404E
:10116800184770BD74A1030860A20308064B07491D
:101178008B4202D30023184670471A88C2F30B0229
:101188009042F8D01433F3E7009D030874A10308D4
:10119800024A136823EA000010607047743C00207C
:1011A800F8B5174D2B78A52B28D16B78BE2B25D1F8
:1011B800022229464FF6FF70FFF7CEF9114FAC1CFB
:1011C80022884AB1A618BE4218D2052A16D9214645
:1011D800FFF7C2F93446F3E721460222FFF7BCF9CC
:1011E8000222A118FFF7B8F90634074B641B1C80CC
:1011F80041F60F53C31A58425841F8BD0020F8BDB4
:1012080000F0030800000408365600202DE9F04FCE
:10121800DFF848914C4F8BB00326A7EB090718223B
:10122800002104A831F0D5FF484BCDF81090059760
:101238001A69120604D5464A5A6002F188325A6081
:1012480001228DF824203422DA60424B424C1B885C
:10125800ADF800300222694604A8FFF761FB0222BC
:1012680069464FF6FF70FFF777F9DFF8F4A080467C
:101278004FF0000B544536D30AAC002524F8245D02
:101288000222214604A8FFF74BFB022221464046D2
:10129800FFF762F940BAC043ADF80800022202A97C
:1012A80004A8FFF73DFB079860B106ABC0F1040244
:1012B8002946184431F08DFF069904A8FFF7D7FA9C
:1012C800079508909DF82430089A23B11F490B69A7
:1012D80043F080030B61013E2DD0002A9FD1FFF718
:1012E8005FFF50B32CE065888DF80DB0C5F30B0592
:1012F800AB1DADF808302388C3F30B02ADF80A2004
:101308001B0B062202A904A88DF80C30FFF708FB76
:10131800062202A94046FFF71FF9616880462A465F
:1013280004A8FFF7FDFA616840462A46FFF714F95A
:10133800143480469EE7002AD1D0052002F068FBCD
:101348000BB0BDE8F08F00BF000004080020024089
:10135800230167458D330308009D030800F0030847
:1013680074A103080378202B024600F10100F9D08C
:10137800092BF7D02D2B2CD02B2B03BF5378B7EE8E
:10138800000A0246B7EE000AA3F13001C8B20928E4
:101398009FED467A10D8F2EE046A07EE901AF8EE3E
:1013A800E77A12F8013FE7EE267AA3F13001C8B2D6
:1013B8000928B0EE677AF0D92E2B4CD003F0DF0362
:1013C800452B0BD0F7EE007A67EE276A20EE260A47
:1013D80070475378BFEE000A0246D5E710B451783B
:1013E8002D2959D02B290ABF9178501C901C002414
:1013F800A1F13003092B53D8002303EB830301EB3E
:10140800430310F8011FA1F13002092AA3F13003A8
:10141800F3D9B3F59A7F28BF4FF49A73072B42D9B3
:10142800DFED236A1A46F7EE007A083A072A67EED4
:10143800A67AFAD803F007032BB1F2EE046A013B4F
:1014480067EEA67AFBD124B3C7EE276A5DF8044B92
:1014580020EE260A70475378A3F13001C8B2092854
:1014680002F10102AAD8F2EE046AF0EE665A07EE1B
:10147800901AF8EEE77A12F8013F87EEA66AA3F110
:101488003001C8B2092866EEA56A37EE067AEED9A9
:1014980094E767EE276AD9E7901C91780124A7E7BB
:1014A800F7EE007ACFE7F7EE007AC5E70000000014
:1014B80020BCBE4CB5EEC00ADFED317AF1EE10FA71
:1014C800CCBF30EE270A30EE670ADFED2E7A20EE29
:1014D800270A30B5FDEEC07A87B017EE904A054668
:1014E80084EAE470002303A9A0EBE470019300935D
:1014F80002932AF09DF9002CACBF20232D2303A8CA
:101508008DF800302FF0DCFD012803A924D0022833
:101518002DD0032805BF3023684668468DF8013072
:1015280031F05FFE68462FF0CBFD0338C4B2224687
:101538006946284631F08CFE00232B5528462FF0AB
:10154800BFFD2E22431C2A540DEB0401E81831F08C
:1015580065FE284607B030BD302368468DF8013057
:101568008DF802308DF8033031F03BFEDAE7302396
:1015780068468DF801308DF8023031F032FED1E73F
:101588006F12033A00007A442DE9F04106461546E9
:101598000846B6FBF2F43CB905FB1464124B1B5D1C
:1015A80000F8013BBDE8F081B4FBF2F767B90E4BD8
:1015B80005FB174705FB1464DA5D00F8012B1B5D7A
:1015C80000F8013BBDE8F081B7FBF2F8B8F1000F75
:1015D80002D04046FFF7D8FF05FB1878024B13F8F6
:1015E800082000F8012BE3E7EC630308104B2DE912
:1015F8003048D3E9004554EA05020BD103460122DD
:1016080000201871587198719A70DA7018801881D2
:10161800BDE83088074B1A6814EB020B45F1000C43
:101628005A466346FEF718FE0120BDE8308800BF21
:1016380050240020F0750020F0B402888578154FFA
:10164800C37804794179A2F2B27202F0030606EB7C
:101658004606013D05EB8605013B37F8156085799F
:10166800008940F2B557920807FB0232931903EB41
:10167800430304EBC303C3EB031301EB8303C3EB83
:10168800031305EB830300214FF47A72C2FB0301B5
:10169800F0BC7047B8320308FAB170B48E1804462B
:1016A80003E0101A14D1B14214D014F8012BA2F19E
:1016B8004103192B11F8013BA3F1410598BF2032D2
:1016C800192D03F12000ECD9D01A01D1002BEAD151
:1016D80070BC7047002070BC7047104670474FF0D0
:1016E800FF32FFF7D9BFA0F16103192B98BF20384B
:1016F8007047A0F14103192B98BF2030704720286C
:1017080005D0093804288CBF00200120704701202B
:101718007047613819288CBF002001207047413874
:1017280019288CBF002001207047303809288CBF49
:10173800002001207047A0F13003092B07D920F0C1
:101748002000413819288CBF002001207047012053
:10175800704730B402681146531C036011F8024BFD
:101768000160D31C517803609378151D05601B0434
:1017780043EA0123D078234343EA006030BC704732
:101788000368591C1A46016012F8021B0260587857
:1017980041EA0020704703685A1C026018787047B5
:1017A80038B504460068154630F082FB22682A44A2
:1017B800226038BD036810B40A0A5C1C04601A7001
:1017C80003685A1C026019705DF8044B704703687F
:1017D8005A1C026010B4197003680A0A5C1C046081
:1017E8001A7003680A0C5C1C04601A700368090EFE
:1017F8005A1C026019705DF8044B704703685A1C44
:10180800026019700368090A5A1C0260197070474F
:101818002DE9F047002488B080460F461E46A146B1
:1018280005AD531C0393117839B3252933D1931C83
:10183800CDF810900393507830284ED04FF0000A1E
:10184800A0F13003DBB2092B42D96C2819D06428E7
:1018580000F0938024D825281CD063D9582876D046
:1018680063281BD131784046B847039A531C039329
:101878001178043601340029D7D1204608B0BDE8D4
:10188800F087039B5A1C03921B78642B7CD02AD8C0
:10189800252B54D1252140460134B847039AC0E787
:1018A800732833D044D975284FD106F1040E306817
:1018B8002B4600220A217646FEF796FC049A0095EC
:1018C800534639464046FEF780FD039A0444A8E78C
:1018D80004AA03A928F0E8FAB7E7D31C0393907881
:1018E8004FF0010AACE7732B10D05BD9752B3AD0B7
:1018F800782B96D1A3F15802B2FA82F230685209D5
:101908002B4610210436FEF76FFCD7E73368049A9C
:101918000093394600234046FEF757FD0436044439
:10192800039A7EE70028B9D1204608B0BDE8F087C1
:101938006E28B3D1039A336804361C6071E72AD93C
:10194800582BD7D0632B8DD06BE77828A6D1A0F180
:101958005802B2FA82F2306852092B461021FEF77B
:1019680043FC0436AAE706F1040E30682B46002231
:101978000A217646FEF738FCA0E7331D3068294671
:101988001E46FEF704FC99E7331D306829461E46BB
:10199800FEF7FDFB92E7002B7FF443AF204608B02B
:1019A800BDE8F0876E2BC6D03BE70EB400B584B017
:1019B80005AB019053F8042B0649039301A8FFF7E0
:1019C80027FF019B00221A7004B05DF804EB03B0F6
:1019D800704700BFC90300082DE9F04707468CB0DF
:1019E8001E469246002A6AD1154614460A8840F2D5
:1019F800B1739A423AD98B78581E0B2836D891F889
:101A080003E00EF1FF301E2830D891F804C0BCF175
:101A1800170F2BD891F80590B9F13B0F26D8887984
:101A28003B2823D8B1F80880B8F57A7F1ED24FF04A
:101A38000108002E34D109890491002CB4BF2D214E
:101A48002B21002CB8BF6442039005910795CDF86F
:101A58000890CDF804C0CDF800E0384606942F4928
:101A6800FFF7A3FF40460CB0BDE8F0870023012133
:101A780018468E46ADF824308DF828308DF8293078
:101A88008DF82A30ADF82C3099469C461A4698466F
:101A98008DF826108DF827100B4609A9002ECAD0FC
:101AA8000390CDF80890CDF804C0CDF800E0384692
:101AB8001B49FFF77AFF40460CB0BDE8F087194C88
:101AC80084FB0234A318D417C4EB6314C4EB0415C5
:101AD800A2EB85052DB2002D0846B8BF6D42FFF771
:101AE800ABFD4FF47A720023804689462FF0B2FF8F
:101AF8003C230AFB030A4FF47A7200234046494606
:101B08002FF0A8FF4FF47A7192B20023C1FB0A2389
:101B180009A8FEF7A1FB24B209A967E73464030802
:101B280014640308898888880FB430B583B006AB7D
:101B38000A490B4853F8042B096800680193FFF71A
:101B480067FE084C0546206803F0ACFE0028FAD072
:101B5800284603B0BDE8304004B0704788360020FE
:101B68008C360020E8220020DFED2B7AB4EEE70A5D
:101B7800F1EE10FA4ADDDFED296A9FED297A01E0DE
:101B8800B0EE670AB4EEC70AF1EE10FA70EE667AA4
:101B9800F6DC9FED247AF4EEC77AF1EE10FA38D528
:101BA800DFED1E6A9FED207A01E0F0EE407AF4EE58
:101BB800C77AF1EE10FA37EEA60AF6D4DFED1B7AF3
:101BC800B4EEE70AF1EE10FA14DDDFED137A37EE22
:101BD800C00A60EE006A9FED166A9FED167ADFED87
:101BE800167AA6EE867A20EE266AE6EE877AA6EEC2
:101BF800270A7047DFED117AB4EEE70AF1EE10FA22
:101C080044BFDFED087A37EEC00AE2E7F0EE407A2B
:101C1800BFE7B0EE670AD1E7DB0F4940DB0FC940E9
:101C2800E4CB1641DB0F49C0E4CB16C1DB0FC93F3B
:101C380092E741B99730083C15A82ABEDB0FC9BF07
:101C480009B909E0194690FBF1F301FB13030846B3
:101C5800002BF7D1084670470146FBE707EE901ABC
:101C6800F8EE677A9FED837A27EE800A20EE070A5E
:101C7800FDEEC07A17EE903A2033402B00F28C80AC
:101C8800DFED7D7AB4EEE70AF1EE10FA40F3E88072
:101C9800B0EE407A9FED796ADFED796A01E0B0EE47
:101CA800677AB4EEE67AF1EE10FA77EE467AF6DC69
:101CB8009FED747AF4EEC77AF1EE10FA40F1CD8018
:101CC8009FED6E6ADFED706A01E0F0EE477AF4EEA0
:101CD800E67AF1EE10FA37EE867AF6D4DFED6B7A13
:101CE800B4EEE77AF1EE10FA51DCDFED697AB4EE82
:101CF800E77AF1EE10FA44BFDFED627A37EEC77A81
:101D080027EE076ADFED635ADFED637ADFED636A7A
:101D18009FED635AE6EE257A67EE065AE6EE276AE5
:101D2800F7EE007AA5EEA67AF0EE675AE7EE055AC6
:101D3800E7EE457A87EEA55ADFED547A30EE277A3A
:101D4800FDEEC76A16EE903A2033402B29D99FED55
:101D5800557AF6EE006AB7EE006AF7EE004AC4EE6E
:101D6800A57A0023836143610362C36180ED045A4D
:101D780067EEA66A27EE866A27EE877AC0ED006AC4
:101D8800C0ED026A80ED016A80ED037A7047DFEDED
:101D98003A7A37EEC77AB3E7B7EE005AF0EE455A0B
:101DA800CAE7B4EEE70AF1EE10FA5FDD9FED336A99
:101DB800DFED336A01E0B0EE677AB4EEE67AF1EE71
:101DC80010FA77EE467AF6DC9FED2E7AF4EEC77AB3
:101DD800F1EE10FA47D59FED296ADFED2B6A01E095
:101DE800F0EE477AF4EEE67AF1EE10FA37EE867AFC
:101DF800F6D4DFED267AB4EEE77AF1EE10FA27DCB6
:101E0800DFED237AB4EEE77AF1EE10FA44BFDFEDA6
:101E18001D7A37EEC77A27EE076ADFED1E4ADFED37
:101E28001E6ADFED1E7AE6EE246A67EE064AE6EEE3
:101E3800267AB7EE006AA4EEA77AF6EE006A36EEC6
:101E4800476AF8EE007A27EE277A66EE266A84E774
:101E5800DFED097A37EEC77ADDE7B0EE677A3DE75E
:101E6800F0EE407A24E7B0EE677AC2E7F0EE477A00
:101E7800AAE700BF27D4D236DB0F4940DB0FC940A1
:101E8800E4CB1641DB0F49C0E4CB16C1DB0FC93FD9
:101E9800DB0FC9BF92E741B99730083C15A82ABEA5
:101EA800F304353F0000008070B406688E4217D9ED
:101EB8000139751E002311F8014F0822634013F001
:101EC800800F4FEA430318BF83F0D503013ADBB212
:101ED800F5D18D42EFD1721C0260337070BC70472F
:101EE8000023F8E710B44C09012250F8243001F01F
:101EF8001F0102FA01F10B4340F824305DF8044B4E
:101F080070474B0901F01F0150F82320012303FA01
:101F180001F1114214BF184600207047074A084BC8
:101F280010781B78074A834296BFC31AC3F180030F
:101F38000020126818441044704700BF585E002003
:101F4800D55D0020F4470020064A074B10781B781F
:101F580083428ABFC3F18003C01AC018C0F17F0052
:101F6800704700BF585E0020D55D002010B50446BC
:101F780000BF8068FEF7C1FE6068FFF71DF8A06823
:101F8800FEF7C0FE00BF10BDF8B584894FF6FF7696
:101F98004FF47A742BB311B30F78013101E0B442D6
:101FA80017D00589013CAD07A4B2F8D507734FF4E3
:101FB8007A7402E0BCB2B4420BD00589ED0704F193
:101FC800FF37F7D5057BEDB20AB115700132013B39
:101FD800E0E7FEF7DEFF003018BF0120F8BDFF275D
:101FE800DFE70120F8BD30B5134C237883B01BB967
:101FF8000120237003B030BD1049052200230D686D
:102008008DF804208DF8053000BFA868FEF775FE2E
:102018006A4601A902236868FFF7B6FFA868FEF7B9
:1020280071FE00BF9DF8013003F0010383F0010049
:10203800237003B030BD00BF1B5D0020085D002089
:1020480070B5064C0646256803E023685B1BB3425F
:1020580003D8FFF7C8FF0028F7D070BDF07500203F
:102068002DE9F04F89B0B2F1000A02900491039370
:1020780040F3C5800B46002201EB8A0153F8040B9C
:102088008B420244FAD1039B0592002B00F0AF80EB
:10209800059B002B7CD05E4B059A1B68DFF8889166
:1020A80000920099DAB25118B1F5807F8CBFC2F561
:1020B8008072009A0192574A92689A4240F282804E
:1020C800554A1178002206928DF81C2002228DF8BC
:1020D8001820002960D01A0E8DF819200DF11A0267
:1020E8001C0C190A9370147051700620FFF7A8FF92
:1020F8000621D9F80000FFF739FF484A0123137079
:1021080000BFD9F800309868FEF7F7FD424BD9F8C0
:1021180000201B785068002B06A90CBF0423052358
:102128000022FFF731FF0024049D029E019FA34671
:1021380029684FEA840800220B46013471B1B9427C
:102148002DD2D9F8000031684068FFF71DFF2A68D2
:10215800336813443360BF1AC5F800B0A24505F1CF
:10216800040506F10406E3D1D9F800309868FEF7B3
:10217800C9FD00BF264B019900981B68421A0092BE
:10218800234A0B441360039A4AB3009A002A88D161
:10219800059809B0BDE8F08F0DF11902A0E7029C7F
:1021A800D9F8003054F80810586800223B46FFF769
:1021B800EBFE54F808202B683A44DF1B44F808204B
:1021C8002F60D1E70598009C1549164A001B059019
:1021D800059800230B70137009B0BDE8F08F059BBC
:1021E800009A9B1A0593059809B0BDE8F08FFFF790
:1021F800FAFE00287FF44CAF039B0593C8E7039CC5
:102208001CB9FFF7F0FE0594C2E700230593BFE76A
:10221800F44700204C1A00201A5D00201B5D0020A6
:10222800585E0020D55D0020085D002070B5104D77
:10223800104E2B7831788B4284B016D00E4A039218
:102248001A4402928CBF0C46CA1A04A98CBFC3F167
:1022580080020024012341F8102D02A802220194D3
:10226800FFF7FEFE002333702B7004B070BD00BF73
:10227800D55D0020585E0020D85D002070B5194C4F
:10228800194D23782978994284B027D0174A0392A8
:102298001A44029234BF0E46CA1A04A934BFC3F1C5
:1022A80080020026002341F8102D02A80222019680
:1022B800FFF7D6FE23781844C0B203062B7848BF30
:1022C80080F080008342207002D0002004B070BDEE
:1022D800002301202B70237004B070BD012004B0CE
:1022E80070BD00BFD55D0020585E0020D85D00207D
:1022F80010B50C4C45F20820FFF7A2FE2068062115
:10230800FFF734FE084B20680122C7211A70FFF737
:102318002DFE06480649074A002303700B70136018
:1023280010BD00BF085D00201B5D0020585E002026
:10233800D55D0020F4470020F0B51F4C83B0277806
:1023480000234FF0030E00930E4615468DF8043017
:102358008DF800E06FB3030E8DF801300DF1020324
:10236800010C020A9870197006205A70FFF768FE6F
:10237800E8B100BF114F3B689868FEF7BEFC2378B0
:102388003A68002B14BF05230423694650680022CD
:10239800FFF7FAFD3B683246002158682B46FFF7E5
:1023A800F3FD3B689868FEF7ADFC00BF284603B014
:1023B800F0BD0DF10103D3E71A5D0020085D002090
:1023C800F0B5124B9D6885B00DB905B0F0BDED0AAA
:1023D80014D0002704AE7C196410E002102269466C
:1023E800FFF7AAFF0F2809DD6B4653F8042B0132CB
:1023F8000AD1B342F9D12546AF42ECDBFFF716FF0D
:10240800034BED021D60E0E7671CF5E74C1A00205E
:10241800F4470020F0B55B4B5B4A97B019689142CE
:1024280000AF00F0A3805949594A00234FF47000C7
:10243800C1F888003B607B60136843F48033136005
:1024480003E03B68B3F5A04F09D0136803F40033E9
:102458007B603B6801333B607B68002BF1D04C4BC1
:102468001B6813F4003318BF01237B607B68012BC2
:1024780052D0464C464B474AE260474A596A116077
:102488005A6A42F080725A625A6942F4FC025A61EE
:102498000025032207F10801012341F6FF764FF0DA
:1024A8009040FD60BE603A73BB732CF073FA4FF630
:1024B800FF7307F108013948BB602CF06BFA07F18C
:1024C80008013748374E2CF065FA07F108013648FD
:1024D8002CF060FA07F1080134482CF05BFA07F198
:1024E800080133482CF056FA07F108002CF0ABFA33
:1024F800BB683049304AA1FB031330499B0CF020DC
:102508004FF0070E5C370B60566084F82300956027
:10251800C2F800E0BD46F0BD294A1D4B12211160EA
:102528005A685A605A685A605A6842F480625A6017
:102538005A6822F47C125A605A6842F4E8125A60C7
:102548001A6842F080721A601A689201FCD55968BC
:102558000F4A21F003015960596841F0020159609E
:10256800536803F00C03082BFAD182E700221A60A3
:1025780062B6144B1B6883F30888134B1B68984793
:10258800FEE700BFFC9F0020EFBEADDE00ED00E0DF
:10259800001002400005FA056860002000040048A9
:1025A800000800483F190100000C004800100048CE
:1025B8000014004883DE1B4310E000E0F47500209F
:1025C8000020024000D8FF1F04D8FF1F70B50F4C31
:1025D8000F4DC0EBC00004EB8004686926693043E6
:1025E800686182B09209667BA1600025012101A87B
:1025F80063618DF804608DF805208DF806508DF81C
:10260800071029F093FE02B070BD00BF601A0020C9
:1026180000100240074BC0EBC00030B403EB800051
:10262800054C056963692B4363610176427630BCCA
:10263800704700BF601A0020001002402DE9F04FDB
:102648005E4C54F8204083B0002C71D0A66D98469B
:1026580091465B4B72682265A160236004F15E01BC
:102668004FF4807304F5AF726161A261E360236186
:102678000746307E2BF07CFAF068A8B1514B002158
:102688005A68904203F11C0300F0928001310C2932
:10269800F6D100207A1CD2B20C21FFF7BBFF236DC4
:1026A800F26862632433E364B068D8B1454B002113
:1026B8005A68904203F11C0378D001310C29F7D1F4
:1026C80000257A1CD2B20B212846FFF7A3FF234628
:1026D800F27E3D492846FFF779FF236DB268A26371
:1026E8002833A36494F85D0002F0E8FA054694F8EC
:1026F8005C0002F0E3FA18F0080F824696F819B069
:102708001AD0CDB118F0110F4FF00B0307F10107E4
:1027180014BF4E213E21EF715A46AB71284601F095
:102728002DFF18F0010F45D0636B5BB3A36B4BB360
:10273800204603B0BDE8F08F18F0010F0CBF4FF032
:102748002E084FF04E0819F0020F09D045B10B22A0
:102758007B1CAA71EB7128465A46414601F00EFFD0
:1027680019F0010FE0D0BAF1000FDDD001370C23CA
:102778008AF807705A4641468AF80630504601F0F2
:10278800FDFED1E7337FB27E8DF804209B0900213E
:10279800012201A88DF805308DF806108DF8072064
:1027A80029F0C4FD204603B0BDE8F08FCDB288E71C
:1027B800C8B26FE72846FEF7A0FAB5E794360020BE
:1027C80090330308601A00206909000800B97047AF
:1027D800F0B595B005462BF069FD6E4EC3680268EA
:1027E80032600446002B00F0C380284602F066FAE7
:1027F800694B186518B1292200238271C371227AA6
:10280800664D2E2101F0BAFE306802F037FC2BF03D
:10281800AFF93068624A038823F001031B041B0CDC
:10282800038014A91E232B8001270F230025138062
:1028380021F84C7D2D230293ADF80C50ADF80650CD
:10284800ADF80E502BF0E0FCE379ADF8145060229F
:102858009907ADF816500695ADF81C50ADF81E5006
:10286800ADF82050ADF82250049200F1838013F0A7
:10287800010F14BF022200224FF48073ADF81470C8
:10288800ADF81C20ADF82030002304AA6179306827
:10289800069301F065FC306861792BF095FC30688F
:1028A800436C43F40043436403889BB243F08003C2
:1028B8000380E3799B0768D56179026A04238B401A
:1028C80022EA03020262026A134303623268354F46
:1028D80013889BB243F001031380207C0022292136
:1028E800FFF798FE3049207C00236022FFF76EFE38
:1028F800E068386029F086FC386803684FF6FE7295
:102908001340036029F07EFC09A829F04DFC3368C8
:102918006279264938680A9134331344099380222E
:102928001023002509A940F22A3E0E920B934FF47A
:1029380000724FF400530D951095139511950F9251
:102948001293ADF830E029F03DFC627933680C2A27
:1029580098BF1749D86898BF31F812503A68154996
:102968000543DD601368012043F00203136008701B
:1029780015B0F0BD13F0010F14BF08222A46042336
:10298800ADF81E20ADF816307EE70122617929F0F6
:10299800A5FA9BE7405B002088220020365B0020D8
:1029A800345B00203C5B002031080008C451002043
:1029B80074610308385B00200348D0F83C3113B138
:1029C80000F59A7018477047601A00200348D0F83D
:1029D800203113B100F58C7018477047601A002039
:1029E8000348D0F804310BB1FC301847704700BFDA
:1029F800601A00200348D0F8E8300BB1E0301847DF
:102A0800704700BF601A00200348D0F8CC300BB1E3
:102A1800C4301847704700BF601A00200348D0F838
:102A2800B0300BB1A8301847704700BF601A0020BB
:102A38000348D0F894300BB18C301847704700BF6A
:102A4800601A00200248836F0BB170301847704736
:102A5800601A00200248C36D0BB154301847704704
:102A6800601A00200248036C0BB1383018477047D1
:102A7800601A00200248436A0BB11C30184770479F
:102A8800601A00200248836803B11847704700BFE6
:102A9800601A0020F0B53E4C059D00EB800004EB69
:102AA80080046468002C71D03A4E49004FF42040ED
:102AB800CFB27065A169090454D46068DFF8E0E01A
:102AC80047F4903100EA0E0001434FF42040616062
:102AD800706503E0411E002848D00846A1698907AF
:102AE800F8D54FF42040A262706503E0421E00282A
:102AF8003CD01046A2695206F8D5274A6168DFF82B
:102B0800A0E0706542EA0342174301EA0E02174348
:102B18006760C3B1013BDBB201332B44A0694FF4BA
:102B2800204210F0040002F1FF3207D1511C26D0D8
:102B3800A06910F0040002F1FF32F7D0626A05F8CC
:102B4800012B9D42EAD14FF42040706502E0431EFC
:102B580060B11846A3699B06F9D520237065E36127
:102B68000120F0BD411E08B10846A3E70B4A1388AF
:102B780001339BB24FF0FF3113807165F0BD0749F7
:102B880072650B8801339BB20B80F0BD2046F0BD07
:102B9800607500208822002000240002345600209E
:102BA800009800FCF0B50D460178012983B0044671
:102BB800164618D0022902D0002003B0F0BD806864
:102BC8001F46FEF79AF845F080016068FEF7F4F9B1
:102BD8003B46324600216068FFF7D6F9A068FEF749
:102BE80091F80120E9E790F90400421CE4D002289A
:102BF800E2DC617900962A46FFF74CFFDDE7F0B585
:102C0800037C012B85B0044663D0022B67D183690E
:102C180013B11A689B881385606940F2E93301E0B3
:102C2800002B6CD00289013B12F0020F9BB2F7D047
:102C3800C323037340F2E93301E0002B5FD002891C
:102C4800013B12F0010F9BB2F7D0037B60694FF094
:102C5800060E838902AE4FF47A734FF6FF71FF2791
:102C680003E0013B9BB28B423CD002899507F8D523
:102C780007734FF47A7302E0ABB28B4232D0028909
:102C8800D20703F1FF35F7D5027BD2B20EB132700D
:102C98000136BEF1010EE8D1A36913B11A689B8809
:102CA80093619DF80C009DF808609DF809109DF847
:102CB8000A509DF80B209DF80D3041EA062143EAA1
:102CC800002342EA0522012021876287A38705B0F5
:102CD800F0BD90F91400431C01D0022805DD002046
:102CE80005B0F0BDFEF755F9D6E702AB617D00935C
:102CF80043220623FFF7CEFE0028D2D1EFE7FEF7E6
:102D080048F9A3E7F0B5037A012B85B0044663D0F0
:102D1800022B67D1036913B11A689B881385E06891
:102D280040F2E93301E0002B6CD00289013B12F03C
:102D3800020F9BB2F7D0BB23037340F2E93301E0E3
:102D4800002B5FD00289013B12F0010F9BB2F7D034
:102D5800037BE0684FF0060E838902AE4FF47A7366
:102D68004FF6FF71FF2703E0013B9BB28B423CD03B
:102D780002899507F8D507734FF47A7302E0ABB26E
:102D88008B4232D00289D20703F1FF35F7D5027B97
:102D9800D2B20EB132700136BEF1010EE8D123690C
:102DA80013B11A689B8893619DF80C009DF8086020
:102DB8009DF809109DF80A509DF80B209DF80D30DC
:102DC80041EA062143EA002342EA05220120E18282
:102DD8002283638305B0F0BD90F90C00431C01D039
:102DE800022805DD002005B0F0BDFEF7D2F8D6E7D1
:102DF80002AB617B00933B220623FFF74BFE0028C2
:102E0800D2D1EFE7FEF7C5F8A3E7B0F1FF3F56D000
:102E1800022854DCF0B4334C00EB800004EB800053
:102E28004468002C5BD0304E49004FF42040CDB2AE
:102E38007065A169090444D460682C4F45F080711D
:102E4800384041F4903101434FF42040616070658F
:102E580003E0411E002838D00846A1698F07F8D53D
:102E68004FF42040A262706502E0421E68B310462B
:102E7800A2691106F9D562681C4945F0007545F448
:102E880080350A4015434FF420406560706502E0C4
:102E9800421ED0B11046A2699207F9D54FF42040DE
:102EA800A362706502E0431E78B11846A3699B06C9
:102EB800F9D520237065E3610120F0BC704700203C
:102EC8007047411E08B10846B3E7094A1388013321
:102ED8009BB24FF0FF3113807165F0BC70472046FC
:102EE800FBE700BF6075002088220020009800FCE6
:102EF8003456002070B40578012D07D0022D02D178
:102F080070BCFEF776B8002070BC7047134670BCE2
:102F18000A46417990F9040077E73122F421E9E77C
:102F28002DE9F04F87B090F855300290002B40F013
:102F3800C281029A137C1032012B1046039200F0D2
:102F48007282022B00F0B281BD4CBE4EDFF8FC92BB
:102F5800BD48DFF8FCE24FF0640A4FF0100C4FF464
:102F68007A75D9F80430C3F30803002B40F0F380D6
:102F7800EFF31183002B40F0EE802168826800BFD8
:102F880023689942F9D1376805FB07F39B1AB3FB0D
:102F9800F7F305FB013101270191D9F80430C3F398
:102FA8000803002B40F09D80EFF31183002B40F0C5
:102FB80098802368816800BF22689342F9D1D6F8C7
:102FC80000B005FB0BF2521AB2FBFBF205FB032320
:102FD800019A9B1AB3F57A7FDFD3BAF1010AC0D1FF
:102FE800029D297C012900F01582022900F04A81FE
:102FF800029B012993F8503000F05081022900F01B
:103008003B81DFF848929048DFF844E24FF00F0A1E
:103018004FF0100C4FF47A75D9F80430C3F3080355
:10302800002B40F0B480EFF31183002B40F0AF8009
:103038002168826800BF23689942F9D1376805FB87
:1030480007F39B1AB3FBF7F305FB01310127019145
:10305800D9F80430C3F30803002B5FD1EFF31183D1
:10306800002B5BD12368816800BF22689342F9D1A5
:10307800D6F800B005FB0BF2521AB2FBFBF205FBC7
:103088000323019A9B1AB3F57A7FE1D3BAF1010AB7
:10309800C2D1029C237C94F84E20012B00F0CC81F5
:1030A800022B00F0D780012B00F0DC80022B00F00F
:1030B800B280012B00F0B980022B00F09880012B20
:1030C80000F09F80022B7ED0012B00F08680022B1F
:1030D80004D1039801223821FDF78BFF07B0BDE822
:1030E800F08FEFF311888CF3128881680368DB0393
:1030F80044BFCEF8007081682368DEF800205FFACC
:1031080088F888F31188D6F800801A4405FB08F37C
:103118005B1AB3FBF8F305FB023359E7EFF31188A9
:103128008CF3128881680368DB0344BFCEF8007013
:1031380081682368DEF800205FFA88F888F3118830
:10314800D6F800801A4405FB08F35B1AB3FBF8F3C2
:1031580005FB023395E7EFF311828CF31288876839
:103168000368D90303D50123CEF8003087682368A4
:10317800DEF80010D2B282F311883268194405FBD8
:1031880002F3DB1BB3FBF2F305FB013103E7EFF3BB
:1031980011828CF3128887680368D90303D5012349
:1031A800CEF8003087682368DEF80010D2B282F3C8
:1031B80011883268194405FB02F3DB1BB3FBF2F3F9
:1031C80005FB013142E71A4637210398FDF711FF45
:1031D800029B1B7C012B7FF47AAF02983822417D39
:1031E80090F91400FFF711FE07B0BDE8F08F182220
:1031F8001C210398FDF7FDFE029B1B7C012B7FF42D
:1032080061AF029C02233722617D94F91400FFF715
:10321800FCFD237C58E718221B210398FDF7E9FEE3
:10322800029B1B7C012B7FF447AF029C18231C22B6
:10323800617D94F91400FFF7E8FD237C3FE700BFA8
:10324800F0750020F475002010E000E000ED00E0CB
:10325800EC7500201A210398FDF7CBFE237C012B87
:103268007FF424AF029C18231B22617D94F914007B
:10327800FFF7CBFD237C1CE71A4619210398FDF7BD
:10328800B8FEBEE66B2103220398FDF7B2FE297C47
:10329800029B012993F850307FF4B0AE02981922AE
:1032A800417D90F91400FFF7B0FDAAE680226B215A
:1032B800FDF79FFE48E61C09013C052C03F00F03AF
:1032C80000F2C380774A32F8140040FA03F2D207BA
:1032D80040F1BB80012505FA03F3013B18402EF0AD
:1032E80009FC714BDFF8DC811E5D064418EBC6044F
:1032F80000F0AB8058F83600A788038A3B407FF47B
:1033080018AE00F13842920A6849E3718B5C03F009
:103318001F025B092021022B05FA02F2A17100F0BD
:10332800BB80032B00F0B380012B00F0AB8004A915
:103338004FF0000A0497CDF814A02BF02BFBA388BC
:10334800029D5B4AEA60B3FA83F3C3F11F035F1C73
:103358003FF4EFADD9B201F0FC0202F1804202F570
:10336800803201F00300D2F808E058F83610514FC7
:10337800DFF854C1504E80004FF00F0808FA00F8EB
:103388002EEA080E07EB830805F10C09C8F8089027
:10339800C2F808E0D2F80890DFF83081C1F387213D
:1033A80081404FF0010E0EFA03F041EA09019160E5
:1033B800CCF800003268C1430A403260D8F80020D7
:1033C8000A40C8F800203268024332605CF80C2CCE
:1033D8003A4E0A404CF80C2CD8F8082006EB0309A2
:1033E8001140C8F808105CF80C2C99F80011024339
:1033F8000F444CF80C2C97F84820F02A2ADC581C6B
:103408003FF497AD012202FA03F32B490A681343EC
:103418000B608EE5697D95F9140003236B22FFF795
:10342800F4FC297CE4E502988023417D90F914009E
:103438006B22FFF7EAFC87E51346617D94F91400D7
:103448001A22FFF7E2FC237C2DE6029A184BD36080
:103458000123DAE77318F02293F810318DF8103051
:1034680004A803238DF811308DF812A08DF813E00D
:1034780087F8482028F05AFFA388B3FA83F3C3F1EA
:103488001F03BCE70E494B691A434A614FE70C49D1
:10349800CB691A43CA614AE709498B691A438A61A9
:1034A80045E700BF506103085C6103089C6103089D
:1034B800930500088822002000040140B832030860
:1034C80000100240586B002014040140040401401D
:1034D8001749184B184A194810B4D1F8884044F4D1
:1034E8007004C1F888401C6844F001041C605C68E2
:1034F80022405A601A6822F0847222F480321A60DC
:103508001A6822F480221A605A6822F4FE025A606D
:10351800DA6A22F00F02DA621A6B002410404FF0C8
:10352800006218639C608A605DF8044B704700BFB6
:1035380000ED00E0001002400CC07FF8CCFC00FF5A
:1035480038B50B4C23688BB15A68821A002A054695
:1035580004DA0CE05A68AA1A002A07DB9A68226083
:1035680018461A6890472368002BF3D138BD38BD38
:10357800304000200B4B002210B4027203F5A074F7
:10358800032102E0072A09DC9979890702D519790C
:10359800815401329C4203F11403F3D15DF8044BCA
:1035A800704700BFA461030810230370704700BF71
:1035B80030B40123022514241521222205724470F7
:1035C8004171C27003700371837030BC704700BFD3
:1035D8002C22022302704370704700BF436A82693D
:1035E800D154436A0169826B01338B4228BF00239F
:1035F8004362002A2FD0EFF31181502383F31288FE
:10360800836B1A68D2072CD470B45E686EB9456AA9
:10361800826A954217D084691444DC600ED9AA1ACC
:103628005A608562002280F854201A6842F001022C
:10363800C9B21A6081F3118870BC70470469A21A74
:103648005A608662EEE7012380F85430C9B281F3EC
:10365800118870BC7047026D136843F080031360D3
:103668007047C9B281F31188704700BF426B10B42C
:1036780062B1436CC2684469D11A013B615C5DF870
:10368800044B08BF13464364C8B27047016A4369D4
:10369800C4685B5C0131A14228BF114601625DF834
:1036A800044BD8B2704700BF836B13B190F8540035
:1036B8007047836A406A181AB0FA80F04009704768
:1036C800416A836A99420AD3CB1A816B026961B154
:1036D8004968501E0B4483420AD2C01A70470269D7
:1036E8001144CB1A816B0029F2D1501EC01A7047C1
:1036F80000207047436B43B1426C5B6893422FBF15
:10370800981AC0689B1AC0187047C269036A9A421F
:103718002FBFD01AC0688018C01A70470A4B30B53E
:1037280003F1140493F900205D78072AC8BF143AFE
:10373800811804330D7313F8025C855413F8012CB7
:103748000A76A342EED130BDD033030803682DE9D1
:10375800F041DF691FB13B46BDE8F0411847002A38
:10376800164611DD04460D460E4400E023689B68AA
:10377800204698470028F9D0236815F8011B1B68D4
:1037880020469847AE42F1D1BDE8F08100232322BC
:10379800027043708370C370704700BF2DE9F04713
:1037A8000569C3681D4028D00F4606464FF00048FB
:1037B8004FF00009B5FA85F328FA03F2D2431B3B10
:1037C80032611540042B16D8DFE803F0312921199E
:1037D80003007B6A002B32D003F1FF3A1FFA8AFA02
:1037E800C7F824903C6A34B123682046514698476C
:1037F8006468002CF8D1002DDCD1BDE8F08738686A
:10380800716B036889B29847002DD3D1F5E77868C2
:10381800B16B036889B29847002DCBD1EDE7B86842
:10382800F16B036889B29847002DC3D1E5E7F868C2
:10383800316C036889B29847002DBBD1DDE7F36A84
:103848001FFA83FACEE700BF30B50446006D6171F8
:103858000368A26823F00103036087B0A37900928C
:1038680013F004023DD04FF4805213F0020301928A
:1038780044D102934FF480630022039311F00103B3
:10388800059237D1049308238D07694648BF0493EE
:1038980028F01AFC6079236DA17900F00202002A51
:1038A80015BF4FF440324FF480324FF400340024F7
:1038B80010F0010F586808BF2246CC074CBF0243DE
:1038C80020EA02025A609A6809074CBF42F00802CF
:1038D80022F008029A601A6842F001021A6007B0E2
:1038E80030BD13F0020301920BD04FF4005513467C
:1038F8000295C1E7042304930C23C5E74FF4005352
:10390800B7E70293B8E700BF10B50446006DA160A1
:10391800036823F001030360A37986B013F004025F
:10392800009141D04FF4805213F00203019244D128
:1039380002934FF4806362790393D1074FF0000339
:103948000493059345BF0423049308230C23694675
:10395800920748BF049328F0B7FB6079236DA179DB
:1039680000F00202002A15BF4FF440324FF48032B3
:103978004FF40034002410F0010F586808BF2246A5
:10398800CC074CBF024320EA02025A609A68090732
:103998004CBF42F0080222F008029A601A6842F00E
:1039A80001021A6006B010BD13F00203019207D09D
:1039B8004FF4005113460291BDE74FF40053B7E7A7
:1039C8000293B8E7022828BF022010B4084C094B1C
:1039D800207000EB8002C0EBC20207495DF8044B7F
:1039E800013003EB4203C0B20B6010F0A9BA00BF6C
:1039F800FF540020443B0020C44F002008B517F0B6
:103A0800F7FFFDF703FCBDE8084017F0D9BF00BF7A
:103A18002DE9F04F013085B0C3B203938E4D8F4F1F
:103A28008F4C904E0A2302933220DFF8409224F004
:103A38007BFF4FF4FA7A4FF0100C4FF47A70D9F8F4
:103A48000430C3F30803002B40F0C880EFF3118360
:103A5800002B40F0C3802968A26800BF2B689942F8
:103A6800F9D1D7F800E000FB0EF39B1AB3FBFEF385
:103A780000FB01314FF0010E0191D9F80430C3F376
:103A88000803002B40F08E80EFF31183002B40F0E9
:103A980089802B68A16800BF2A689342F9D1D7F8BA
:103AA80000B000FB0BF2521AB2FBFBF200FB03233F
:103AB800019A9B1AB3F57A7FDFD3BAF1010ABED116
:103AC800039B002B40F0C4804FF47A7ADFF89C9176
:103AD80050464FF0100CD9F80430C3F30803002BFC
:103AE80040F09980EFF31183002B40F0948029680F
:103AF800A26800BF2B689942F9D1D7F800E000FB13
:103B08000EF39B1AB3FBFEF300FB01314FF0010EDD
:103B18000191D9F80430C3F308033BBBEFF31183D9
:103B280023BB2B68A16800BF2A689342F9D1D7F854
:103B380000B000FB0BF2521AB2FBFBF200FB0323AE
:103B4800019A9B1AB3F57A7FE3D3BAF1010AC2D17D
:103B5800029B013B02937FF467AF4349434B4448C0
:103B6800444A0860DA6005B0BDE8F08FEFF31188C9
:103B78008CF31288A1682368DB0344BFC6F800E011
:103B8800A1682B6832685FFA88F888F31188D7F83B
:103B980000801A4400FB08F35B1AB3FBF8F300FB40
:103BA8000233CDE7EFF311888CF31288A1682368FC
:103BB800DB0344BFC6F800E0A1682B6832685FFAEF
:103BC80088F888F31188D7F800801A4400FB08F3B6
:103BD8005B1AB3FBF8F300FB023369E7EFF31182DA
:103BE8008CF31288D4F808E02368D90303D501239D
:103BF8003360D4F808E02B683168D2B282F31188B8
:103C08003A68194400FB02F3A3EB0E03B3FBF2F38B
:103C180000FB01312EE7EFF311828CF31288D4F800
:103C280008E02368D90303D501233360D4F808E0FA
:103C38002B683168D2B282F311883A68194400FBC4
:103C480002F3A3EB0E03B3FBF2F300FB01315DE7D4
:103C580018462AF0C9FB37E7F0750020F4750020F4
:103C680010E000E0EC750020FC9F002000ED00E073
:103C7800EFBEADDE0400FA0538B5434B5A89998981
:103C8800914224BF00225A81198ADA89914224BFBD
:103C98000022DA81DA788AB3072A2FD03B493C4DD3
:103CA80091F85300012400210A282C709C70D971C6
:103CB8003DD00C2865D0DFED377A8ABB364C9FEDB6
:103CC800370AA278002918BFF0EE407A062A04D8ED
:103CD800334901EB820191ED050A217959B3013A83
:103CE800032A4DD8F7EE007A87EE800A2EF0B4FA50
:103CF8002388984228BF1846208038BDD97921B139
:103D080098780428B8BF04209870204890F8530089
:103D18000A280CD00C28CED1DFED227A002ACDD08B
:103D2800072ACBD00A282CD1DFED1F7AC6E70A2054
:103D3800DFED1E7AC1E79B78154A07EE103A117835
:103D4800B8EEC77A27EE277A07EE901AF8EEE77AE8
:103D580067EE877AB4EEE70AF1EE10FA10DDC0EEEE
:103D6800077AFDEEE77A17EE903A102BA8BF1023DA
:103D7800012BB8BF0123DBB28B4238BF0B4613704F
:103D880038BDDFED0B7A99E7906C0020A46C002019
:103D9800046000206F1203392C7100206F12033861
:103DA800D03303080AD7A3390F506E3A5304E938C1
:103DB8006F12833A2DE9F047A64FA74E17F018FE69
:103DC800BE421ED2DFF80C83DFF80C9344462588E8
:103DD80062197DB14A450DD2052D0BD9338861880A
:103DE800C3F30B03994200F0DA8014462588621960
:103DF800002DEFD1716830461436FDF793F9BE42B5
:103E0800E4D3964A1378A3F1170102290FD99449EC
:103E180011F83300002840F0EE80D80001444978BA
:103E280029B1904911F83330002B00F00C818E4BEA
:103E38005A78022A40F2D98000228C495A701A789E
:103E48008B48022A016000F2CC8002EB8201894B88
:103E5800C2EBC10203EB4203998C5A8C864C914207
:103E6800236001D300225A84844B9A78042A00F0F4
:103E7800E18032B91A88B2F5F07F84BF4FF4F0724E
:103E88001A807F4DFFF7F8FE2B687E4A1A40002AF9
:103E980000F0DC80D80700F1C880590400F1C08028
:103EA8001A0700F1B8809B0400F1AE8025F0BAFD36
:103EB80010B975480EF05EFF8020FDF769F94FF4E0
:103EC8000070FDF765F94FF40010FDF761F94FF048
:103ED8000070FDF75DF94FF08060FDF759F913F0B8
:103EE80051FC0021302269482FF073F9206812F044
:103EF8004BFB674B276803F1500102E004339942FA
:103F08006DD01A78002AF9D19C78D8788442F5D2F5
:103F18006049614B0D79614961480A70614E624C94
:103F28000460C822642111FB0521002259609A60AF
:103F3800DA601A615A619A61DA6183F8202083F89D
:103F4800212037601BF036FD584B9FED595A1B88CE
:103F5800584A9FED596A5079584906EE903AF8EE5A
:103F6800E66A1388C5EE265A07EE103A5388127986
:103F7800C1ED005A07EE903AB8EEC77A504BF8EE0A
:103F8800E77A18725A7227EE067A67EE867ABDE8E3
:103F9800F04783ED017AC3ED007A17F011BD63791C
:103FA8009B077FF422AF716894F804A03046FDF7B0
:103FB800B9F83388BAEB133F04D01436BE42FFF485
:103FC80005AF1EE773887068AA1FC3F30B039A42F4
:103FD80004F10601A8BF1A462DF06AFFEDE7012299
:103FE80096E700221A70234B36E7204902EB42027B
:103FF80001EB820123E7D8000C186468002C7FF4D9
:104008000DAF1724147009E72E48FDF7C1F84020BA
:10401800FDF7BEF84AE72C48FDF7BAF82B6842E7E7
:104028002A48FDF7B5F82B683AE72948FDF7B0F8B4
:104038002B6832E79A8AB2F57A7FBFF422AF4FF441
:104048007A729A821DE718231370F0E643F0010391
:104058002B601FE774A10308009D03080C4800208B
:10406800285E0308785C0308FF540020E84A002013
:10407800C84F0020443B0020C44F00202C71002072
:10408800743C002009600002485D0020D423002011
:104098009440002088390020244B0020AC200020C8
:1040A8001824002008240020166000201026002074
:1040B800C0C9FB484424002017B7D1381426002073
:1040C8008837002009400002016000020920000230
:1040D8000860000202F003080000040808B517F0A1
:1040E80087FCFDF793F817F06BFCFFF763FE0120E0
:1040F800BDE808400FF024BF38B50C4C0C4DAC425D
:1041080006D2616820461434FDF70CF8AC42F8D3A7
:10411800084A094B094C1460002209491A705A7060
:1041280008480860BDE838401CF0C8BA009D03087C
:1041380074A10308C44F0020FF540020443B002012
:10414800C84F0020E84A002008B5FFF7D5FF17F050
:104158004FFCFDF75BF8BDE8084017F031BC00BF25
:10416800F0B50C292BD8DFE801F06F2A2A2A4C2A4F
:104178002A2A2B2A2A2A0700046AB2F80CE0978810
:104188001668674D24F480540462036A4468C16960
:1041980023F4005343EA0E3321F4E641A84243EAEC
:1041A800073341EA062100F0B58005F50065A8420D
:1041B80000F0B08092684460C16102640362F0BD9F
:1041C800046A96899588D2F800E0554F24F48074E3
:1041D8000462036A4468C16923F4007343EA06234E
:1041E80021F07301B84243EA052341EA0E017ED06B
:1041F8004C4DA8427BD092684460C161C26303629F
:10420800F0BD046A96899588D2F800E0444F24F0FE
:1042180010040462036A4468816923F0200321F0D2
:10422800807143EA061321F4E641B84243EA0513D4
:1042380041EA0E2148D03B4DA84245D092684460DF
:10424800816182630362F0BD046A9389B2F804E075
:104258001768334E24F001040462056A44688169D2
:1042680043EA0E0321F4803125F002059BB221F0C8
:104278007301B04243EA050341EA070114D0294D0E
:10428800A84211D005F54065A8420DD005F5806516
:10429800A84209D005F58065A84205D09268446017
:1042A800816142630362F0BDD689158A578A23F07B
:1042B800080333433D43D68824F4407423F00403B1
:1042C800ADB233432C43E9E7D589178AD68823F062
:1042D800800343EA051324F44064558A23F040031D
:1042E80044EA870443EA061344EA8504A6E7D58925
:1042F800178AD68823F4006343EA052324F440543C
:10430800558A23F4806344EA071443EA062344EAFF
:10431800051470E7158A24F4804444EA851449E7B3
:10432800002C0140003401402DE9F84F4FF48C7205
:1043380000218248824C834D834E844FDFF82882C7
:10434800DFF828922EF045FF81488249DFF820E205
:10435800DFF820C200221359834200F0C380B3F172
:10436800804F00F0D580AB4200F0D980B34200F016
:10437800D880BB4200F0D780734500F0D6806345F3
:1043880000F0A680434500F0D2804B4500F0D28073
:10439800DFF8E4A1534508BF4FF4802300F09A806A
:1043A8001432B2F5AA7FD6D1654D6B4F6B4E05F529
:1043B800AA784FF0030A4FF0020903E01435454587
:1043C80000F08E80AB79002BF8D02B791C09013CCA
:1043D800052C03F00F03F1D837F8140040FA03F264
:1043E800D207EBD54FF0010B0BFA03F3013B184052
:1043F8002DF080FB5A4B1B5D184416EBC004DDD032
:1044080056F830305748297A03F13842920A825CCC
:1044180002F01F005209022A0BFA00FB71D0032A8E
:1044280068D0012A05D14B4A4A4852694BEA020230
:104438004261B4F804E0BEFA8EF2C2F11F0292B2F1
:10444800D00803EB800002F00702046A92004FF0E4
:104458000F0C0CFA02FC24EA0C040462046A01FA48
:1044680002F22243002402624FF0010C224603E0CC
:10447800102A04F10204A1D00CFA02F030EA0E016D
:1044880002F10102F4D1D3F808B00AFA04F1C943E1
:104498000BEA010BC3F808B0D3F808B0C3F808B0AA
:1044A800B3F804B01FFA8BFB2BEA000098809888B9
:1044B80080B29880186808401860D3F800B009FAEC
:1044C80004F040EA0B001860D8680140D960CFE7D3
:1044D8004FF40053D1F818A043EA0A038B615FE751
:1044E800BDE8F88FD1F818A04FF4006343EA0A0337
:1044F8008B6155E7174A1748D2694BEA0202C26135
:1045080097E7144A134892694BEA0202826190E7DE
:104518000123D1F81CA043EA0A03CB6140E7022338
:10452800F7E70423F5E71023F3E72023F1E74FF437
:104538008033CFE74FF40033CCE700BF1C420020A4
:10454800A461030800040040000800400010004077
:10455800002C01400010024050610308586B0020F5
:104568005C6103089C61030800400140004401406D
:10457800001400400034014000480140002867D082
:1045880003682DE9F04F03F138445C4EA40A012575
:10459800345D04F01F066409022C05FA06F558D0AC
:1045A800032C00F0A580012C58D08088B0FA80F444
:1045B800C4F11F04A4B2E50803EB850504F0070461
:1045C8002E6AA4000F27A74026EA07062E622E6A45
:1045D80001F00307A2407C1E3243012CC1F3810C79
:1045E800C1F300182A62C1F341113CD9C60700F192
:1045F8008980850700F19580440700F1A3800207B0
:1046080000F1B180C60600F1BF80850600F1CD80BB
:10461800440600F1DB80020600F1E980C60500F1DE
:10462800F780850500F10581440500F11381020535
:1046380000F12181C60400F12F81850400F13D813C
:10464800440400F14B81020400F15981BDE8F08F68
:1046580070472B4CA6693543A561A6E7284C6669C7
:1046680035436561A1E7002422464FF0010E4FF063
:10467800030904E00132102A04F10204E6D00EFA1C
:1046880002F636EA0005F5D1D3F808A009FA04F5D0
:10469800ED430AEA050AC3F808A0D3F808B00CFAF3
:1046A80004FA4AEA0B0AC3F808A0B3F804A01FFAF0
:1046B8008AFA2AEA06069E80B3F804A008FA02F6E7
:1046C80046EA0A06B6B29E801E682E401E60D3F8DF
:1046D80000A007FA04F646EA0A061E60D3F80CA002
:1046E80001FA04F605EA0A0A46EA0A05DD60C1E7A6
:1046F800034CE6693543E56157E700BF9C61030851
:10470800001002401A6822F003021A601A683A433D
:104718001A60DA6822F003020A438507DA607FF537
:104728006BAF1A6822F00C021A601A6842EA870214
:104738001A60DA6822F00C0242EA81024407DA6061
:104748007FF55DAF1A6822F030021A601A6842EAF3
:1047580007121A60DA6822F0300242EA0112DA60BF
:1047680002077FF54FAF1A6822F0C0021A601A6874
:1047780042EA87121A60DA6822F0C00242EA81121D
:10478800C606DA607FF541AF1A6822F440721A60F3
:104798001A6842EA07221A60DA6822F4407242EA8A
:1047A80001228506DA607FF533AF1A6822F4406289
:1047B8001A601A6842EA87221A60DA6822F44062AC
:1047C80042EA81224406DA607FF525AF1A6822F4AE
:1047D80040521A601A6842EA07321A60DA6822F40C
:1047E800405242EA0132DA6002067FF517AF1A68D2
:1047F80022F440421A601A6842EA87321A60DA687C
:1048080022F4404242EA8132C605DA607FF509AFF8
:104818001A6822F440321A601A6842EA07421A609B
:10482800DA6822F4403242EA01428505DA607FF50F
:10483800FBAE1A6822F440221A601A6842EA8742DC
:104848001A60DA6822F4402242EA81424405DA60BA
:104858007FF5EDAE1A6822F440121A601A6842EA2F
:1048680007521A60DA6822F4401242EA0152DA600A
:1048780002057FF5DFAE1A6822F440021A601A6852
:1048880042EA87521A60DA6822F4400242EA815208
:10489800C604DA607FF5D1AE1A6822F040721A6059
:1048A8001A6842EA07621A60DA6822F0407242EA3D
:1048B80001628504DA607FF5C3AE1A6822F04062AF
:1048C8001A601A6842EA87621A60DA6822F040625F
:1048D80042EA81624404DA607FF5B5AE1A6822F0D4
:1048E80040521A601A6842EA07721A60DA6822F0BF
:1048F800405242EA0172DA6002047FF5A7AE1A68F4
:1049080022F040421A601A6842EA87771F60DA6824
:1049180022F0404242EA8171D960BDE8F08F00BFC1
:1049280003682DE9F04F03F13845644EAD0A0124C0
:10493800755D05F01F066D09022D04FA06F400F0F6
:10494800A280032D00F0A480012D52D08088B0FAF7
:1049580080F4C4F11F04A4B2E50803EB850504F054
:1049680007042E6AA4000F27A74026EA07062E622E
:104978002E6A01F0030702FA04F47A1E3443012A6E
:10498800C1F3810CC1F300182C62C1F3411135D970
:10499800C60700F19780850700F1A380440700F15E
:1049A800B180020700F1BF80C60600F1CD80850600
:1049B80000F1DB80440600F1E980020600F1F7808F
:1049C800C60500F10581850500F11381440500F154
:1049D8002181020500F12F81C60400F13D81850483
:1049E80000F14B81440400F15981020455D4BDE81B
:1049F800F08F334D6E6934436C61A7E7002422467B
:104A08004FF0010E4FF0030904E00132102A04F1BF
:104A18000204ECD00EFA02F636EA0005F5D1D3F816
:104A280008A009FA04F5ED430AEA050AC3F808A044
:104A3800D3F808B00CFA04FA4AEA0B0AC3F808A03B
:104A4800B3F804A01FFA8AFA2AEA06069E80B3F889
:104A580004A008FA02F646EA0A06B6B29E801E6864
:104A68002E401E60D3F800A007FA04F646EA0A06AC
:104A78001E60D3F80CA001FA04F605EA0A0A46EA11
:104A88000A05DD60C1E70E4DAE693443AC615DE7F0
:104A98000B4DEE693443EC6158E71A6822F0404246
:104AA8001A601A6842EA87771F60DA6822F0404283
:104AB80042EA8171D960BDE8F08F00BF9C610308AC
:104AC800001002401A6822F003021A601A683A437A
:104AD8001A60DA6822F003020A438507DA607FF574
:104AE8005DAF1A6822F00C021A601A6842EA87025F
:104AF8001A60DA6822F00C0242EA81024407DA609E
:104B08007FF54FAF1A6822F030021A601A6842EA3D
:104B180007121A60DA6822F0300242EA0112DA60FB
:104B280002077FF541AF1A6822F0C0021A601A68BE
:104B380042EA87121A60DA6822F0C00242EA811259
:104B4800C606DA607FF533AF1A6822F440721A603D
:104B58001A6842EA07221A60DA6822F4407242EAC6
:104B680001228506DA607FF525AF1A6822F44062D3
:104B78001A601A6842EA87221A60DA6822F44062E8
:104B880042EA81224406DA607FF517AF1A6822F4F8
:104B980040521A601A6842EA07321A60DA6822F448
:104BA800405242EA0132DA6002067FF509AF1A681C
:104BB80022F440421A601A6842EA87321A60DA68B8
:104BC80022F4404242EA8132C605DA607FF5FBAE44
:104BD8001A6822F440321A601A6842EA07421A60D8
:104BE800DA6822F4403242EA01428505DA607FF54C
:104BF800EDAE1A6822F440221A601A6842EA874227
:104C08001A60DA6822F4402242EA81424405DA60F6
:104C18007FF5DFAE1A6822F440121A601A6842EA79
:104C280007521A60DA6822F4401242EA0152DA6046
:104C380002057FF5D1AE1A6822F440021A601A689C
:104C480042EA87521A60DA6822F4400242EA815244
:104C5800C604DA607FF5C3AE1A6822F040721A60A3
:104C68001A6842EA07621A60DA6822F0407242EA79
:104C780001628504DA607FF5B5AE1A6822F04062F9
:104C88001A601A6842EA87621A60DA6822F040629B
:104C980042EA81624404DA607FF5A7AE1A6822F01E
:104CA80040521A601A6842EA07721A60DA6822F0FB
:104CB800405242EA0172DA6097E600BF10B5040973
:104CC800013C052C17D80D4B33F8142000F00F00C9
:104CD80042FA00F313F001030DD0012303FA00F0A8
:104CE800013810402CF006FF054A064B125D1044AF
:104CF80003EBC00010BD002010BD00BF50610308C9
:104D08005C610308586B002001490248FEF746BD64
:104D18000C4300200048014001490248FEF73EBD0F
:104D2800BC4200200040014001490248FEF736BD60
:104D3800944200200008004001490248FEF72EBDB9
:104D48006C4200200004004002494FF08040FEF70A
:104D580025BD00BF4442002010B5064C0648214638
:104D6800FEF71CFD04F1C8010448BDE81040FEF739
:104D780015BD00BF1C420020002C0140004401402A
:104D880001490248FEF70ABD1C420020002C0140E0
:104D98002DE9F0410468514DA30AAB4200F084802C
:104DA8000AD94F4DAB4277D00135AB425FD0023DB7
:104DB800AB426DD0BDE8F0814A3DAB4270D00135C1
:104DC800AB4258D0B3F5801FF4D14FF0480E0126FE
:104DD80047794FEA970C00296AD0B00063468519D5
:104DE8000227D4F80C809F400CEB4503BFB23D4D21
:104DF80003F1040C47EA080745F8231045F82C206E
:104E0800E760EFF31181502282F31288821905EBD3
:104E1800C2021369002B32D013620433821905EBE6
:104E2800C202576917B11F6053690433821905EB31
:104E3800C202976917B11F6093690433821905EBA1
:104E4800C202D76917B11F60D36904330027CAB2F9
:104E58001F6082F31188304405EBC000036A8BB9E8
:104E6800E3684FF6FE721340E360BDE8F0814FF44B
:104E7800887E0626ACE74FF0980E0326A8E705EBD8
:104E88000E03CBE7E36843F00103E360BDE8F0817C
:104E98004FF0C00E04269BE74FF0E80E052697E773
:104EA8004FF0700E022693E74FF0200E00268FE792
:104EB800BF08022306FA03F0BB40DB43E768094D4D
:104EC8009BB23B4087190CEB470CE3600CF10403E1
:104ED80045F82C1045F8232093E700BF4B0010003D
:104EE800510010001C42002030B503685C4D188842
:104EF8005C4CB4FBF2F20139013AAB4294B283B094
:104F080089B282B266D05848834263D0B3F1804FE9
:104F180060D0A0F5983083425CD000F58060834271
:104F280058D0524883425BD000F5806083427DD0E0
:104F380022F4407200F58C3092B283421A80D96212
:104F48001C850ED0484A93420BD002F5406293422A
:104F580007D002F58062934203D002F58062934243
:104F680001D100221A8601225A611A883C4992B25C
:104F780042F001028B421A8062D0B3F1804F61D0B7
:104F88003B4A934260D002F5806293425ED002F5BC
:104F9800006293425CD002F5806293425AD002F5D7
:104FA8009032934258D002F54062934256D002F5AF
:104FB800806293421ED002F58062934208BF0922A4
:104FC80019D002A84FF0012340F8043D27F0AEF9AC
:104FD80003B030BD254822F07002834292B2A3D1BB
:104FE80001201A80D9621C8558611A8892B202433E
:104FF8001A80C5E708221F4B03EBC20301A893F8E8
:1050080035408DF80440012300228DF805308DF8D5
:1050180007308DF8062027F089F91B2CD8D1164BBC
:10502800019301A827F082F903B030BD01201A804E
:10503800D9621C8558611A8892B202431A809CE78B
:105048000022D8E70122D6E70222D4E70322D2E7DA
:105058000422D0E70522CEE70622CCE70722CAE7DA
:10506800002C014000A24A04003401400010004016
:1050780000040040D033030819010001204B984276
:105088002DD0B0F1804F2CD0A3F5943398422AD07C
:1050980003F58063984228D003F50063984226D030
:1050A80003F58063984224D003F59033984222D0C8
:1050B80003F54063984220D003F58063984207D0F7
:1050C80003F58063984208BF092202D00020704788
:1050D80008220C4B03EBC20393F8340070470022FC
:1050E800F7E70122F5E70222F3E70322F1E70422BA
:1050F800EFE70522EDE70622EBE70722E9E700BF25
:10510800002C0140D03303082DE9F04F013085B061
:10511800C3B203930B4602918B4C8C4E002B00F0CC
:105128009A8032208A4D8B4FDFF82C9223F0FCFBBB
:105138004FF4FA7A4FF0100C4FF47A70D9F8043023
:10514800C3F30803002B40F0DE80EFF31183002B3C
:1051580040F0D9802968A26800BF2B689942F9D12C
:10516800D7F800E000FB0EF39B1AB3FBFEF300FB3D
:1051780001314FF0010E0191D9F80430C3F308034F
:10518800002B40F08780EFF31183002B40F08280E2
:105198002B68A16800BF2A689342F9D1D7F800B0FC
:1051A80000FB0BF2521AB2FBFBF200FB0323019A3D
:1051B8009B1AB3F57A7FDFD3BAF1010ABED1039BFC
:1051C800002B40F0BD804FF47A7ADFF88C9150467E
:1051D8004FF0100CD9F80430C3F30803002B75D135
:1051E800EFF31183002B71D12968A26800BF2B68E7
:1051F8009942F9D1D7F800E000FB0EF39B1AB3FBF4
:10520800FEF300FB01314FF0010E0191D9F8043093
:10521800C3F3080313BBEFF31183FBB92B68A16831
:1052280000BF2A689342F9D1D7F800B000FB0BF20F
:10523800521AB2FBFBF200FB0323019A9B1AB3F547
:105248007A7FE3D3BAF1010AC4D1029B013B0293EE
:10525800002B7FF466AF05B0BDE8F08FEFF311883F
:105268008CF31288A1682368DB0344BFC6F800E00A
:10527800A1682B6832685FFA88F888F31188D7F834
:1052880000801A4400FB08F35B1AB3FBF8F300FB39
:105298000233D2E7EFF311888CF31288A1682368F0
:1052A800DB0344BFC6F800E0A1682B6832685FFAE8
:1052B80088F888F31188D7F800801A4400FB08F3AF
:1052C8005B1AB3FBF8F300FB023370E7EFF31182CC
:1052D8008CF31288D4F808E02368D90303D5012396
:1052E8003360D4F808E02B683168D2B282F31188B1
:1052F8003A68194400FB02F3A3EB0E03B3FBF2F385
:1053080000FB01317FE7EFF311828CF31288D4F8A8
:1053180008E02368D90303D501233360D4F808E0F3
:105328002B683168D2B282F311883A68194400FBBD
:1053380002F3A3EB0E03B3FBF2F300FB013118E712
:10534800184629F051F83EE710E000E0EC7500201F
:10535800F0750020F475002000ED00E0204B5B683C
:10536800C3F3080330B4BBB9EFF31183A3B91D4BE2
:105378001D4C1868A16800BF1A689042F9D11B4BF0
:105388001C684FF47A7202FB04F3591AB1FBF4F16A
:1053980030BC02FB00107047EFF31182102383F337
:1053A800128811498C680B6813F4803F104B02D0A7
:1053B800012018608C680B49D2B20D68186882F316
:1053C80011880A4B19684FF47A72284402FB01F3DA
:1053D8001B1B30BCB3FBF1F302FB0030704700BF6E
:1053E80000ED00E0F075002010E000E0F47500200A
:1053F800EC7500202DE9F84F8046FFF7AFFF254EEA
:105408002549DFF8A0E0254A254D844610274FF4AA
:105418007A740120DEF80430C3F30803D3B9EFF33C
:105428001183BBB90B68D2F808A000BFD1F800906F
:105438004B45F7D1D6F800B004FB0BF9A9EB0A09E4
:10544800B9FBFBF904FB0393A3EB0C034345E1D33E
:10545800BDE8F88FEFF3118A87F31288D2F808B005
:105468001368DB0344BF2860D2F808B00B68D5F88E
:1054780000905FFA8AFA8AF31188D6F800A0994456
:1054880004FB0AF3A3EB0B03B3FBFAF304FB0933A6
:10549800DAE700BFF4750020F075002010E000E0A6
:1054A800EC75002000ED00E02DE9F04FDFF830C189
:1054B800474A4849484E494D8046102718F1FF3859
:1054C800C0F08480DCF80430C3F30803002B5CD1FF
:1054D800EFF31183002B58D10B68946800BF08685C
:1054E8008342F9D1D6F800904FF47A7000FB09FE98
:1054F800AEEB040EBEFBF9FE00FB03EEDCF8043055
:10550800C3F308034FF47A740120FBB9EFF3118356
:10551800E3B90B68D2F808A000BFD1F800904B455A
:10552800F7D1D6F800B004FB0BF9A9EB0A09B9FBCF
:10553800FBF904FB0393A3EB0E03B3F57A7FBDD20B
:10554800DCF80430C3F30803002BDFD0EFF3118A33
:1055580087F31288D2F808B01368DB0344BF2860C9
:10556800D2F808B00B68D5F800905FFA8AFA8AF387
:105578001188D6F800A0994404FB0AF3A3EB0B03A7
:10558800B3FBFAF304FB0933D5E7EFF3118487F390
:105598001288D2F808901368D80303D501232B602A
:1055A800D2F808900B682868E4B284F31188D6F81A
:1055B80000A04FF47A7400EB030E04FB0AF3A3EB8C
:1055C8000903B3FBFAF304FB0E3E97E7BDE8F08F3F
:1055D80010E000E0F0750020F4750020EC75002064
:1055E80000ED00E030B4EFF31183102282F312884B
:1055F8000649074C0A680748013200250A602560F9
:10560800DBB2026883F3118830BC7047F075002064
:10561800EC75002010E000E00F4B1B88014643B9F1
:105628000E4B0F4A1B7810680BB981F00101FBF78C
:105638006EBB0C4B5A691AB118B91A6810605874C5
:105648007047094A18681188084A92FBF1F201214B
:1056580002605974704700BFC8750020CA750020E1
:10566800CC750020D0750020E875002020A1070027
:105678001D4B70B59C68236D626BDD69C2B1A36B6D
:105688002BB12B0702D5236D08221A6270BD2A069A
:10569800F7D5A26A616A8A4220D0511CA069A1622A
:1056A800825C2069266D81423285EAD3A362E8E7ED
:1056B800A906E4D5E26A22B1988C216B80B29047A2
:1056C800DDE7E1699B8C6069DBB24E1CE6614354FF
:1056D800E169E368994228BFE261D0E7226D136867
:1056E80023F080031360CCE7943600201D4B70B57F
:1056F8005C68236D626BDD69C2B1A36B2BB12B07AC
:1057080002D5236D08221A6270BD2A06F7D5A26A4F
:10571800616A8A4220D0511CA069A162825C20691A
:10572800266D81423285EAD3A362E8E7A906E4D56B
:10573800E26A22B1988C216B80B29047DDE7E1697B
:105748009B8C6069DBB24E1CE6614354E169E368F7
:10575800994228BFE261D0E7226D136823F08003E5
:105768001360CCE7943600201D4B70B51C68236D80
:10577800626BDD69C2B1A36B2BB12B0702D5236D18
:1057880008221A6270BD2A06F7D5A26A616A8A429F
:1057980020D0511CA069A162825C2069266D8142DB
:1057A8003285EAD3A362E8E7A906E4D5E26A22B122
:1057B800988C216B80B29047DDE7E1699B8C60692A
:1057C800DBB24E1CE6614354E169E368994228BFA5
:1057D800E261D0E7226D136823F080031360CCE701
:1057E8009436002070B4EFF31186502383F31288A7
:1057F800836B1A68D20720D45D686DB9446A826ADF
:10580800944217D081691144D9600ED9A21A5A60FE
:105818008462002280F854201A6842F00102F1B232
:105828001A6081F3118870BC704701698A1A5A603E
:105838008562EEE7012380F85430F1B281F31188D4
:1058480070BC704703685B6A03B11847704700BFB4
:1058580003681B6A03B11847704700BF03682DE946
:10586800F041DF691FB13B46BDE8F0411847002A07
:10587800164611DD04460D460E4400E023689B6879
:10588800204698470028F9D0236815F8011B1B68A3
:1058980020469847AE42F1D1BDE8F08103689B6984
:1058A800184700BF03685B69184700BF0368DB68D7
:1058B800184700BF03689B68184700BF03685B6808
:1058C800184700BF03681B68184700BF10B40B4B8C
:1058D8000B4A1C7801238340234052F8200031B939
:1058E800B3FA83F149095DF8044BFBF710BA191CA8
:1058F80018BF01215DF8044BFBF709BAB875002001
:10590800BC75002008B501210220FFF7DFFF094B15
:105918001B7803F00503052B08D000210120FFF7B1
:10592800D5FF00210846FFF7D1FFFEE711F0C6F9C1
:10593800F3E700BF90360020054B53F8203033B111
:105948001A689B88918A0B4218BF1B0493617047A1
:10595800BC750020036803F138422DE9F04F920A24
:10596800584DAA5C02F01F0552090124022A04FAC4
:1059780005F400F08C80032A00F08E80012A3CD0C8
:1059880001F003077A1E012AC1F3810CC1F3001844
:105998008088C1F3411135D9C60700F19780850782
:1059A80000F1A380440700F1B180020700F1BF8035
:1059B800C60600F1CD80850600F1DB80440600F1C3
:1059C800E980020600F1F780C60500F1058185052A
:1059D80000F11381440500F12181020500F12F81B6
:1059E800C60400F13D81850400F14B81440400F1B7
:1059F8005981020455D4BDE8F08F334A55692C43C8
:105A08005461BDE7002422464FF0010E4FF0030910
:105A180004E00132102A04F10204ECD00EFA02F676
:105A280036EA0005F5D1D3F808A009FA04F5ED43E4
:105A38000AEA050AC3F808A0D3F808B00CFA04FA71
:105A48004AEA0B0AC3F808A0B3F804A01FFA8AFAB6
:105A58002AEA06069E80B3F804A008FA02F646EA87
:105A68000A06B6B29E801E682E401E60D3F800A0BB
:105A780007FA04F646EA0A061E60D3F80CA001FAF3
:105A880004F605EA0A0A46EA0A05DD60C1E70E4A95
:105A980095692C43946173E70B4AD5692C43D4610B
:105AA8006EE71A6822F040421A601A6842EA87775D
:105AB8001F60DA6822F0404242EA8171D960BDE88D
:105AC800F08F00BF9C610308001002401A6822F0A2
:105AD80003021A601A683A431A60DA6822F003026D
:105AE8000A438507DA607FF55DAF1A6822F00C0279
:105AF8001A601A6842EA87021A60DA6822F00C0211
:105B080042EA81024407DA607FF54FAF1A6822F053
:105B180030021A601A6842EA07121A60DA6822F03C
:105B2800300242EA0112DA6002077FF541AF1A68D3
:105B380022F0C0021A601A6842EA87121A60DA680C
:105B480022F0C00242EA8112C606DA607FF533AF5E
:105B58001A6822F440721A601A6842EA07221A6028
:105B6800DA6822F4407242EA01228506DA607FF59B
:105B780025AF1A6822F440621A601A6842EA87223E
:105B88001A60DA6822F4406242EA81224406DA6046
:105B98007FF517AF1A6822F440521A601A6842EA71
:105BA80007321A60DA6822F4405242EA0132DA60B7
:105BB80002067FF509AF1A6822F440421A601A6893
:105BC80042EA87321A60DA6822F4404242EA8132B5
:105BD800C605DA607FF5FBAE1A6822F440321A6017
:105BE8001A6842EA07421A60DA6822F4403242EA46
:105BF80001428505DA607FF5EDAE1A6822F440228D
:105C08001A601A6842EA87421A60DA6822F4402267
:105C180042EA81424405DA607FF5DFAE1A6822F471
:105C280040121A601A6842EA07521A60DA6822F4C7
:105C3800401242EA0152DA6002057FF5D1AE1A68D5
:105C480022F440021A601A6842EA87521A60DA6837
:105C580022F4400242EA8152C604DA607FF5C3AEFC
:105C68001A6822F040721A601A6842EA07621A60DB
:105C7800DA6822F0407242EA01628504DA607FF550
:105C8800B5AE1A6822F040621A601A6842EA876262
:105C98001A60DA6822F0406242EA81624404DA60FB
:105CA8007FF5A7AE1A6822F040521A601A6842EAD5
:105CB80007721A60DA6822F0405242EA0172DA602A
:105CC80097E600BF2DE9F04F4A484B4B4B4C4FF03D
:105CD80090414FF0010A4FF002094FF004084FF0CD
:105CE800080C4FF0100E20274026802530F8022B94
:105CF80012F0010F03D01960A3F804A0083312F0C2
:105D0800020F03D01960A3F80490083312F0040FAF
:105D180003D01960A3F80480083312F0080F03D0E9
:105D28001960A3F804C0083312F0100F03D01960EB
:105D3800A3F804E0083312F0200F02D019609F8006
:105D4800083312F0400F02D019609E80083312F019
:105D5800800F02D019609D80083312F4807F05D02F
:105D68004FF4807B1960A3F804B0083312F4007F65
:105D780005D04FF4007B1960A3F804B0083312F47F
:105D8800806F05D04FF4806B1960A3F804B0083316
:105D980012F4006F05D04FF4006B1960A3F804B03B
:105DA800083312F4805F05D04FF4805B1960A3F8C4
:105DB80004B0083312F4005F05D04FF4005B19609B
:105DC800A3F804B0083312F4804F05D04FF4804B89
:105DD8001960A3F804B00833D20B04D04FF4004282
:105DE80019609A80083301F58061A1427FF47EAF83
:105DF800BDE8F08F50610308586B00200018004878
:105E08002DE9F04FC04B1E788BB0002E40F0BC80BF
:105E1800BE4BBF4C1D78DFF818A3DFF81893DFF8E6
:105E2800188305F00105A4F10A0B54F80A3CBBB12C
:105E3800CC2707FB06B71846FFF740FD80B154F89A
:105E48000A0CFFF733FD14F8023C8BB9242831D033
:105E5800F5B154F80A3C1846FFF730FD0028EED19A
:105E68000136032E04F1CC04DFD10BB0BDE8F08F6E
:105E7800012B23D0022B2BD0032B37D0042B67D038
:105E8800052B40D0062B4FD054F80A2C1346D2E7E6
:105E980054F80A3C23281A4600F089819D4991F854
:105EA8002A108142C7D19C4BCAF80090C3F80C80D5
:105EB8001346C0E7012304F8023CCAE74D2854F80A
:105EC8000A2C0CBF0223002304F8023C1346B2E755
:105ED80000233C2804F8023C45D03E28D4D10122B6
:105EE800032304F8012C04F8023CB2E7C02814D8B4
:105EF8000022042304F8050C04F8040C04F8062C0A
:105F080004F8023CA5E714F8063C14F8052C9A425C
:105F18002FD814F8043C834203D0002304F8023C31
:105F280097E7062304F8023C14F801ECBEF1000FD1
:105F380000F08081BEF1010F00F0C481013600231A
:105F4800032E04F8023C04F1CC047FF46EAF8CE716
:105F580014F8043C04F8030C5840052304F8040C16
:105F680004F8023C75E7032204F8013C04F8022C0B
:105F78006FE714F8042CF9184240013304F8042C94
:105F880004F8063C887264E7644B186800283FF4FC
:105F98006CAFFBF773F8DFF8A4A1614DDFF8A091AF
:105FA800DAF80000FFF78AFC00283FF45EAFDAF861
:105FB8000000FFF77BFC09281BD03F2819D02B686D
:105FC800002B67D1042800F0AB810C2800F0E88092
:105FD8007F28E5D0A0F12002D2B25E2AE0D80BB922
:105FE8002028DDD05A1C09F803002A6021F0A8FBFC
:105FF800D6E72C68002C5BD14A4FA34607F5987862
:10600800BBF1000F08BFBB4608374745F8D1BBF1C5
:10601800000F00F07A81083FDBF800003A68065D5F
:10602800135D9E42204402EB040140F06C81661E21
:106038004E4422460BB9FD2A5DD906F8013F0132CC
:106048002A6010F8013F11F801EF9E45F2D00AB11D
:106058005F4512D0344821F07BFB5F4508D35BF8DD
:10606800080B21F075FB092021F06AFBBB45F6D926
:106078002E4821F06DFB2A680024944290D2661EB7
:106088004E4416F8010F21F05BFB2B6801349C424B
:10609800F7D385E70C2800F083800A2852D00D2812
:1060A80050D07F2800F0FB80FF2B3FF679AF91E7B7
:1060B8001C4E002706F59878BB4602E00836464590
:1060C8000DD0224631684846FBF7E6FA0028F5D19C
:1060D800B346002FF2D1374608364645F1D13B4644
:1060E8005F469B46002B97D1002F3FF459AF0E48CF
:1060F80021F02EFBB3E7511C202009F8020029608B
:1061080009F801300A46A3E7CC4A00204D76002062
:1061180072480020485D002000ED00E0C8390020EA
:10612800CC3A0020A4430308646403086C640308A1
:10613800FC9F0020EFBEADDE0400FA0530590020B8
:10614800CC39002021F085FB23217D482DF058F81B
:10615800002800F0E380A0EB0900286088B1431E06
:1061680019F80310202940F0E98009EB030204E044
:1061780012F8011D202946D10346581E002BF7D1DD
:106188002B604FF48072002148462DF022F86D4BA9
:106198001B78002B3FF469AE6B4821F0D9FAFFE673
:1061A8006A4821F0D5FA684821F0D2FAF8E6684939
:1061B8006848C978684ADFF8D4E11360003118BF2D
:1061C8000121017065495160402193601173557335
:1061D800634964480B600432CEF80020594A012311
:1061E800137021F067FD584821F0B2FA4FF40060AF
:1061F8000CF09AFD5C4B93F82A30232B00F0968024
:1062080014F8023C3EE62B60584C002204F59878BE
:1062180009F8032002E0083444457BD02168484649
:1062280012F0DCFB0028F6D0444573D26368984727
:106238000023A5E74E4BADF822E00FCB0DF1280C5B
:1062480002AF87E80F004CF824ED14F8051C14F889
:10625800033C069404EB010E624639464FF0010CEC
:1062680006A8CDF81CE0ADF820308DF824C002F067
:106278006DFFE8B9019F002304F8023C002F3FF4AA
:10628800EFAD54F80A0C0DF011F8013654F80A0C69
:10629800B847032E04F1CC047FF4C7ADE5E5013B14
:1062A800002234482B6009F8032021F051FA77E6E0
:1062B800029A314B03923946A4F10A0002930CF07A
:1062C80049FFD7E714F8053C14F8032C0694234437
:1062D80007936E2A4FF0000308930993ADF8202026
:1062E8007FF42CAE06A8FBF756FA06A8FBF748FA87
:1062F800074606A8FBF744FA06A8FBF741FA1F4B26
:106308001F6058601AE62246A1E61D48083F21F0A2
:106318001FFAA4E61B4821F01BFA89E728681DE745
:10632800074811F0A5FE0BB0BDE8F08F164A14F827
:10633800023CC2F80C80CAF80090A3E5034663E764
:10634800CC390020CC4A00206C640308746403082C
:10635800FF540020AC290020E8220020553700080F
:1063680030590020A0640308485D0020A4430308B6
:10637800503403089C6403087C7A0020D82E00203F
:10638800646403088064030800ED00E0C839002055
:106398002DE9F04F2DED068BAB4BAC4A1C7897B02E
:1063A80000F59C41203181460B911160002C00F0D2
:1063B800E086A74A1268904240F28380A54A069276
:1063C8001668A549A54A0591013C1C70A44B049286
:1063D80006F480560893002E40F08180A14B1B786C
:1063E800022B01F03881042B01F0A381012B01F06D
:1063F80057819D4B9945089B9B7800F28E85002B11
:1064080040F08F85994B0793069B1E6816F48057BA
:1064180040F07D86DFF894A2049BB3F90610059B33
:106428005D8BA942B4BF00250125914B1B6813F071
:1064380080535ED0079A127812F001025FD0059857
:10644800408C884241F39682002D5ED1894C94F8A5
:106458008C10002959D188488849006890F82D0087
:1064680000240C604C608C60854900284ED108706F
:10647800002A4FD0F2064DD5824A1278D40649D464
:10648800002F47D1002B45D1700243D47E4B1B7897
:10649800002B02F003827D4B9B78002D42F0958201
:1064A8003BB17B4A7B4B12681B689B1A002BC2F2DC
:1064B8006D8210206F4C0DF05DFC012384F88D3047
:1064C80028E0644B06931E68644B634A049306F401
:1064D8008056634B05920893002E3FF47FAF00214E
:1064E8006348FBF70EFD00287FF478AF16F094FFA1
:1064F80074E770029ED4079A127802F001025D4C8C
:10650800002184F88C10002DA5D05D490120087069
:10651800002AAFD1604B1A78002A79D10599049CDA
:10652800488BB4F90070898BB4F90240B842B4BF03
:106538008026002646F04003B942D8BF33469B0860
:1065480043F08006A042B8BF3346049F43F040069C
:10655800A142C8BF33469B08B7F90440B7F90660A3
:1065680043F08007A042B8BF3B4643F04007A14232
:10657800C8BF3B469B0843F080073E4C8642C8BFD5
:106588003B4643F0400794F88EE08E42B8BF3B4646
:106598009E4501F04884A4F8902084F892203A4956
:1065A80084F88E300E78002E01F03D835F2B01F0C9
:1065B8009D836F2B01F0FC83079B1B78DF0727D493
:1065C80094F8921021BBB4F99030322B20DD94F866
:1065D8008E200120572A84F8920001F05087069BEC
:1065E8001B685D0741F18B825A2A41F0888294F832
:1065F8009430002B42F0628194F8963083F00103C6
:1066080084F89630002B42F0C9810C200DF0B2FBC3
:10661800224B0993224B234D0A93069B1B685F0765
:1066280000F1EB860DF150091F4E0B950022C9F8B9
:1066380004203446149240F6330B4FF0190840F208
:106648008337049D37E000BF2C400020D83F00204E
:10665800284000202C6F00201C5D00203E61002097
:10666800244B002022470020404B4C004D76002050
:10667800EC5F002038230020C44F0020784700201A
:10668800E02500207C770020AC200020306000202E
:10669800F075002034430020934B0020644F002005
:1066A800C84F0020C04F002094400020E440002044
:1066B8000434544522D0A178E378994218FB01703C
:1066C800F6D294F801E00EF1040E18FB037135F9C7
:1066D8001E305B45A8BF5B46B3F5617FB8BF4FF47A
:1066E80061739842E4DA9942E2DB21782729DFD8FE
:1066F80048460434FBF7F6FB5445DCD1624A0B9D4F
:106708001378624A99E8030082E80300002B40F0FE
:10671800B2855F4B1A78002A00F0EE8501215B48AC
:10672800FBF7EFFB002840F0DC82089BDB78002BAE
:1067380040F0D7822B881FB227F001071FFA87F88D
:106748004345A5F8008001F00580524F4FF002093B
:106758000E204FF0140B4FF0FF0A87F8009087F8CF
:1067680001B087F802A00DF005FB49464748B5F887
:106778000080FBF7C6FB002800F0CE8228F001035A
:106788009BB243452B800AD00E2087F8009087F8EB
:1067980001B087F802A00DF0EDFAB5F8008018F006
:1067A800020F01F098813C4B3C4A197850680B93D2
:1067B80018F0030F08BF81F00201C1F340010C92E9
:1067C800FAF7A5FA24213148FBF79BFB30B9079A61
:1067D80013785F0744BF23F004031370099B1B68F9
:1067E80013F00A0F11D006212848FBF78AFB00286E
:1067F80001F097802B88580641F12282072123480F
:10680800FBF77FFB002840F0B2870C211F48FBF7FD
:1068180078FB2A88002800F02E8342F480739A427D
:106828002B8009D01B4B022214211A700E20FF2244
:1068380059709A700DF09EFA194B1B78082B00F0CE
:1068480026830E2B00F02383069BD3F8008018F4D0
:10685800806F5FD0134B1B79002B00F0248214212A
:106868000A48FBF74EFB002840F0228229F032FB51
:1068780001200DF08DF9002849D0DFF82CA0002761
:106888004FF0CC0BA14614E050710020EC5F0020C3
:10689800CC4A002034590020B8750020BC7500206F
:1068A8000C480020884D002068480020DFB2022FE5
:1068B8002CD80BFB07F87B1C5AF80840002CF5D1A4
:1068C800032290F9023002940192C278E24951F809
:1068D8002220009218462246234601210CF0C4FDCE
:1068E800034607EB470000EB0010099353B121461C
:1068F8000AEB8000CC222CF06CFC099B4AF808308B
:106908000137FFB223F0F4FA0028D0D14C46069B99
:10691800D3F80080079B93F800A0D04B1AF0010A27
:1069280000F02B8201221A700A9B04991B68B1F9A6
:1069380006105A89CA4801279142077080F20382DB
:10694800C84B4FF07E521A60059BC74FB3F818909A
:10695800049B97F90420B3F90030387897F801C000
:10696800002AA3EB090714BF01224FF0FF32002FC2
:10697800B8BF7F42B7F5FA7FA8BF4FF4FA77B8429D
:1069880080F2DE813F1A07EE907AF8EEE77AB74F89
:106998004B45C7ED007A03DAF1EE677AC7ED007A66
:1069A800049BB3F902E0AEEB0903002BB8BF5B42CE
:1069B800B3F5FA7FA8BF4FF4FA73984280F29D822C
:1069C8001B1A07EE903AF8EEE77AF145C7ED017A1F
:1069D80003DDF1EE677AC7ED017A049BB3F9040091
:1069E800A0EB0903002BB8BF5B42B3F5FA7FA8BF41
:1069F8004FF4FA736345CCBFA3EB0C03002302FBEF
:106A080003F207EE902AF8EEE77A4845C7ED027AD6
:106A1800BCBFF1EE677AC7ED027A18F4805800F02F
:106A28004982B1F5FA6F924BA8BF4FF4FA61B1F5FC
:106A38007A7F1A78B8BF4FF47A71A1F57A71002A73
:106A480041F026818B4ADFF844E282FB0130CB1704
:106A5800C3EB6013581C6FF0630C3EF910003EF94D
:106A680013E00CFB0313A0EB0E0003FB00F382FB07
:106A78000312DB17C3EB62139E440FFA8EFE07EE78
:106A880090EAB8EEE78A87ED038AB8F1000F40F084
:106A9800B2832B885A0640F1FB807749774A91EDFB
:106AA800018AD2ED019A92ED026A91ED034A92EDC4
:106AB800030A91ED029A92ED007AD1ED005AD7EDD2
:106AC800011A97ED002A6E4A6E4938EE445A79EE5B
:106AD800C63A77EE007A65EE233A75EEC96A75EE26
:106AE800890A37EE401A66EEA76AB0EE633AA0EE5E
:106AF800813A13F00303B0EE665A78EE044A79EE51
:106B0800867AA0EE815AF0EE638AA4EEA73AD4EE14
:106B1800A78AA4EEE75A33EE263AF0EE687AF0EE4A
:106B2800674AF6EE008A35EE88AAE0EEC14A28EEFA
:106B3800C33A35EE635A77EE293A77EEE67AAAEE4B
:106B4800233A25EE285A76EE403A34EE49AAE0EE8A
:106B5800817A74EEA64AAAEE235A34EE094A37EE31
:106B6800697A64EEA84A63EE036AE4EE074A75EEB2
:106B7800C85A36EE006A67EEA87AB0EE667A95EEE5
:106B8800057AE5EE056AE5EE867AB1EE648AF0EEFE
:106B9800665AF0EE476AB1EE674AE8EE246A63EE99
:106BA800270A67EEA43AE4EE275AB1EE450AB0EE9A
:106BB800606AB0EE631AA4EE277A23EE244AE7EE61
:106BC800A76AA5EE246AA0EE031AE8EE245AB0EEEE
:106BD800448A31EEA19AE0EE240AA5EE278A66EEF1
:106BE800A16A72EE028AE5EE033A61EE211A26EEF8
:106BF800096AA4EEA47AA0EE274A0CBFD7ED022AB0
:106C0800DFED212A82ED005AA2EE256AE8EEA06A9D
:106C1800E2EE081A73EEA33A27EE227A34EE044A1B
:106C2800F0EE005AE3EEA26AA4EE226AA1EEA57A7B
:106C3800C7ED016AC1ED366A81ED356A87ED006AF4
:106C480081ED377A82ED013AC2ED027AC2ED034A4C
:106C5800F3B987ED027A1BE0AC6303084E76002097
:106C6800182600209425002008600020984D002058
:106C7800382F00201F85EB5154140020BC00002041
:106C8800F400002038230020000000009039002084
:106C9800BAF1000F40F0348129F030FE17B0BDEC96
:106CA800068BBDE8F08F079B1B78D9077FF5DEAD13
:106CB8004FF40F7024F040FF00283FF428AE0CF08A
:106CC800BBFB4FF40F7024F0E9FE00283FF41FAE21
:106CD8000CF0B2FB4FF40F7024F0E0FE0028EED168
:106CE80015E6099B1B689B077FF524ADB5F8008066
:106CF80018F0010F10D148F0010398452B800BD0F4
:106D08009A4B022214211A700E20FF2259709A7091
:106D18000DF030F8B5F8008028F002039BB2434527
:106D28002B803FF440AD914B02201421FF221870B4
:106D38000E2059709A700DF01DF8B5F8008032E5F4
:106D4800DFED8B7A23E6B1F5FA6F80F27D84187A4D
:106D58008B1A03FB00F3C2F5FA6293FBF2F3C3F15B
:106D6800640307EE903AF8EEE77A9FED827A824B59
:106D780067EE877AC3ED007AE6E51B780693002B69
:106D88007FF4D2AD7D4A1268002A3FF4CDAD7C4A2B
:106D9800079212F8030CDFF828B21146D71E10F03C
:106DA80055FC9BF80090079A002800F03B86069B4C
:106DB800B9F1000F53D107F10801787910F046FCBA
:106DC800002841F043856F49B87A10F03FFC00284D
:106DD80000F03B86B9F1020F41F04B856A49F87B18
:106DE80010F034FC002841F040856849387D10F0E7
:106DF8002DFC002800F03B86B9F1040F41F02285F4
:106E08006349787E10F022FC002841F0178561491B
:106E1800B87F10F01BFC002800F03B86B9F1060F84
:106E280041F008855C4997F8230010F00FFC002812
:106E380041F0FC84594997F8280010F007FC002815
:106E480000F03B86B9F1080F41F0E884544997F8FF
:106E58002D0010F0FBFB00283FF466AD09231A460D
:106E680002EB820217444F4A7878B9788BF80030E1
:106E78001070517058E522F480739BB29A422B80AF
:106E88007FF4D0AC484B1B78082B7FF4DAAC2A8807
:106E980022F040039BB29A422B803FF4D5AC334B8F
:106EA800022214211A700E20FF2259709A700CF0D9
:106EB80061FFC9E4059B5A8B9142C0F24884B1F541
:106EC800FA6FD4BFC2EB0101C2F5FA614FF47A73CD
:106ED80003FB01F135480378C2F5FA62B1FBF2F120
:106EE800002B3FF4AFAD4378314A01FB03F182FB3D
:106EF8000123C917C1EB6311A4E5DFED1D7A64E531
:106F08000B9B19780C9B01F001011868F9F7FFFE3B
:106F180017B0BDEC068BBDE8F08F13B9089A0123B2
:106F28009370244B089A1D7892F8214007931B20F0
:106F380010F0C4FB012C05F00108814600F0EB8637
:106F480005F00205089A1C4E92F82030DFF874A06C
:106F58001A4F09959346052B00F27D87DFE813F059
:106F6800BC00B2003400FA00FC00EF0034590020E5
:106F7800000000000AD7233C94250020507600200A
:106F8800DE580020E8580020ED580020F258002074
:106F9800F7580020FC58002001590020065900200D
:106FA8000B590020547600200C480020382F002070
:106FB8001F85EB514D76002088390020BC4F0020FA
:106FC80000000020AC200020012C04BF05238BF812
:106FD8002030B8F1000F12D0059B3088B3F9181093
:106FE8000022134661F30F0260F31F4261F30F039F
:106FF800049861F31F430360032342600993B14D72
:10700800DBF814102A68914280F0FD8547F2305170
:107018000322CBF81C108BF8202002200BF084FEF2
:1070280016F0FAF92968DBF81C200A440421CBF889
:1070380018208BF82010012C40F053872A68DBF8C1
:107048001810914280F007879AF8000020B910F0D4
:1070580035FB002840F0FF863A6822F002023A60C9
:107068002A687388642101FB03234FF4806000229F
:10707800CBF810308BF820208BF803200BF024FE7F
:107088009BF8203067E710F01FFB012807D18D4DD2
:1070980072882B68642101FB0233CBF81030B9F1F8
:1070A800000F02D0B379002B4BD1012C00F0D3860E
:1070B800844DDBF810102A689142C0F01F87012325
:1070C8008BF82030012C3AD0F379012B46D010F000
:1070D8007BFA9BF820303EE7B8F1000FD3D1099D29
:1070E8004FF48060B9F1000F00F03E830BF004FE0E
:1070F800089A00231361002D3FF486A928460CF056
:1071080039FE069B1E6816F480573FF483A91D219B
:107118006D48FAF7F6FE00287FF47CA96B4B03F163
:10712800500A03E004339A4500F09B861A78262A11
:10713800F8D19978DA789142F4D2FFF76DB9614DB8
:107148008EE710F041FA03224FF47A738BF820206F
:10715800CBF81C305B4D60E75A4D6CE710F034FA01
:10716800032240F6B8338BF82020CBF81C30554D5D
:1071780053E7574F3B78002B01F05582554BDFF80A
:107188006C81DFF86CB1DFF86CA1059345465E466B
:10719800049099460EE019F804109847032C28DC4F
:1071A80088B93B782AF8020F01349C4205F104059E
:1071B80080F24881072CE1B23046DBF80430EADD82
:1071C800984700B2EDE738F824206B88801A4FF40E
:1071D8007A719B1A01FB00F040F6CA0290FBF3F0AB
:1071E8000844904240F2EE23A8BF10469842B8BF28
:1071F800184600B2D5E71D213348FAF782FE28B1B8
:1072080000F0EBBD0436B4423FF443AC3178262994
:10721800F8D1B278F3789A42F4D2089BDB78002B45
:107228007FF437AC2848FAF76CFEDFED2B7A00289C
:1072380001F0FD8138EE678A284A2949FDEEC87AAF
:10724800CDED047ABDF910301B0382FB0302DB1776
:10725800C3EBA212C9F57A731BB203FB02F343F323
:107268000F334B4407EE903AF8EEE77A0123C7ED67
:10727800037A0B700DE4154B03E004339C423FF492
:1072880048AA19782329F8D19878DA789042F4D264
:107298000D48FAF736FE00283FF43BAA114B1B684D
:1072A80013F4003341F0918200220F4B1046995C91
:1072B800142902F10C0201F05F8101301828F6D17F
:1072C800FFF727BAF0750020EC5F002094400020FB
:1072D8005C4100201C5D002000007A44D34D621000
:1072E8000C260020E85700209C5403087041002019
:1072F8000C4B002036230020DFF8F092DFF8F0A2D4
:10730800AB4F0B9209F15A084FF0010B494619F897
:10731800010C10F09BF900B399F8040099F80230B9
:1073280099F803E000EB400107EB8101013BD1F83C
:10733800A02003EB4303534493420ED097F8CC208C
:10734800C1F8A0300BFA00F022EA00000B9B81F88C
:107358009CE0C1F8A43087F8CC0009F10609C145C2
:10736800D4D1944B944A1B780B930A9BDFF884A2E0
:1073780012681B680C93AAF19C094FF0000B904609
:10738800DAF8043083B31F7877B3DAF80820A8EB6B
:107398000202002A0CDB99F8CC20012101FA0BF13A
:1073A80022EA010208F5FA7189F8CC20CAF8081017
:1073B8000B9ACAB19AF8002059780432D2B200293F
:1073C80040F0DE8205990498098B30F9122001F10A
:1073D800C800824240F3578599F8CC109A7841FA50
:1073E8000BF3D80740F1E1850BF1010BBBF1040F5A
:1073F8000AF10C0AC4D1FFF791B96D4C94F8963094
:107408005BB1079B1B78DE0707D5049BB3F9062001
:10741800059B5B8B9A4200F3BA8511216748FAF7FE
:1074280070FD002800F0948294F89A302BB994F8F3
:10743800943013B93223A4F89830012384F89A3091
:10744800FFF7F0B8DDF810905D4A06925D491268C2
:1074580042F2010AA1FB091B12EA0A0A4FEA9B1B26
:1074680000F07382584D5948524C59492E7800788B
:10747800267008701EB156490E7886F001064C4CED
:107488000F2184F82410002B00F0E283059D514B56
:10749800B5F826C0B5F824E0059D109318462D8B45
:1074A80000784D4B129594F8255009954B4D04954D
:1074B800A3FB00535B0803EB4303C31ADBB20F9033
:1074C800CDF834C002F480520C9304F128000BF577
:1074D8009673CDF8449097F80080DDF82490DFF893
:1074E80018C109943D4C0E91139200210A930896F5
:1074F800CDF81CE0089B002B00F02783099B079D13
:1075080033F911201FFA82FEAE454FEA410303D337
:107518000D9DAE4540F25E835CF82120934580F0D6
:107528001E83E25EBAF1000F40F03383013141451A
:10753800E25200F10600DDDB0E9A099C284B84F824
:1075480024200F2A49460CBF01220022DDF844906E
:1075580084F825101A7000F08283224B1B491C4ABC
:10756800DFF854B008931C46042001230B701370F5
:107578000BF0DAFBDBF80030A1686268E3605B1AA5
:10758800934284BF002384F82130069B3C781E6810
:10759800002C01F07C80059A134DB2F824E0178B7B
:1075A8000E4916F48056284640F08283324636E06B
:1075B800382300208D510020F0750020EC5F00205A
:1075C8002C6F0020D34D6210B43F002044140020DB
:1075D8004514002049400020ABAAAAAA3E61002019
:1075E800C24B0020244B0020A4410020F557002066
:1075F80060340308D42300204C4000206F12833FDE
:10760800437803EB830303EB830303F2EE239BB27C
:107618000132A24221F8023B00F102000ED015F817
:107628001230002B00F0DA82022BE9D001320B88ED
:1076380021F8023BA24200F10200F0D1109A13781F
:1076480001331370FEF7C7BE1B7AC3F1640307EE5C
:10765800903AFFF788BB059A0499537DD27D013B88
:1076680031F913301AB1C3F53B6308331BB2A3F5E4
:107678007A7307EE903A1FED1F7ACC4AF8EEE77A54
:1076880040F2FF3167EE877AFCEEE77ACDED077AB4
:10769800BDF81C308B4228BF0B461380FEF7A9BEED
:1076A800C34CD4F88830A9EB0303002BFEF6A1AE37
:1076B800C04AC14B527C059933F812308A7DDFED00
:1076C800BF6A9FEDBF6AC97D9BB207EE102A07EE1D
:1076D800903AB8EEC77AF8EEE77A27EE267A67EEA0
:1076E800867A0B9AC4F88820C7EE876A40F2FF3280
:1076F800FCEEE67ACDED077ABDF81C30934228BF40
:10770800134609B1D31A9BB2AE48AF4D0178AF4CBE
:1077180035F81160226825F81130921B13440131A5
:10772800A24D236001F00F021B0902702B80FEF7A7
:1077380060BEFDF713FEA64BA64A1B68C31A934208
:107748007EF757AE994B00221A80FEF752BE41468B
:10775800FFF7C0BB0221A048FAF7D3FB00283FF48B
:10776800DBAA2F80FFF71BB80BF0AEFAC0E49B4AE8
:10777800B2F90030002BB8BF5B42B3F5E17FBFF62A
:1077880044A8B2F90230002BB8BF5B42B3F5E17FE1
:10779800BFF63BA8924B93ED096AD3ED076A93EDC8
:1077A800057AD3ED037A76EE866A77EE877A76EEF7
:1077B800A66AB7EE007A37EE666A77EEA77AB0EE79
:1077C800C66AF0EEE75AB4EEE56AF1EE10FAB4BF15
:1077D800B0EE655AB0EE465AB5EE405AF1EE10FAE0
:1077E80040F0A6839FED7F7AB4EEE56AF1EE10FAD9
:1077F80044BF9FED7D6A36EE477AB7EE006AF4EE35
:10780800C66AF1EE10FAC8BFDFED786AF5EEC07A05
:10781800C8BF36EEC77AF1EE10FA48BFB1EE477A24
:10782800F6EE007A27EE677ADFED6F7A77EE276A51
:10783800BDEEE66A16EE103A2033402B40F254862D
:10784800DFED6B6A6B4ADFED6A7AC2ED006AFDEE26
:10785800C76AC2ED017A16EE903A2033402BC2ED8A
:10786800027A49D8DFED617AB4EEE77AF1EE10FAE0
:1078780041F30C809FED606ADFED606A01E0B0EED5
:10788800677AB4EEE67AF1EE10FA77EE467AF6DC2D
:107898009FED5B7AF4EEC77AF1EE10FA40F1FA87C1
:1078A8009FED556ADFED576A01E0F0EE477AF4EE96
:1078B800E67AF1EE10FA37EE867AF6D4DFED4A7AF8
:1078C800B4EEE77AF1EE10FA40F3A086DFED477ADE
:1078D80037EEC77A27EE076ADFED4B5ADFED4B6AC2
:1078E800DFED4B7AE6EE256A67EE065AE6EE267A73
:1078F800A5EEA77AF0EE477A464BC2ED037A1A68EE
:1079080012F4003240F05386434B1046995C0A2922
:1079180002F10C0200F0588501301828F6D1FEF764
:1079280074BF2A8822F040039BB29A422B803EF40F
:1079380065AF3A4B022214211A700E20FF225970AB
:107948009A700CF017FAFEF759BF35490E7891E591
:1079580094F89430002B3EF465AE079B1B7813F027
:1079680001037EF45FAE012284F8943084F89520F8
:10797800FEF758BE0E4C012184F88C10FEF7C5BDE9
:10798800012900F03F8599F8CC20012303FA0BF375
:107998000BF1010B1343BBF1040F89F8CC300AF14A
:1079A8000C0A7FF4EDACFEF7B9BE00BF8477002067
:1079B8003823002038750020587500200000C84280
:1079C8000000804423470020284700202447002047
:1079D8005824002060E31600EC5F0020704F002060
:1079E800CC000020A7DFA834DB0FC93FDB0F4940DC
:1079F8000000000054140020DB0FC940E4CB1641FE
:107A0800DB0F49C0E4CB16C192E741B99730083C77
:107A180015A82ABEE85700209C54030834590020B2
:107A28008D510020511D78790FF010FE00283FF489
:107A3800CAA9B9F1010F40F0098707F10D01B87A19
:107A48000FF004FE002840F01487B449F87B0FF0CB
:107A5800FDFD00283FF4C9A9B9F1030F40F00587DF
:107A6800AF49387D0FF0F2FD002840F0EB86AD49B4
:107A7800787E0FF0EBFD00283FF4C9A9B9F1050F96
:107A880040F0DC86A849B87F0FF0E0FD002840F000
:107A9800D186A64997F823000FF0D8FD00283FF4B7
:107AA800C9A9B9F1070F40F0C186A14997F8280084
:107AB8000FF0CCFD002840F0B1869E4997F82D00C4
:107AC8000FF0C4FD00283EF42FAFB9F1090F3EF4C2
:107AD8002BAFFFF7C3B948F0020343452B803EF4B0
:107AE80062AE954B022214211A700E20FF225970A3
:107AF8009A700CF03FF9B5F80080FEF754BE5D2A85
:107B080000F058825B2A00F0C6855E2A00F04A869B
:107B1800562A00F04B86972A00F09C86A72A00F088
:107B28003586864D2B889B0740F0F485A2F1B70374
:107B3800072B00F2A982DFE813F06902A702A70267
:107B4800A7025B02A7024D024D02079B002B3FD004
:107B58005CF8212093454FEA4103FFF4E2AC784AF0
:107B6800774DD25C05EB030E002A00F09480022AC0
:107B780047D19EF8012002EB820202EB820202F258
:107B8800EE2292B2032933DD12B2BAF1000F3FF4AC
:107B9800CDAC0C9D20F81520B9F1000F03D10F9D35
:107BA800022D7FF6C3ACB0F802900288B0F804E06A
:107BB8004A449644634A0FFA8EFE82FB0E52624D87
:107BC800A2EBEE7225F803E012B24FF00109ADE422
:107BD8001A464B000A9D4CF82150A3E4D3B2022B5D
:107BE80004D9032B7FF422AD734611E53B460FE51C
:107BF800012505FA01FE0E9D25EA0E0512B20E9525
:107C080090E4E25ABEE7514A1278002A7FF4FEA9AE
:107C1800B8F1000F3FF4FAA9012C40F01C819BF841
:107C28002030FFF798B931464948FAF76AF9002831
:107C380000F09A8084F8936016F01CF8FEF7BCBC3C
:107C480043F0400293422A807FF473AEFEF7D6BD1C
:107C5800404B414A109201221A70404B04931B2159
:107C68003B48FAF74EF900287FF477AC3C4BDFF835
:107C7800F4B008931946DBF80030CA688B609B1A89
:107C8800C82B00F2F584069B1E6806F48056D5E4DE
:107C98005B78FFF729B9CAB2022A40F2B083032AF7
:107CA800AFD1129A139D079E002D08BF324669E78F
:107CB80000220FE0437803EB830303EB830303F213
:107CC800EE239BB20132A24221F8023B00F10200EE
:107CD8003FF4B4AC15F812301BB1022BEAD00B8874
:107CE800F0E7D3B2032BFAD83B46EBE7B2F5FA7FBD
:107CF800FEF68EAC94F89230002B7EF489AC079B8C
:107D08001B7801210B4084F8921000F0D58315F000
:107D180083FBFEF77DBC0025FFF714B9ED58002062
:107D2800F2580020F7580020FC5800200159002084
:107D3800065900200B59002034590020C04F00205C
:107D4800A441002056555555A8230020D0250020D1
:107D5800EC5F0020C24B0020494000203E6100201B
:107D6800244B0020F0750020079BAF4A1B78106059
:107D7800D9077EF525ACAD4B1B78002B3EF448ACFB
:107D8800089BDB78002B7EF443AC94F893300133E6
:107D9800DBB2032B84F893307EF63AACA44B5B78C5
:107DA80013B9002D7EF434AC15F036FBFEF704BC95
:107DB800B2F5FA7FFEF62CAC94F89230002B7EF4E4
:107DC80027AC079A12780121D20784F8921000F1A3
:107DD8000B8415F04FFFFEF71BBC089BDB78002BCC
:107DE8007FF414AADFED937A934938EE678AC9F5D0
:107DF800FA63FDEEC87A1BB2CDED047ABDF9102006
:107E0800120381FB0201D217C2EBA11203FB02F39A
:107E180043F30F334B4407EE903AB8EEE78A87ED09
:107E2800038AFFF7F3B9854A83491068B4F99020AB
:107E3800C66981FB06018911F617701A00F5FF4023
:107E48007F3082423EF7ABAB891B0A4412B2A4F8DA
:107E58009020FEF7A4BB099D002D3EF4D5AAFFF79C
:107E68004DB9774A059BD588049A1B8BB2F9061041
:107E78005A1B914240F388802B449942B4BF002595
:107E88000125FEF7D2BAC8398A4242DA99F8CC10ED
:107E98009A7841FA0BF3D9073FF5A6AA5242012076
:107EA8000D920CF04DF87B1E0D9A162B00F25081A6
:107EB800DFE813F02202360209025B024A026F026F
:107EC800F401DF01CA01B501A0014E015B028D0179
:107ED8006F02F401DF017901650151013E012801BA
:107EE8001401AB460899DBF80020CB69099D1344BF
:107EF8008B61002D3EF488AAFFF700B90FF064FBF0
:107F0800032140F6B8328BF82010CBF81C20FFF77D
:107F180084B899F8CC30012202FA0BF223EA020362
:107F280008F5FA7289F8CC30CAF80820FFF75CBA6D
:107F3800B4EEE56AF1EE10FA8CBFB0EE654AB0EE29
:107F4800464AC4EE054A9FED3F2A9FED3F5ADFEDB2
:107F58003F1ADFED3F2A9FED3F3ADFED3F3A9FEDB5
:107F68003F4AA4EE825AE4EEE12AA4EE857AA4EE12
:107F7800A23AB0EE475AB0EE637AA4EE837AA4EE42
:107F8800874A84EE057A2FE40125FEF74EBA0021D0
:107F98003348F9F7B6FF00287FF43FAA322384F864
:107FA8009600A4F89830FFF738BA002A0CBF0120D1
:107FB800022075E72B4B002201202B492B4C0B602C
:107FC8002B4B09932B4B22702B4D0A930BF0B8FFC8
:107FD800FEF723BB274A254B0A921146274A0A6017
:107FE80002225A70224B09930FF0CCFBFEF715BB07
:107FF800204A1E4B0A921146214A0A6000225A70F2
:108008001B4B09930FF0BEFBFEF707BB194A174B32
:108018000A9211461B4A0A6001225A70144B0993AE
:108028000FF0B0FBFEF7F9BA384300208D5100205D
:108038003060002000007A44D34D62105879002047
:108048006C39002099FB243F69A2163E39094E3D40
:10805800E3B59E3E88FA163E45FE7F3FA7DFA8346B
:10806800EC5F0020443B0020C44F0020FF54002058
:10807800644F0020C84F0020C04F0020004B002054
:10808800E84A0020F44A0020792A00F074847A2A09
:1080980000F066849E2A00F05B849D2A00F05084DC
:1080A800AE2A00F04584AD2A00F03A84EF2A00F0A9
:1080B8003484FD2A00F01F84FB2A00F09884FE2AED
:1080C80000F09284F72A00F08C847B2A00F00C845C
:1080D800BA4B0993BA4B0A93FEF79FBAD9F8D00066
:1080E800B84B90F836109B7811446429A8BF6421D6
:1080F80021EAE17180F83610002B40F094840EF0EC
:1081080099FB40E4D9F8D000AE4B90F837109B7833
:108118001144FE29A8BFFE2121EAE17180F8371039
:10812800002BECD016200FF013FBD9F8D000E6E7AF
:108138000C98A44B41781144B1F5967FA8BF4FF431
:10814800967121EAE17141709B78002B40F06484BC
:10815800D9F8D000D3E7D9F8D0009A4B81781144E8
:10816800C829A8BFC82121EAE17181709B78002B3A
:10817800C5D014200FF0ECFAD9F8D000BFE7D9F831
:10818800D000904B41781144C829A8BFC82121EAE2
:10819800E17141709B78002BB1D013200FF0D8FA11
:1081A800D9F8D000ABE7D9F8D000864B0178114454
:1081B800C829A8BFC82121EAE17101709B78002B6A
:1081C8009DD012200FF0C4FAD9F8D00097E77D4B64
:1081D8000C989B78417911446429A8BF642121EA4D
:1081E800E1714171002BB3D00E200FF0B1FAD9F82C
:1081F800D00084E7D9F8D000724B017A9B781144FB
:10820800C829A8BFC82121EAE1710172002B3FF4F7
:1082180076AF0B200FF09CFAD9F8D0006FE7D9F8A9
:10822800D000684BC1799B781144C829A8BFC821E0
:1082380021EAE171C171002B3FF461AF0A200FF010
:1082480087FAD9F8D0005AE7D9F8D0005D4B817980
:108258009B781144C829A8BFC82121EAE17181711E
:10826800002B3FF44CAF09200FF072FAD9F8D00078
:1082780045E7D9F8D000534B417993F802E011440F
:10828800C829A8BFC82121EAE1714171BEF1000FD8
:1082980040F0B083112F7FF461AF30E7D9F8D000F8
:1082A800484B017993F802E01144C829A8BFC821B6
:1082B80021EAE1710171BEF1000F40F07C83102FBB
:1082C8007FF460AF1BE70C993E4B0F790D93174471
:1082D800642FA8BF642727EAE7770F710FF052FAD7
:1082E8000D9B9B78002B3FF433AF032039460FF0EA
:1082F8002FFAD9F8D00002E70C98324B01781144D4
:10830800FA29A8BFFA2121EAE17101709B78002BB4
:108318003FF41EAF01200FF01BFAD9F8D000EEE6AB
:108328000C98284B817811446429A8BF642121EA5C
:10833800E17181709B78002B3FF40AAF02200FF0A7
:1083480007FAD9F8D000DAE60C981E4BC1799B7869
:10835800114481F30801C171002B3FF4F9AE0520E7
:108368000FF0F6F9D9F8D000C9E60C98154B8179C9
:1083780093F802E011446429A8BF642121EAE1715D
:108388008171BEF1000F40F03F830D2F7FF420AFC5
:10839800DEE6D9F8D0000B4BC17893F802E011441F
:1083A800C829A8BFC82121EAE171C170BEF1000F38
:1083B80040F0F7820F2F7FF4F9AEA0E6644F00205B
:1083C800C84F00207E770020B549D1F800E0420070
:1083D800BEF1000F08D0171803EB87079EF801E0DD
:1083E8007F787745BEF411AA1044AE4FAE4A03EB2E
:1083F800800300200B6038801060FEF706BA129ADE
:10840800FFF7C0BB04999B7831F91220B2F5617F60
:108418004FF4966191FBF3F3C0F2EF8040F633011D
:108428009142A8BF11460C2FA1F5617191FBF3F1A0
:1084380000F0D481182F7FF4A6AAC9B2C8290B4628
:10844800A8BFC823D9F8D020D77DD8B2B8423FF406
:108458009AAADF1B954BD07548BF0737FF109B784A
:108468000137FFB23BB9002F3FF48DAA38460BF015
:1084780067FDFFF788BA18200FF06AF9F3E78C4A0E
:108488008C4B099210461A688B494FF47A73B3FBE8
:10849800F2F3C3EB431203EB82030268DB005607D7
:1084A800A1F8A8307EF5B6A8844B854D0A221A801B
:1084B800844B0A93FEF7B1B88349096811F4003177
:1084C80040F0A681814B08465D5C0F2D01F10C013F
:1084D80075D001301828F7D1FA3A0023A4F8902073
:1084E80084F89230FEF794B8B4EEE77AF1EE10FA19
:1084F80040F3F281DFED765A9FED766A01E0F0EE07
:10850800676AF4EEC66AF1EE10FA76EEE57AF6DC02
:10851800DFED716AF4EEE67AF1EE10FA40F1D981F6
:10852800DFED6B5A9FED6D6A01E0F0EE667AF4EECE
:10853800C67AF1EE10FA77EEA56AF6D4DFED687A1E
:10854800F4EEE76AF1EE10FA40F31481DFED657A94
:1085580077EEE66A66EEA65A9FED635A9FED636A68
:10856800DFED637AA5EE856A26EEA55AE5EE867AF2
:10857800E5EE276AFFF766B94949D1F800E04200FD
:10858800BEF1000F08D0171803EB87079EF801E02B
:108598007F787745BEF4BDA80244424F424803EBBA
:1085A800820300220B603A800260FEF7B2B8514B9A
:1085B8001B78032B00F036810022FFF7A5B9384954
:1085C8000F68450037B12E1803EB86067F7876785A
:1085D800BE4281D20544334E334803EB8503002560
:1085E8000B603580056077E7434A31491360354BA6
:1085F8000991334D0A93FEF710B80C2F00F005814E
:10860800182F7FF4C0A900210B461BE7DFED3B7A4A
:10861800B4EEE77AF1EE10FA44BFDFED2F7A37EEC9
:10862800C77AFFF757B9364A0592FEF70DBF38EEFD
:10863800678A344B34491870FDEEC87AC9F5FA6375
:10864800CDED047ABDF91020120381FB0201D21787
:10865800C2EBA1121BB203FB02F343F30F334B44EB
:1086680007EE903AF8EEE77AC7ED037AFEF711BA0B
:10867800264A069B1E68136823F004031360089AB1
:10868800012306F4805682F82130FEF7D7BF06F49E
:108698008056FEF7D3BF1E4B012202208DE400BF97
:1086A8008C250020782600207C2600207E7700205C
:1086B800644F00201C6F0020A46C00206679002005
:1086C800C04F0020C84F0020E85700209C540308E2
:1086D800DB0FC940E4CB1641DB0F49C0E4CB16C120
:1086E800DB0FC93FDB0F494092E741B99730083C9F
:1086F80015A82ABE9C77002038430020DB0FC9BF8D
:108708001C5D00200C260020D34D6210BC4F0020B9
:10871800923B00200023BB2A149300F0B480B72AB0
:1087280000F0AD80BE2A00F0A880BD2A7FF4ACAC72
:108738004FF6FE71BE4ABF48D689099090893344E6
:108748000144D381918113F053F9F8F75FFD13F0D9
:1087580037F9FBF72FFB01200BF0F2FBB4F8903050
:10876800B54A0A92FA3B0022A4F8903084F8922085
:10877800FDF753BFDFEDB17AF4EEE76AF1EE10FAD8
:1087880044BFDFEDAF7A77EEE66AE3E6AD4AA94B80
:1087980009931378AC4D43F004031370A64B0A9366
:1087A800FDF73BBFA94B0222032006E413F020F992
:1087B800F8F72CFD13F004F9FBF7FCFA01200BF095
:1087C800BFFB94F88E20FFF7A6B9A14B1B78032BAB
:1087D8007EF46AAD0BF0B2FAFDF79BBFCFB29D4BAA
:1087E8000E915B78BB423FF4CEA89B4B0D93384665
:1087F8000CF07AF90D9B0E999B781BB1C9B20C202D
:108808000EF0A6FF0137FFB22DE600273946E6E74E
:108818008F490978032962D0194653E608231A4676
:10882800FEF71EBB0BF08AFAFDF7EFBF07231A46C7
:10883800FEF716BB06231A46FEF712BB05231A4697
:10884800FEF70EBB04231A46FEF70ABB01231A469D
:10885800FEF706BB814B774A09924FF4C8721A801B
:10886800754B794D0A93FDF7D8BE03231A46FEF7D8
:10887800F7BA02231A46FEF7F3BA02215AE7194655
:108888004FF6FE7356E71946022353E7F0EE477A90
:10889800FEF7FEBFB0EE677AFFF710B8002D3DF483
:1088A80008AE6F4C94F88D30002B3DF433AE0BF0CE
:1088B80045FA002384F88D30FDF72CBE5D4B0993F3
:1088C8005D4B84F8941084F895005F4D0A93FEF789
:1088D80095BDF0EE676A31E6F0EE667A18E60BF0C1
:1088E8002DFAB4F99020F7E54FF4FA6102200CF064
:1088F80019F8FFF7EDBB002101200CF013F8B4F8CC
:1089080090304C4A0992963B4B4AA4F89030002389
:108918000A9284F89230FDF780BE00210846ECE701
:10892800FF21002026F080FA94F88E20FFF7BEBBC6
:108938000121002026F078FA94F88E20FFF7B3BBC7
:108948000021FF2026F070FA94F88E20FFF7A8BBCC
:108958000021012026F068FA94F88E20FFF79DBBCD
:10896800404A344B0993137A43F001031372324B94
:108978000A93FDF752BE3B4A2E4B0993137A23F014
:10898800010313722C4B0A93FDF747BE344C14F0C5
:1089980043FD002384F88D30FDF7BCBD0B20FDF7A7
:1089A80035BE0F200E930D920EF0D2FED9F8D000EE
:1089B8000E9B0D9AFEE410200E930D920EF0C8FE49
:1089C800D9F8D0000E9B0D9A79E4002B3FF469AFDB
:1089D8002549264A09684FF47A7000FB031313608F
:1089E8005FE70021042088E70021032085E70021B4
:1089F800022082E711200E930D920EF0A9FED9F8FD
:108A0800D0000E9B0D9A45E40D200E930D920EF0AA
:108A18009FFE0E9B0D9AB8E415200EF099FED9F82A
:108A2800D000FFF76CBB17200EF092FEFFF790BB4B
:108A380010600020644F0020C84F0020DB0FC9BF22
:108A4800DB0F49C07C770020C04F0020E03B0020AE
:108A58009C770020FF5400207E7700206879002052
:108A680038230020A84B0020F07500203443002054
:108A78002DE9F047C74C636820469847002800F066
:108A8800C380C54B1B780122042B84F83C2000F0DE
:108A9800BD80B4F91610B4F91820B4F91A3021635E
:108AA8006263A363BD4B1B88002B69D0BC4DD4ED1A
:108AB8000C7AD5ED004A95ED050A95ED015A95ED2C
:108AC800067AD5ED035A95ED026AF8EEE76AD5ED18
:108AD800047AA4EEA60AA5EE267A67EEC07AA5EE79
:108AE800C07AE6EE267A85ED057AC5ED067A29F094
:108AF800B3FBD4ED0D6AD5ED094A95ED0E0A95ED57
:108B08000A5A95ED0F7AD5ED0D7AD5ED0C5A95EDFB
:108B18000B6A2063F8EEE66AA4EEA60AA5EE267AAA
:108B280067EEC07AA5EEC07AE6EE267A85ED0E7A73
:108B3800C5ED0F7A29F090FBD4ED0E6AD5ED124AF7
:108B480095ED170A95ED135A95ED187AD5ED167A25
:108B5800D5ED155A95ED146A6063F8EEE66AA6EE4F
:108B6800A40AA6EE857A67EEC07AA0EE657AE6EEEC
:108B7800867A85ED177AC5ED187A29F06DFBA06322
:108B8800884FA17F884816F097FE3B88002B40F05D
:108B98008480864ED6F8E050854B1B685B0743D42B
:108BA800B5F90070216B636BA06B824A824E92ED1F
:108BB800026AD2ED006AD2ED015AC91B2163B5F9E8
:108BC8000270DB1B6363B5F904703568C01B07EEE0
:108BD800900AB8EEE75A07EE901AB8EEE77A07EE71
:108BE800903AF8EEE77A36EE056A36EE877A77EE4F
:108BF800A57A0135A06382ED026A82ED007AC2EDA2
:108C0800017A3560BDE8F087BDE8F0876B4BB4F9B1
:108C18001600B4F91810B4F91A2018802063598086
:108C280061639A80A2633DE7B6F89820322A00F083
:108C38008880002A66D196F89530002BB0D060481D
:108C4800D6F8FC205F4980FB0273D217C2EB2312CF
:108C58002A80D6F8002180FB0273D217C2EB2312B8
:108C68006A80D6F80431A78A80FB0302DB17C3EBBE
:108C78002213DB1BAB800023CB6086F8953012F003
:108C8800B7FEF8F7C3FA12F09BFEFBF793F8012042
:108C98000BF056F9D6F8E05082E7444E226BD6F82E
:108CA800E050B3F5C87F4FF0000323632B80398869
:108CB80018BFD6F8E400B7F8008008BF0020B1F567
:108CC800C87F18BFD6F8E830616B02440B44002017
:108CD800B8F5C87F6063C6F8E420C6F8E830688055
:108CE80052D0D4F838E0D6F8EC10A0637144B8F14B
:108CF800010FA880C6F8EC1068D008F1FF38A7F873
:108D0800008049E7D6F8FC00236B00210344C6F82D
:108D1800FC3021632980D6F80001636B616303444A
:108D2800C6F800316980A36BD6F80401A163034437
:108D3800012AC6F80431A98075D0013AA6F898200E
:108D480079E72B8820491F48276BA6F8F0300023C5
:108D5800B5F802E0B5F804C0C0684B608B602363C7
:108D6800C6F8FC702B80616BC6F8001163636B80DA
:108D7800A16BC6F80411A363A6F8F2E0A6F8F4C044
:108D8800C6F8F800AB80D8E7A36BC6F8EC30A06350
:108D9800A880B2E7784F0020104C00203C43002008
:108DA8004043002068790020A84F00203823002085
:108DB8002C6F00207C37002078370020144C0020CE
:108DC8001F85EB511060002034240020DFF804C117
:108DD800DFF8F0E0C8328CFB02A9C833D217C2EB27
:108DE800E9128CFB03A9DB17C3EBE913C8316B80CD
:108DF8002A808CFB013CA28ACB17C3EBEC139B1A8D
:108E0800AB80CEF80C0012F0F3FDF8F7FFF912F082
:108E1800D7FDFAF7CFFF40460BF092F8B7F800807D
:108E2800D6F8E05069E7254B86F89A101B6886F853
:108E3800942013F4003334D119462148475C0B2F92
:108E480001F10C0110D00133182BF7D1B6F8F0104E
:108E58001C4B2980B6F8F270B6F8F400D6F8F81072
:108E68006F80A880D96068E7174FD7F800C059000D
:108E7800BCF1000F09D001EB030E00EB8E0E9CF83D
:108E880001C09EF801E0E645E0D20B44DFF848E077
:108E98000E4900EB830000233860AEF800300B6009
:108EA800D4E70B4B1B78032B01D00B46C5E70AF020
:108EB80045FFD6F8E050B6F89820C7E7E8570020F5
:108EC8009C540308106000208C2500207C2600207C
:108ED8009C7700201F85EB51782600202DE9F0476C
:108EE8008C4B1B78DB07074644D58B4B8B4D1C7886
:108EF8008B4E012C59D01CD3022C07D189498A4AA0
:108F080009881288914201D901241C70EB7AE3B1D7
:108F18002B89D3B1854B1B78BBB10BF007FE00281A
:108F280000F09B802B7B83422CBF012100213170F4
:108F38000CE07C497E4A098810886A7B801A88423E
:108F4800E2DAEB7A0024002BE2D131782A79632A1D
:108F580006D8022C774E00F0BA803378002B5DD10A
:108F6800754AAB7A8C4238BF0C461470002B4CD132
:108F7800BDE8F0876B4B694D19885B88E878CB1A98
:108F880083EAE3728142A2EBE3721DD32B788B4212
:108F98001AD3614B1C78E01E012861D9674909780A
:108FA80002294FD0012C5E4EA5D15F4A5D49128837
:108FB800687B0988121A914239DD5D4A12888A4213
:108FC800A4D200241C70A1E7B1EB400FE1DC524BA6
:108FD8001C78E11E012940F29480022ADEDC574900
:108FE8004F4E0878DFF84481DFF844C1DFF838E1F4
:108FF80000210324022834701C7088F80010ACF893
:109008000010AEF8001081D11FE0012C71D0022CA5
:109018000BD10720BDE8F0470AF0ACBE7068381ADB
:10902800474B984258DD72709AE7BDE8F0870224F2
:109038001C706BE7022AD2DD4049097802294FF0FB
:10904800040464D13949364E09783E48022ACCBF17
:1090580000220122C28081804BE70221317075E72E
:10906800022A9BDC95F800C091FBFCFC0CF1010C7A
:10907800BCF1080FDFF8B4A0304EA87895F801E0ED
:1090880096F800802A4CDFF8A090254EA8BF4FF034
:10909800080C8AF800C01FFA8CFA10FB0AF01EFBB5
:1090A8000AFE80B2DFF88CA02080A9F800E0002436
:1090B8004FF0640EB8F1020F34701C70CAF8044007
:1090C8008AF801E07FF439AF0FFA8CF1BDE7307808
:1090D800A0B9012377603370C2F164021A4B00FB18
:1090E80002F083FB0023C017A0EBA350643070701C
:1090F80036E70820BDE8F0470AF03CBE7368F81A66
:109108008EE7032C96D10D49097802299AD0044E8E
:10911800FCE600BF4D760020302F0020544F002081
:10912800402F0020304D0020342F0020964D002085
:10913800322F0020382F00209C770020104C002070
:109148007F969800144C00206BCA5F6B2DE9F04F96
:1091580095B0B0F908500D81EDB2442D00AF0C4622
:10916800904600F0D182064643D9812D00F0068250
:1091780000F29980542D00F0CE8040F228816E2DA7
:1091880000F09082802D40F02581C44B93F800A018
:109198000AF1020A1AF0FF0A00F09980C04BDFF8C2
:1091A8003483C04EDFF830B39A4403F101090A252D
:1091B80016E0322D00F09583A5F13C00C0B21328CB
:1091C80040F2958300232268511C216015702268A3
:1091D800CA4502F101012160137078D019F8015BCA
:1091E8000A2DE6D1BBF80030FF2BA8BFFF23DBB266
:1091F800E9E7052D00F0768220D8022D00F0838063
:1092080040F29B81032D00F04482042D40F0E2805F
:10921800A54920462A46F8F7C3FA00212046F8F760
:10922800EDFA22680021531C0125236028462B46AD
:10923800543711706381BD46BDE8F08F242D60D08E
:1092480040F20D81282D00F0E681382D40F0C280D3
:109258000A68964B0125511C21601570226805216A
:1092680050192060117022680A215019206011706D
:10927800226800215019206011702268197850194D
:109288002060117022685978501920601170226886
:109298009978531923602B461170284654376381F7
:1092A800BD46BDE8F08FA02D19D040F21B81B82D26
:1092B80000F0ED81FE2D40F08D807D4D05F1080612
:1092C80035F8021B2046F8F799FAAE42F8D1012585
:1092D8002B46284654376381BD46BDE8F08F754B51
:1092E80008461968F8F773FA734B20461968F8F7B7
:1092F8006EFA724B196820460125F8F768FA2B4672
:10930800E7E76F4BF6E704226E4920460125F8F798
:1093180047FA2B46C1E70B68DFF8C081591C0122C8
:1093280021601A70236800259A1822601D7023682E
:1093380098F85520591C21601A70236898F8542011
:10934800591C21601A70B8F850102046F8F756FAE0
:1093580023685A1C22601D7023682822591C21602A
:109368001A70B8F852102046F8F748FAA8F1020522
:1093780008F14E0635F8021F2046F8F73FFAAE42CC
:10938800F8D12268504B0D21501C20605D181170D7
:10939800226813F8011F501C9D4220601170F7D1FC
:1093A80023680222591C21601A70B8F8561020460A
:1093B800F8F724FAB8F858102046F8F71FFA0125EC
:1093C800B8F85A102046F8F719FA2B4665E7522DD7
:1093D8003FF427AF2146284608F096FC03460028AC
:1093E8007FF475AF742D00F0BB80772D0DD13268F6
:1093F800716891421EBF531C33601178334A08BF0D
:10940800194620460AF04EFE61E7F52D01F0ED827F
:10941800472D00F0A581392D326800F0AA8200F2AC
:10942800A082212D01F0A082292D40F0E382531C57
:10943800336013780A2B01F06483502B41F0B1811B
:109448003046F8F79DF9DFF89880A8F80000304614
:10945800F8F796F90125A8F802002B461DE7202DFC
:10946800B8D10B681A4D591C6A7821601A702368A4
:109478002A78591C21601A702368AA78591C21601F
:109488001A7029892046F8F7B9F923686A79591CAE
:1094980021601A702268A979C5E600BFF14B002047
:1094A800A8340308E02E0020055500202F3B00209B
:1094B800144C0020ACF7FF1FB0F7FF1FB4F7FF1FD5
:1094C800743C0020A86403086D770020712D010802
:1094D800544F002067666666082F0020107700202A
:1094E800BC2E0020822D7FF475AF0B688A4A8B4D05
:1094F80011788B4A581C2060197011892046F8F79A
:109508007DF9884B22681B88FF2B02F10101A8BF57
:10951800FF2321601370A96881F3100189B22046E6
:10952800F8F76CF9296801F30F0189B22046F8F7BA
:1095380065F97D4B2268197875E6012D7FF44AAFED
:109548000B680022591C21601A7023685A1C22607B
:109558001D7022682521531C23602B4611709CE640
:109568003268716891421EBF531C336011786F4A8C
:1095780008BF194620460AF095FDA8E66C4B1E78F0
:10958800043616F0FF063FF4A2AE6A4BDFF8C88136
:109598001E4403F1010A4FF00A0924E0B9F1500F03
:1095A80000F09D81B9F15A0F00F0B681B9F1320F80
:1095B80000F0B681A9F13C00C0B2132840F2B38193
:1095C8000025294623685A1C2260204683F800900B
:1095D800F8F714F929462046F8F710F9B2453FF490
:1095E80076AE1AF8019BB9F10A0FD7D1524B9D6894
:1095F800196805EB85054FF6FF736D009D42A8BFFE
:109608001D469942A8BF194625EAE57521EAE17188
:10961800ADB289B2D6E70B68DFF84091474E591CC6
:10962800022221601A7023684FF006085A1C226033
:1096380083F8008023680A22591C21601A70236865
:1096480001255A1922601D70B9F800102046F8F754
:10965800D5F8B9F802102046F8F7D0F823685A1957
:10966800226083F8008023685022591921601A70FB
:1096780023680022591921601A7031882046F8F7AA
:10968800BDF871882046F8F7B9F82B4605E62C4B4B
:1096980030E60B685A1C0A601D700B685A1C0A6079
:1096A8001D70BEE51F4B0A681B881C4DFF2BA8BF09
:1096B800FF23511C21601370A96881F3100189B23E
:1096C8002046F8F79BF81F4B20461988F8F796F8BC
:1096D800296801F30F0189B220460125F8F78EF8B1
:1096E8002B46DAE50B2218492046F8F759F80822E4
:1096F80016492046F8F754F8012507221449204650
:10970800F8F74EF82B46C8E5002A3FF4E0AD114BB8
:10971800136001252B46C0E5964D00201C4D002006
:10972800544F0020304D00209C770020C92D01089F
:10973800F14B0020B8340308882E0020BC2E0020EE
:10974800E857002084770020B0640308BC6403084D
:10975800C8640308E51C0108CC2E00200060002026
:10976800726835687B623046551BF7F7F2FF052DA6
:1097780038627B6A01F2B8818026B346012594E8F5
:109788000600521A103AB242B8BF1FFA82FB944A36
:10979800396A92683A61521A9345396A7B6220465F
:1097A800FA6088BF1FFA82FBF8F711F87B6A002B72
:1097B80001F07881002D41F0F7802368C7F800D0C8
:1097C8005D71C0B00533C7F804D0FB61BBF1000F71
:1097D80001F0FD823B6A3A69934281F0F4823E6A65
:1097E8007D62AA46A846BC608025FB68A3EB0808F2
:1097F8007B4BB8F5807F9B6828BF4FF4807806EBD9
:1098080008029A4288BFA3EB0608F8F70FFD7C68A8
:10981800424621463046F8F78FFDF969B86104EBF6
:10982800000C0B787B6164452ED2DFF8C4910CF1F3
:10983800FF3C04F1FF3E1EF8013F09EB830219F8D3
:1098480023405688ECB100234FF4004204F1FF385E
:1098580032424FEA520202D00878284308706D0855
:1098680006D10AF1010A4D701FFA8AFA01318025E2
:10987800D34503D8E6456CD343456ADB01339C42A4
:10988800E6D1F445D7D1F9617B6ABA6913449BB232
:10989800D3457B6206D97B6A3A6A9846D6183B69F3
:1098A8009E42A2D3BC68802D1CBF0AF101031FFA97
:1098B80083FA0AF1020189B22046F7F79FFF23686D
:1098C800796A01255A19226020461D70F7F796FF1C
:1098D8002368534423602B46D7F800D0DDE4414B7E
:1098E80085E63388FF2BA8BFFF23DBB26BE417F0B4
:1098F8002BFE00283FF466AC03780A2B2FD8B0F96A
:10990800023088FB0312DB17C3EBA2039BB2FF2BC9
:10991800A8BFFF23DBB256E4334A92E8220068E688
:1099280098E8220065E617F00FFE00283FF448AEDD
:1099380003780A2B3FF644AEB0F90430B0F90610AC
:1099480003EB830383F3500521EAE171ADB289B2D9
:1099580038E6FB69BC681A463B7D1370A3E7002311
:10996800D8E7552D17D0572D44D14FF0FF352B464A
:1099780093E4531C336013780A2B01F0C9803046F6
:10998800F7F709FF3046F7F706FF01253046F7F7E6
:1099980002FF2B4681E4531C336092F80080B8F133
:1099A800FF0F01F04D81B8F1FE0F01F0C080304685
:1099B800F7F7E6FE96E80C009B1A002B07DD531C10
:1099C800336013781BB9B8F10C0F41F27781B8F105
:1099D800270FCAD8054B012523F818002B465CE44D
:1099E8004C1A0020C02E0020D82E0020107700200E
:1099F800C834030870680B3D811AEF2DB5D80FF2F3
:109A0800080E5EF825F000BFC7A800087399000883
:109A180073990008739900087399000873990008EE
:109A280073990008739900087399000873990008DE
:109A380073990008739900087399000873990008CE
:109A480073990008739900087399000873990008BE
:109A580073990008739900087399000873990008AE
:109A68007399000873990008FDA800087399000805
:109A780071A50008739900082BA7000873990008BE
:109A8800739900087399000803A7000873990008E0
:109A9800A9A600087399000877A60008739900081A
:109AA80051A60008739900083FA60008739900089A
:109AB800E7A500087399000893A5000873990008A2
:109AC800739900087399000873990008D7920008E1
:109AD80073990008D5A700087399000873990008BE
:109AE800BBA700087399000861A7000873990008CC
:109AF80073990008739900087399000855A700081E
:109B080073990008739900087399000887A80008DA
:109B18007399000839A80008739900087399000818
:109B28002FA5000873990008739900087399000815
:109B380073990008739900087399000873990008CD
:109B4800C1A4000873990008A5A300087399000828
:109B580033A30008739900089BA2000873990008B2
:109B680073A200085FA4000819A4000873990008EC
:109B7800739900087399000873990008739900088D
:109B8800739900087399000873990008739900087D
:109B9800739900087399000873990008739900086D
:109BA800739900087399000873990008739900085D
:109BB800739900087399000873990008739900084D
:109BC800739900087399000873990008739900083D
:109BD800739900087399000873990008739900082D
:109BE800739900087399000873990008739900081D
:109BF800739900087399000873990008739900080D
:109C080073990008739900087399000873990008FC
:109C180073990008739900087399000873990008EC
:109C280073990008739900087399000873990008DC
:109C380073990008739900087399000873990008CC
:109C480073990008739900087399000873990008BC
:109C580073990008739900087399000873990008AC
:109C6800739900087399000873990008739900089C
:109C7800739900087399000873990008739900088C
:109C8800739900087399000873990008739900087C
:109C9800739900087399000873990008739900086C
:109CA800739900087399000873990008739900085C
:109CB800739900087399000835A40008739900087F
:109CC80057A200082DA2000873990008739900088C
:109CD800739900087399000873990008739900082C
:109CE800739900087399000873990008739900081C
:109CF800739900087399000873990008CFA10008A8
:109D08007399000897A1000873990008F5A0000846
:109D180095A0000879A00008739900085FA00008C2
:109D28007399000837A0000873990008D79F0008A6
:109D380073990008A79F0008739900087399000891
:109D48007D9F00084F9F00083B9F0008139F000855
:109D5800F39E0008C99E00087399000873990008CB
:109D6800739900087399000873990008739900089B
:109D7800739900087399000873990008739900088B
:109D8800739900087399000873990008739900087B
:109D98007399000873990008A99E00087399000830
:109DA800739900084F9E000873990008739900087A
:109DB80073990008EB9D00087399000873990008CF
:109DC80073990008D19D0008B74B1B78DB073FF556
:109DD800CCAD0125F9F712FEF9F7ECFF2B46FFF79A
:109DE8005CBA3046F7F7CCFC3368B8851A46591C7C
:109DF800316012F8021B326087F82E105A7887F803
:109E08002F20DA1C32609A7887F830201A1D3260C9
:109E1800DA7887F831205A1D32601B7987F832309A
:109E280007F12C000023BB86F7F706FC9F4AA04BDE
:109E38001268801A4FF0010561F10001C3E90401BD
:109E48002B46FFF72ABA531C336013780F2B3FF6C3
:109E58008CAD911C3160C3EBC30396495078C8544C
:109E6800D01C30600B4491785970111D3160D17845
:109E78009970511D31601179D970911D31605179F6
:109E88001971D11D31609179597102F10801316060
:109E9800D2799A7101251EF0B3FC2B46FFF7FDB964
:109EA8003046F7F76DFCDFF81482A8F80E0030464C
:109EB800F7F766FC0125A8F80C002B46FFF7EDB96B
:109EC8003046F7F75DFCDFF81482A8F8100030463A
:109ED800F7F756FCA8F812003046F7F751FC0125B1
:109EE800A8F814002B46FFF7D8B91346511C316067
:109EF80013F8020B3360D31C51783360927819F051
:109F080083F800287FF4E3A92FE51346511C31603C
:109F1800694913F8020B08703360684953788B70ED
:109F2800D31C3360664B92789A7001252B46FFF755
:109F3800B4B9644B644918684E22012527F0B8FF6C
:109F48002B46FFF7AAB91146531C33605F4B11F833
:109F5800020B1870316051785970D11C31609278B9
:109F68009A703046F7F70CFC594B0125D8802B46E0
:109F7800FFF793B93046F7F703FCDFF85481A8F8E8
:109F880000003046F7F7FCFBA8F802003046F7F768
:109F9800F7FB0125A8F804002B46FFF77EB9DFF888
:109FA800409199F80030002B3FF491A9DFF83481F3
:109FB80000253046F7F7E4FB0CF06CFD99F800300B
:109FC800A8EC010A01359D42F3DBFFF780B90D29A2
:109FD8007FF4CBAC531C33601578072D3FF6C5AC26
:109FE800DFF8049130464FF00C08F7F7C9FB08FB7F
:109FF80005F809EB0805A8803046F7F7C1FBE880AB
:10A008003046F7F7BDFB336828811A46591C316082
:10A0180012F8021BA97232605B78EB723046F7F7D0
:10A0280098FB012549F808002B46FFF736B9531C61
:10A0380033601078060600F188861B4B1B78DD0715
:10A048003FF545A9032828BF00200125F9F7BAFCE8
:10A058002B46FFF722B9144B1B78D8073FF537A9D1
:10A068000125FAF771F8F9F7A5FE2B46FFF715B9A0
:10A078000D4B1B78DA073FF52AA9164A13780125F4
:10A0880043F0040313702B46FFF707B9064B1B7800
:10A09800D9073FF51CA9104B4FF4C87201251A8047
:10A0A8002B46FFF7FAB800BF4D760020F075002068
:10A0B80040240020FC560020906C002010600020F6
:10A0C80020600020C44F0020143F030808600020CF
:10A0D8006C3900207C770020687900202C710020E2
:10A0E800F14B0020105900203C56002009297FF729
:10A0F8003CACDFF8B8831346511CD8F800503160E7
:10A1080013F8021B297033605378AB70D31C33608B
:10A118009378642B02F10401A8BF64236B7131604A
:10A12800D378642B02F10501A8BF6423AB713160B9
:10A138001379EB71931D33605379642B02F1070196
:10A14800A8BF64232B7231609379EB7002F1080386
:10A158003360D3792B713046F7F712FB7268336896
:10A168006881D11A00290CDD591CD8F8000031602B
:10A17800521A002A1978417203DD9A1C32605B7802
:10A18800437001250DF0FEFA2B46FFF786B8B94B50
:10A198001868D31C014621329D1E356013F8035CF4
:10A1A8000D705D1E356013F8025C4D70336013F856
:10A1B800015C8D7003339A4201F10301ECD10CF07C
:10A1C80039FBFFF784B8C1F34705122D3FF6CDAB35
:10A1D800C5B107F1500307F12A0A03EB4508D14638
:10A1E800A8F126083046F7F7CBFA29F8020FC1453F
:10A1F800F8D1A14B3AF8022F23F8022FD145F9D113
:10A20800112D09D89D4A6B00023B134400212232CC
:10A2180023F8021F9A42FBD1994A01231D46137065
:10A22800FFF73BB8531C974833600178137800292F
:10A2380040F0518504220270934A9B001380FBF77B
:10A248008DF8924B012598612B46FFF726B8DFF869
:10A25800608200233046C8F80030F7F77AFA012503
:10A26800C8F800002B46FFF718B81346511C316098
:10A27800874913F8020BC8703360864953784B71CD
:10A28800D31C3360844B9278DA7001252B46FFF794
:10A2980004B83046F7F774FA3046F7F771FA3046E3
:10A2A800F7F76EFA3046F7F776FA3368714D1946C4
:10A2B800581C2A68306011F8020B82F82C003160B3
:10A2C800597882F83610D91C31609B7882F837307B
:10A2D8003046F7F760FA3046F7F75DFA3046F7F799
:10A2E8005AFA3046D5F80080F7F74AFAA8F83A0043
:10A2F8003046D5F80080F7F743FA33687268A8F853
:10A308003800D11A01290ADD591C2A6831601B78E6
:10A3180082F82E303046F7F73EFA33687268D31A5F
:10A32800032B00F31D85286849E7531C3360514D02
:10A33800DFF88081137888F805303046D5F800902A
:10A34800F7F71EFAA9F820003046D5F80090F7F77D
:10A3580017FA72683368A9F81E00D11A072900F3A2
:10A36800D884D11A032900F36685D21A002A05DD9C
:10A37800591C2A6831601B7882F82630F9F77CFC72
:10A3880022F01EF9454B1B68002B00F0F784286863
:10A3980001250BF0BFFE2B46FEF77FBF1346511C6D
:10A3A8003160DFF8108113F8021B88F8021033605F
:10A3B8003B4953780B70D31C33603A4D93782B711B
:10A3C800131D3360D378092BA8BF09233046AB701F
:10A3D800F7F7D6F9336872682880D11A012905DDA4
:10A3E8003046F7F7CDF933687268E8819A4240F051
:10A3F8008084F9F741FC336872689A423EF467AF8B
:10A408005A1C32601B78EB7001252B46FEF745BFBE
:10A41800531C33601378002B00F062844FF4004023
:10A42800012508F081FC2B46FEF737BF1346511C67
:10A43800316013F8025B3360D31C50783360917835
:10A44800002D00F06084012D7EF441AF0AF030FB4E
:10A458002B46FEF722BF144B1B7813F001017FF443
:10A4680084AA531C3360107801250AF05BFA2B4646
:10A47800FEF713BFC44F00207A5900207C590020F2
:10A4880078590020224700208477002040240020AB
:10A49800106000204879002020600020F04700204C
:10A4A800046000202C7100204D760020C84F002049
:10A4B800E8570020906C0020CF4B1B68002B3EF41F
:10A4C80006AF1CF0A3FCFF283EF401AF3046F7F7B7
:10A4D80057F93F2840F2BD84DFF84883002588F803
:10A4E800005033687268A8F80400D21A012A7EF76F
:10A4F800EEAE1A46591C316012F8021B88F8021099
:10A5080007F15000326000225D7800F8242D1CF01D
:10A518004FFC97F82C30AB423EF4D9AE28461CF0DD
:10A528006BFCFEF7D4BEB54B1B78012B3EF6CFAEC5
:10A538001146531C3360DFF8F08211F8023B88F8AB
:10A5480002303160D31C92F801E03360C31A012B4A
:10A55800917840F31E843046F7F712F90125A8F8E0
:10A5680000002B46FEF799BEDFF8C0820023C8F82A
:10A5780000303046F7F7EDF8D8F8003001250343EE
:10A58800C8F800302B46FEF788BE0723B1FBF3F36B
:10A59800C3EBC305491B7FF4E8A9DBB203F1FF391C
:10A5A8005FFA89F9002B3EF492AEDFF854A209F164
:10A5B80001090D46531C336092F90020904B4FF06F
:10A5C800000893F90210914203F1080300F0138385
:10A5D80008F10108B8F1050FF3D1FFF7C6B9531C0C
:10A5E800336013780E2B3FF6C0A9911C3160557863
:10A5F800032D3FF6BAA98348062101FB03F143184E
:10A6080002F1030E5D71C6F800E095784554111DFE
:10A618003160D1785970511D316011799970911D4F
:10A6280031605179D970D11D316092791A71012543
:10A638002B46FEF732BE531C3360734B12785A75A3
:10A6480001252B46FEF729BE531C336015781F2DB4
:10A658003FF68BA905297FF488A93046F7F779F8E2
:10A668006A4B43F8250016F029F8FEF730BE674D0F
:10A6780005F140083046F7F783F83368A5F88000FD
:10A68800591C1A46316012F8021B85F88210326094
:10A698005B7885F883300435A845EBD1FEF717BE03
:10A6A800531C594D336013782B723046F7F768F80E
:10A6B800A8833046F7F764F828833046F7F760F840
:10A6C80032686883531C33601278EA747268D31A4C
:10A6D800032B00F391833368D11A052900F37C8397
:10A6E800D21A002A7EF7F3AD5A1C32601B7885F81F
:10A6F800213001252B46FEF7D0BD531C3360444959
:10A7080015780D70C01A00287EF7E1AD931C3360F0
:10A718005378003318BF012301254B702B46FEF7F1
:10A72800BCBD3046F7F72CF8DFF8E880C8F8000021
:10A738003046F7F725F8C8F804003046F7F720F850
:10A748000125C8F808002B46FEF7A7BD0125F7F735
:10A75800CFFD2B46FEF7A1BD531C33602C4B12785E
:10A76800DFF8C8801A700023C8F800303046F6F7C2
:10A77800F0FF3368D8F800202349264D10435A1CAF
:10A78800C8F8000032601B780B723046F6F7F8FF05
:10A7980028603046F6F7F4FF68603046F6F7F0FFB9
:10A7A800A8603046F6F7ECFF3046F6F7E9FFFEF70B
:10A7B8008EBD194B02F108010132326012F8010C0A
:10A7C80003F8010F9142F7D1FEF781BD1346511CE2
:10A7D8003160124913F8025B8D70336055784D7003
:10A7E80083423EF474ADD31C33600D4B92781A72D9
:10A7F80001252B46FEF751BD50760020623C002013
:10A80800485D0020F45700201C5D002010500020F7
:10A818000C480020C03600201B5D0020306000205E
:10A8280040240020547600207E770020743C0020CD
:10A83800531C336092F80080B8F1110F3FF695A8C9
:10A84800931C3360C34D537805F818303046F6F73B
:10A8580097FF40F6CA039842A8BF184640F2EE2375
:10A86800984205EB4801B8BF18460125A0F2EE2230
:10A878002B46192092FBF0F24A70FEF70EBD1346E4
:10A88800511CB54D316013F8021B297133605378A0
:10A898006B713046F6F774FF336828805A1C3260B3
:10A8A8001B78AB713046F6F76BFF336868805A1C2B
:10A8B80032601B78EB7101252B46FEF7EEBCA74BE7
:10A8C80010294FF0000228BF10211A605A609A60C0
:10A8D800DA601A7400293EF4FAAC3268013B11447C
:10A8E8000132326012F8010C03F8010F8A42F7D1E5
:10A8F800FEF7EDBC511C316015783B62132D3FF615
:10A9080034A8911C316050787A6209F005FC00285F
:10A918003FF42BA87A6A9249007801F82500D01CE8
:10A92800306001EB850590786870101D3060D07834
:10A93800A870501D30601279EA703B6A01F150022C
:10A9480002E004318A4207D008780028F9D18D78CE
:10A95800C8788542F5D20123824A83F00103012594
:10A9680013702B46FEF799BC1346511C31607E4D7F
:10A9780013F8021B6970336053782B70D31C336053
:10A988009378AB703046F6F7FBFE33682881591C84
:10A998001A46316012F8021B697132605B78AB713C
:10A9A80001252B46FEF779BC704B3A6A9B68D4F8B0
:10A9B80000905A449A4200F27081F7F737FC5A46E1
:10A9C8004946386AF7F7B8FC23680344236086428F
:10A9D8007EF77DAC002100E0236801305A1CB042AC
:10A9E80022601970F8D1FEF772BC336872689A4217
:10A9F80040F0CE805E4BFF221A704FF0000A5D4D8A
:10AA080012F0CEFC514620225B4885F800A028F0C1
:10AA1800E0FB87F82CA097F82C30072B00F259811F
:10AA2800DFF86491544E524697F82C3003EB4303F9
:10AA380009EBC3035B7CE3B197F82C3003EB4303CA
:10AA480009EBC30320215B699BB197F82C3003EB1A
:10AA5800430309EBC303586946F82200F5F791FF51
:10AA68002B7856F82300F6F74DF92A780132D2B23E
:10AA78002A7097F82C300133DBB287F82C3097F81E
:10AA88002C30072BD0D92368591C21601A70B8F1D3
:10AA9800000F3EF41CAC394BC8F8003001252B469A
:10AAA800FEF7FBBB002D7FF47FAF59462046F6F733
:10AAB800A5FE23685A1C22601D702C4B26689D68D1
:10AAC8003B6A0BEB0302AA4240F26F813B6AED1A24
:10AAD800F7F7ACFB2A463146386AF7F72DFC2368AE
:10AAE80003442360FEF7F3BB3046F6F749FE3268AD
:10AAF80071687B6A9142834673D106461D46FEF70C
:10AB08003EBE3046F6F73CFEDFF88080FEF79DBC7F
:10AB1800931C33601A4B51781970D11C31609178AD
:10AB28005970111D3160D2789A70FEF7D0BB931C12
:10AB380033605578022D3EF618AF3046F6F720FE02
:10AB4800104B03EB45034FF0FF35A3F856002B4697
:10AB5800FEF7A3BBA441002088390020EE54002052
:10AB680094400020AC200020544F00204C1A0020B4
:10AB780040240020B35A0020745A0020E55D0208E2
:10AB88002F3B0020107700206C7000200060002010
:10AB98005A1C19463260B74811F8022B027031600E
:10ABA8005B784370042A03D9FF2A7EF43AAB24E782
:10ABB800B1490978994205D8022A7EF432ABFF2BB5
:10ABC8007EF42FAB236801255A1922601D70B8F155
:10ABD800000F3EF47CABA94BC8F800302B46FEF7BB
:10ABE8005CBB511C316012781D46131C064618BF09
:10ABF8000123FEF7C4BD0AEBC80B30468BF80220D0
:10AC0800F6F7BEFD33682AF838001A46591C316039
:10AC180012F8021B8BF8031032605A788BF8042064
:10AC2800DA1C32609A788BF806201A1D32600135DA
:10AC3800DB788BF80530A9457FF4BCACFEF747BB41
:10AC48003046F6F7A8FD3368DFF834821A46591CF7
:10AC5800316012F8021B88F8551032605B7888F86A
:10AC680054303046F6F78CFDA8F850003046F6F719
:10AC780087FD3046F6F784FD96E80C009B1A012BF9
:10AC8800A8F852007EF723AB3046F6F779FD012588
:10AC9800A8F85A002B46FEF700BB3A6AA3EB020855
:10ACA800F7F7C4FA42464946386AF7F745FB23687E
:10ACB80003442360002D3EF40AAB88E6704B003055
:10ACC800984418BF0120012588F85E002B46FEF73E
:10ACD800E4BA5246D7E604297EF4F9AAFFF7ACBADB
:10ACE800684A1368012523F4004313602B46FEF7D6
:10ACF800D4BA5A1C32601B78003318BF012388F875
:10AD08000730FFF776BB01250BF022FC2B46FEF738
:10AD1800C4BA3046F6F734FDA8F80A003046F6F70C
:10AD28002FFDA8F80C003046D5F80090F6F728FD5E
:10AD3800A9F822003046D5F80090F6F721FD3368CF
:10AD48007268A9F82400FFF70CBB00F07F00032805
:10AD580028BF0020012509F0C7FE2B46FEF79DBA43
:10AD68003046D5F80080F6F70BFDA8F832003046DB
:10AD78002E68F6F705FDB086FFF7D5BA4248434975
:10AD8800434A444B036001250B6013602B46FEF7D2
:10AD980084BA414B1A88012512FB0EF22B4692FB0E
:10ADA800F1F2A8F80020FEF778BAF7F73FFA5A460A
:10ADB8003146386AF7F7C0FA23680125034423604F
:10ADC8002B46FEF76ABA7D62AA46FEF772BDDA46DE
:10ADD800C7F824B0FEF76DBD5A1C32601B78EB72C1
:10ADE8003046F6F7B6FC3368E8605A1C32601B78C8
:10ADF8002B743368726873E43046F6F7C1FCA88494
:10AE08003046F6F7BDFC33687268E884D11A032926
:10AE18007FF762AC1A46591C316012F8021BA977F9
:10AE280032605B7885F820303046F6F7A9FC336845
:10AE38007268688450E43046F6F7A2FCA8F80E0061
:10AE48003046F6F79DFC33687268A8F81000FFF7E3
:10AE58008CBAC50800F0070301350133EDB2DFF8FD
:10AE68003C802846194688F8013016F013FBFFF796
:10AE780036BB00BF40240020F14B0020FD1C010818
:10AE880010770020BC4F0020A8370020FC37002096
:10AE9800643800205F0500086C5E002054760020AE
:10AEA8002DE9F04F2DED0E8BDFF8F4B097B0DBF8FD
:10AEB8000420079058469047002800F08E82BBF87F
:10AEC800A87000218BF85110002F6DD1BBF93A0002
:10AED800DBF82450DBF82810BBF93860DBF8204099
:10AEE800BBF93C20DFF8BCA0401B521ACBF830005D
:10AEF8009BF85210CBF83420341B0BF12C00CBF804
:10AF08002C4014F0D9FCDAF80020910041F179873F
:10AF1800DBED0C5A1F4CDBED0B7A1F4994ED406AB0
:10AF2800D4ED416A94ED427AD4F80C2109681B4BA0
:10AF38000593B8EEE58ADBED0D5AF8EEE77AF8EE00
:10AF4800E58A013277EE867A38EE268A78EE878AA5
:10AF58008A42C4ED407A84ED418AC4ED428AC4F83D
:10AF68000C2101F04A8393F800E0BEF1140F02F0BF
:10AF78009B870023D4F814510693062D01F2978479
:10AF8800DFE815F00416161728152917020CC6163F
:10AF98008A1500BF68240020B0430020104C002010
:10AFA800A46C00202C6F0020DE4BDF481A68089341
:10AFB8004FF47A76B6FBF2F2C2EB421602EB860247
:10AFC800D600DA4BDFF8C88344780593B6B2B742A7
:10AFD8001D78B8F9060003F08980DBF87C30BBF9EE
:10AFE8003810DBF8602003F1010E07EE901A0A44CE
:10AFF800BEF1010FCBF87CE0CBF86020F8EEE77AE1
:10B0080003F08180DBED1B5ADBED1D6A07EE10EAC9
:10B0180037EEE56AB8EEC75A012F86EE057A37EEA5
:10B02800257A77EEC77A8BED1C7AE7EE866A8BED88
:10B038001B7AF0EE667ACBED1E6ACBED1D6A03F043
:10B048000384DBF89030BBF93A10DBF8642003F195
:10B05800010E07EE901A0A44BEF1010FCBF890E0FA
:10B06800CBF86420F8EEE77A03F06880DBED205A2D
:10B07800DBED226A07EE10EA37EEE56AB8EEC75A4A
:10B08800012F86EE057A37EE257A77EEC77A8BEDB3
:10B09800217AE7EE866A8BED207AF0EE667ACBEDC0
:10B0A800236ACBED226A03F0A783DBF8A430BBF94F
:10B0B8003C10DBF8682003F1010E07EE901A0A44F1
:10B0C800BEF1010FCBF8A4E0CBF86820F8EEE77AE0
:10B0D80003F04F80DBED255ADBED276A07EE10EA17
:10B0E80037EEE56AB8EEC75A012F86EE057A37EED5
:10B0F800257A77EEC77A8BED267AE6EE276A8BED0E
:10B10800257AF0EE667ACBED286ACBED276A03F054
:10B118006683874CA8F80600BBF8A820059B013A6F
:10B128001D78ABF8A82008990022072D4A608A608C
:10B13800CA6040F05981FAF711F9059BDFF850828F
:10B148001D78079BC01A94F82831A8F800000993C5
:10B15800002B40F04F81744A5279002A01F07A811D
:10B16800744A1278013AD2B2072D84F8282102F0E5
:10B178001A8200230A93704BD4F83421D3F800A024
:10B18800684B0893079B9FED6D6AD4ED4C9A6C4908
:10B19800C4F834319A1A07EE902AF8EE677AB7EEB7
:10B1A800007AC6EE278A0025664BDFF8E891DFF8BB
:10B1B800E881654F06932E46D1ED006A94ED4BDA8F
:10B1C8009FED629ADFED62AA9FED62CA9FED62AAC7
:10B1D800DFED62BA9FED62BA77EE69CA6CEEA6CA75
:10B1E800F4EEC7CAF1EE10FA88BFF0EE47CA5D4B1D
:10B1F80099ED008A2B44D3ED007AF5EE407AF1EE12
:10B2080010FA17D0584B2B4493ED007A78EE476A22
:10B21800B0EEE66AF4EEC67AF1EE10FA08D5F5EE6D
:10B22800C06AF1EE10FACCBF37EE878A37EE678A2C
:10B2380083ED008A4D4B1A88930739D0022E37D0F8
:10B248009AF82E104A4B07EE901A2B4493ED007A89
:10B258004B42F8EEE76A07EE903A26EE877AF8EE68
:10B26800E77AB4EEE77AF1EE10FA0AD407EE901A0C
:10B27800F8EE677AF4EEC77AF1EE10FA88BFF0EECE
:10B28800477A3C4B3C4903EB460331F91600B3F9C6
:10B298000C30C31A07EE103AB8EEC77AD007E7EEBB
:10B2A800497A41F17380354B93ED008A27EE888AFD
:10B2B800089B94F868212B4493ED01EA78EE4EDA66
:10B2C800002A00F0F7802E4BD4F86C2107991B68F0
:10B2D8008A1A9A4240F3EE809AF84830022B02F01C
:10B2E800A181022E04F04584264B1B68990700F1C2
:10B2F8009780254B87ED00CA1B689342C0F2CA802D
:10B30800F7EE007AF4EEE79AF1EE10FA40F1D28007
:10B3180008991E4BD1ED017A93ED007AF0EEE77AA9
:10B328003CE000BF1C6F0020906C0020104C0020F7
:10B338006824002004600020C44F002000247449C1
:10B34800B83800206C47002078470020CDCCCC3D91
:10B35800AE47813F000000000000C84200003443AF
:10B36800610BB63BAC380020AC250020C04F002054
:10B37800B825002010600020704F0020943800206D
:10B38800C0380020644F0020BC380020C838002096
:10B39800144C0020A025002084470020F4EEC77A32
:10B3A800F1EE10FA40F18680D1ED027AF0EEE77AFC
:10B3B800B4EEE77AF1EE10FA7CDDD1ED037AF0EE27
:10B3C800E77AB4EEE77AF1EE10FA73DD0F4B1B68FB
:10B3D8009B075FD50E490F4B43E00F4B0F4C1D7871
:10B3E8000593072D3FF4A7AE94F828310993002B55
:10B3F8003FF4B1AE013B84F82831012D01F0A88259
:10B4080017B0BDEC0E8BBDE8F08F00BF644F002075
:10B41800704F002010600020104C0020682400208D
:10B42800D34BD449DFF8C8E331F916C09EED008A42
:10B43800DFF8C0E387ED00CA03EB460028EE098A6F
:10B44800B0F90C00A0EB0C0007EE900AF8EEE77AD2
:10B45800DEF8000027EE888A904278EE4EDABFF6D2
:10B468004FAFB3F90C20B1F900E0C348AEEB020EC0
:10B4780000688EEAEE72A2EBEE7282421ADAB3F933
:10B488000E30B1F90220D21A82EAE273A3EBE2731A
:10B4980098420FDDB94B1A88002384F86831002AD6
:10B4A80043F06A85B64AB74B1178186881F00101F4
:10B4B800F5F72DFCB44B2B4493ED000A069B2DEEBB
:10B4C800000A022E20EE2D0AA3EC010A069304F0CE
:10B4D8000D83AE4BD7ED006A93ED007AAC4BD3EDFC
:10B4E800007AAC4B93ED006AAB4B67EE277A2B449E
:10B4F80027EEAC7AD3ED007A67EE277AF0EE665A3B
:10B50800EDEEA75AB1EE467AB4EEE57AF1EE10FA0E
:10B5180008DCB4EEE56AF1EE10FA8CBFB0EE657A9D
:10B52800B0EE467A94ED4C6AF7EE007AB4EEE76A2C
:10B53800F1EE10FAACBF0123002343B1F0EEE66A46
:10B54800F0EEC77AF4EEE67AF1EE10FA01D587ED5F
:10B55800007A022E04F0AC82904A914B52F82600F1
:10B568001B68B0EE4E0A98478E4A8F4B52F8260059
:10B578001B6898479AF8373023B18C4B1B88002BEF
:10B5880000F06B87B0EE4C8A894B38EE400A2B44AA
:10B5980093ED008A83ED000A9AF8483030EE480AA5
:10B5A80020EE288A002B33D0824B1B7813F001033E
:10B5B80000F0B886F7EE007AF4EEE79AF1EE10FAAA
:10B5C80094F86831C1F2E684002B00F0EB87D4F8D8
:10B5D8006C31079AD31A784A12689A4218DD774B69
:10B5E800D3ED007AF0EEEDDAF4EEE7DAF1EE10FAE8
:10B5F80042F12980614B1A88002384F86831002AB7
:10B6080000F09C866E494A6912B10A6813604B744F
:10B618006C4B94F878212B4493ED000A2DEE000A28
:10B6280020EE088A88ED008A32B9069B87ED00CAA9
:10B6380003ED01CA88ED00CA0136032E09F1040999
:10B6480008F1040807F1040705F104057FF4CFADFC
:10B65800059B1A78072A01F0B384012A01F0908724
:10B668000023069394F88021002A41F07E81DFF8B8
:10B6780088A1554BDAF800201968D60491F82C00F7
:10B6880000F10687DFF87491504AB9F81A3092ED44
:10B69800006A4F4A4F4DD2ED005AD5ED036A4E4A23
:10B6A80084ED646A07EE103A4C4B92ED005AD3EDE4
:10B6B800007AD3ED013AD3ED024A84ED626AB8EE1E
:10B6C800C77A35EEC64A012236EEC77A84ED614A5A
:10B6D800C4ED655A84F89821C7EE055A0A8D53427D
:10B6E80006EE103A3E4BDFED3F6A93ED005A3E4BB3
:10B6F80093ED004AB7EE007AF4EEC75A35EE045AD5
:10B70800F1EE10FA88BFF0EE475A35EE275AB8EE38
:10B71800C66AF4EEE65AF1EE10FA07EE902AB4EE95
:10B72800C65AB8BFF0EE665AF1EE10FAC4ED685A80
:10B73800B8EE677A01F10483B4EEC75AF1EE10FA55
:10B7480088BFB0EE475A264BDFED286AD3ED017A61
:10B75800254B93ED014A77EE847A25EE265A77EE4B
:10B76800A37AB4EEE76AF1EE10FA52DC48E000BFC3
:10B7780010600020704F0020C4380020C8750020D9
:10B78800CA750020CC75002068380020A437002036
:10B7980004000020DC38002074380020AC3700207A
:10B7A800A837002000380020FC370020C04F0020B8
:10B7B800D82500204D760020C0380020CC38002045
:10B7C800D075002080380020C44F0020885E0020FB
:10B7D800F45F0020984D002074390020784700203D
:10B7E8006C47002000000000844700206F12833A55
:10B7F80094380020BC3800202C6F00201C5D0020ED
:10B80800B4EEE77AF1EE10FA8CBFB0EE676AB0EEEC
:10B81800476AEC4B4A8DD3ED027A9FEDEB7A53429F
:10B8280004EE103A74EEA77AB8EEC44A26EE076A18
:10B83800F4EEC47AF1EE10FA0AD407EE102AB8EE44
:10B84800474AB4EEE74AF1EE10FA88BFB0EE674A0D
:10B85800DE4ADFEDDD7A527824EE274A0AB9B1EEE6
:10B86800444A002841F0D085B7EE003AD84E3278E5
:10B87800002A02F04B86D749DFEDD77AD1ED024A8C
:10B88800D1ED016A91ED037A66EE244AE5EE264A87
:10B89800E4EE074A63EE244AF4EEE74AF1EE10FAC2
:10B8A800B4BFF0EE673AF0EE643A98BFF0EE647A0F
:10B8B800012ACDED0E4A02F04E8691ED067AD1EDC1
:10B8C800052AD1ED076A26EE077AA5EE227AA4EEBC
:10B8D800267A23EE077AB4EEE77AF1EE10FAB4EEA0
:10B8E800E37A8CBFF0EE676AF0EE476AF1EE10FA81
:10B8F80088BFF0EE676AB4BFF0EE637AF0EE477A7D
:10B90800022A8DED0F7A00F0DE8091ED0A7AD1EDF2
:10B91800092AD1ED0B3A26EE077AA5EE227AA4EE93
:10B92800237A23EE077AB4EEE67AF1EE10FAB4EE53
:10B93800E77A8CBFF0EE663AF0EE473AF1EE10FA8D
:10B9480098BFF0EE636AA8BFF0EE477A032A8DED40
:10B95800107A00F0B88091ED0E7AD1ED0D2AD1ED74
:10B968000F3A26EE077AA5EE227AA4EE237A23EE82
:10B97800077AB4EEE67AF1EE10FAB4EEE77A8CBF05
:10B98800F0EE663AF0EE473AF1EE10FA98BFF0EEB4
:10B99800636AA8BFF0EE477A042A8DED117A00F0A9
:10B9A8009280D1ED123AD1ED112A91ED137A66EE1B
:10B9B800233AE5EE223AE4EE073A63EE233AF4EE50
:10B9C800E63AF1EE10FAF4EEE73A8CBFB0EE667A9A
:10B9D800B0EE637AF1EE10FA98BFF0EE476AA8BFAE
:10B9E800F0EE637A052ACDED123A6CD0D1ED163A15
:10B9F800D1ED152A91ED177A66EE233AE5EE223A53
:10BA0800E4EE073A63EE233AF4EEE63AF1EE10FA82
:10BA1800F4EEE73A8CBFB0EE667AB0EE637AF1EEF8
:10BA280010FA98BFF0EE476AA8BFF0EE637A062ACC
:10BA3800CDED133A47D0D1ED1A3AD1ED192A91ED4F
:10BA48001B7A66EE233AE5EE223AE4EE073A63EE15
:10BA5800233AF4EEE63AF1EE10FAF4EEE73A8CBF48
:10BA6800B0EE667AB0EE637AF1EE10FA98BFF0EEB7
:10BA7800476AA8BFF0EE637A072ACDED143A22D0C0
:10BA880091ED1E7AD1ED1D2AD1ED1F3A26EE077AE7
:10BA9800A5EE227AA3EE847A27EE037AB4EEE67A4C
:10BAA800F1EE10FAB4EEE77A8CBFB0EE666AB0EE4B
:10BAB800476AF1EE10FA8DED157A98BFF0EE466AF6
:10BAC800A8BFF0EE477A77EEE67AF7EE006AF4EE72
:10BAD800E67AF1EE10FAC4ED4C7A43F3D78586EE98
:10BAE800A77A022ADDED0F7A67EE244A67EE877A95
:10BAF800CDED0E4ACDED0F7A2DD0DDED107A67EE43
:10BB0800877A032ACDED107A25D0DDED117A67EE1C
:10BB1800877A042ACDED117A1DD0DDED127A67EE11
:10BB2800877A052ACDED127A15D0DDED137A67EE06
:10BB3800877A062ACDED137A0DD0DDED147A67EEFB
:10BB4800877A072ACDED147A05D0DDED157A27EE30
:10BB5800877A8DED157A2149096811F080530A9387
:10BB680001F0CB81F6EE005AC4ED685A002A02F0C3
:10BB78009D8494F998311A4994ED656AC87894EDD2
:10BB8800645ADAF80010DFF868E0164FDEED004A74
:10BB9800B7F906E0B9F81A700B9707EE103A124B8E
:10BBA800D4ED616A1D78114BD4ED627A1B78089345
:10BBB800BDEEC66A01F4805316EE10CABDEEC56A22
:10BBC8000D9317E06C4700206F12833A0C48002051
:10BBD800F14B0020E438002000000000EC5F00205A
:10BBE800244B00203E6100204D760020507100203B
:10BBF800E038002001F4800301F01007B8EEC77A9E
:10BC08000C9305F0010816EE101A002840F064871E
:10BC1800002F41F0D582D34D9DED0E5A95ED006A67
:10BC2800D14825EE866AA5EE076AB0EE675AA6EEF9
:10BC3800265ABDEEC56A16EE10EA16EE107AE645EB
:10BC4800A8BF67467145C8BF0F4606EE107AB8EE22
:10BC5800C66A012A80ED006A00F0DC8095ED046A6E
:10BC68009DED0F5A25EE866AA5EE076AB0EE675A73
:10BC7800A6EE265ABDEEC56A16EE10EA16EE107A42
:10BC8800E645A8BF67467145C8BF0F4606EE107A5D
:10BC9800B8EEC66A022A80ED016A00F0BB8095ED15
:10BCA800086A9DED105A25EE866AA5EE076AB0EE81
:10BCB800675AA6EE265ABDEEC56A16EE10EA16EECB
:10BCC800107AE645A8BF67467145C8BF0F4606EE1D
:10BCD800107AB8EEC66A032A80ED026A00F09A80EC
:10BCE80095ED0C6A9DED115A25EE866AA5EE076A58
:10BCF800B0EE675AA6EE265ABDEEC56A16EE10EAF1
:10BD080016EE107AE645A8BF67467145C8BF0F46CC
:10BD180006EE107AB8EEC66A042A80ED036A79D076
:10BD280095ED106A9DED125A25EE866AA5EE076A12
:10BD3800B0EE675AA6EE265ABDEEC56A16EE10EAB0
:10BD480016EE107AE645A8BF67467145C8BF0F468C
:10BD580006EE107AB8EEC66A052A80ED046A59D054
:10BD680095ED146A9DED135A25EE866AA5EE076ACD
:10BD7800B0EE675AA6EE265ABDEEC56A16EE10EA70
:10BD880016EE107AE645A8BF67467145C8BF0F464C
:10BD980006EE107AB8EEC66A062A80ED056A39D032
:10BDA80095ED186A9DED145A25EE866AA5EE076A88
:10BDB800B0EE675AA6EE265ABDEEC56A16EE10EA30
:10BDC80016EE107AE645A8BF67467145C8BF0F460C
:10BDD80006EE107AB8EEC66A072A80ED066A19D010
:10BDE80095ED1C6A9DED155A65EE865AE7EE055AE3
:10BDF800E6EEA57AFDEEE77A17EE905AAC45A8BFB5
:10BE0800AC46A942D8BF614607EE901AF8EEE77A29
:10BE1800C0ED077AB8F1000F00F06C87534A12683A
:10BE2800002A40F07487524A127892B1307868B18B
:10BE38004D4FDFF85C810025E8B2D8F80030B7EC48
:10BE4800010A9847307801358542F5DB494A12687E
:10BE58009047059B1A78072A01F0A1800026DAF896
:10BE68000020530500F1D187434B1B78BBB1434AEF
:10BE7800B9F81A30B2F906209A4210DC404B1B7808
:10BE8800012B01F09583192B01F092830E2B06D01C
:10BE9800082B04D03B4D0023AB60C4F8403194F824
:10BEA800AA5125B1384B1B889F0741F02F8394F87E
:10BEB800B021002A40F0488799F81E70002F00F042
:10BEC8002984022F01F0D582032F41F0CE8299F800
:10BED8002030C3EB431103EB8101C90089B299F803
:10BEE8001F300233DBB2002A00F05585002900F02C
:10BEF800528526480768B1FBF7F10FB2A4F8E07144
:10BF0800002B03F0438007EE907AF8EEE77AF7EE1D
:10BF1800006A86EEA77A1B4D012BD4ED7D6AD5ED1C
:10BF2800007A77EEE67A67EE877AC4ED797A3BD0C5
:10BF3800D5ED017AD4ED7E6A77EEE67A022B67EECC
:10BF4800877AC4ED7A7A2FD0D5ED027AD4ED7F6A5C
:10BF580077EEE67A032B67EE877AC4ED7B7A23D0F7
:10BF680018E000BFE4380020CC470020005D002026
:10BF7800787400204C710020AC2000203E61002025
:10BF88000C480020984D0020C04F0020F0470020AA
:10BF980044710020D5ED037AD4ED806A77EEE67A15
:10BFA80067EE877AC4ED7C7A05990978092903F048
:10BFB800ED81002F40F3B4839BB394ED7D7AD4EDEB
:10BFC800797A77EE877A012BC4ED7D7AC5ED007A10
:10BFD80021D094ED7E7AD4ED7A7A77EE877A022BA7
:10BFE800C4ED7E7AC5ED017A15D094ED7F7AD4ED53
:10BFF8007B7A77EE877A032BC4ED7F7AC5ED027AD8
:10C0080009D0D4ED807A94ED7C7A77EE877AC4ED06
:10C01800807AC5ED037A013B022BB8BF0223DBB25D
:10C028000993099B002A18BF02239E46C84BDFEDDF
:10C03800C96A1A68059B91781878137807EE903AC0
:10C04800F8EEE77AB0EE007A67EEA67AF4EEC77AF1
:10C05800F1EE10FA40F35F86DFEDBF6A37EEC77A7C
:10C06800B0EE676AA7EE266AF0EE466A95ED007AAA
:10C078009FEDBA6A27EE066AF0EEC65A84ED546A56
:10C08800C4ED575A99B107EE101AB8EEC75A9FED8A
:10C09800B17A66EE064A25EE075AB7EE007A37EE11
:10C0A800457A64EEA54AA4EE857A26EE076A9FEDE6
:10C0B800AC7A537926EE877A27EE067ACBB1DFED94
:10C0C800A56A9FEDA86A65EEA65A06EE903AF8EEC4
:10C0D800E66A65EEA65AF4EEC65AF1EE10FA01F3D6
:10C0E8008981B7EE006A76EE655AC6EE256A27EEB4
:10C0F800267A0C289FED9C8ADFED9C6A00F0248745
:10C10800B4EEC87AF1EE10FA98BFB0EE478AB4EEF2
:10C11800E68AF1EE10FAB8BFB0EE668A84ED4E8A70
:10C12800BEF1000F00F0DD80B0EE007AF4EEC77AC1
:10C13800F1EE10FA05DD37EEC77ADFED876AE7EE34
:10C14800267A95ED017ADFED856A27EE267AF0EEFC
:10C15800C75A84ED557AC4ED585A99B106EE901A2B
:10C168009FED7C6AF8EEE66A27EE075A66EE866A65
:10C17800B7EE006A36EE666A25EE255AA5EE266AFF
:10C1880027EE067ADFED766A937967EEA67A67EE90
:10C19800877AABB107EE103AB8EEC77A9FED6D6AB1
:10C1A800DFED706A27EE257A27EE067AB4EEE67A96
:10C1B800F1EE10FA41F31081DFED6D6A67EEA67AB1
:10C1C8000C2800F0A186DFED686A9FED687AF4EE2E
:10C1D800E67AF1EE10FA88BFF0EE667AF4EEC77AE6
:10C1E800F1EE10FAB8BFF0EE477ABEF1010FC4EDD8
:10C1F8004F7A76DD5378DFED576A07EE903AF8EE1E
:10C20800E77AB0EE007A67EEA67A537AF4EEC77A48
:10C21800F1EE10FA05DD37EEC77ADFED4F6AE7EE8B
:10C22800267A95ED027ADFED4D6A27EE267AF0EE52
:10C23800C75A84ED567AC4ED595A9BB106EE903A26
:10C248009FED446AF8EEE66A27EE075A66EE866ABC
:10C25800B7EE006A36EE666A25EE255AA5EE266A1E
:10C2680027EE067ADFED3E6AD37967EEA67A67EEA7
:10C27800877AFBB107EE103AB8EEC77A9FED356AB8
:10C28800DFED386A27EE257A27EE067AB4EEE67AED
:10C29800F1EE10FA01F39C80B5EEC07AF1EE10FAD7
:10C2A80002F1FE82B7EE006A36EE477AC6EE076AFA
:10C2B80067EEA67A0C2800F06586DFED2B6A9FED05
:10C2C8002B7AF4EEE67AF1EE10FA88BFF0EE667A91
:10C2D800F4EEC77AF1EE10FAB8BFF0EE477AC4ED83
:10C2E800507A092800F0FC8599F82150002D40F07B
:10C2F800B185002384F8B0311E4B1B7823B91E4D3D
:10C30800AA78002A41F0C180059B1D78072D7FF48B
:10C3180074A8F9F723F8194B059A801B1578D8806B
:10C32800FFF76BB894F86821002A3FF471A9144A02
:10C3380084F868311288002A7FF464A9114A124BE4
:10C348001178186881F00101F4F7E1FCFFF760B992
:10C35800C84F00200AD7233CD7A368416F12033B7C
:10C3680000004843A4707D3F00C0F94400C0F9C4F0
:10C378000000C842CC4A00207E770020144C0020E0
:10C38800C8750020CA750020CC75002094ED577A36
:10C39800B1F90000D4ED586AB1F902E0E24AF4EECE
:10C3A800C76A80EAE0738EEAEE71A3EBE073F1EE00
:10C3B80010FAA1EBEE71B8BFF0EE476A8B42B8BF36
:10C3C8000B4607EE103A1378B8EEC77A27EE097ACB
:10C3D800002B40F0B880D54B93ED006AB4EEEA6AC2
:10C3E800F1EE10FA41F14C80F7EE005A75EEC65A9C
:10C3F8003BEEC77A65EE8B5ACD4BA7EE256A93EDD7
:10C40800007A26EE076AB5EEC06AF1EE10FA40F23D
:10C418007085CAEE065AB7EE007AB0EE476AA6EE05
:10C42800E56AF0EE466AF4EEC76AF1EE10FA88BFE4
:10C43800F0EE476AF5EEC06AF1EE10FAB8BFF0EE1A
:10C448004C6ABC4B93ED007A67EE877AA7EEA68A12
:10C45800FEF72EBF0122FEF787BEB74BB74A2B4423
:10C4680093ED007AD2ED007AB54B67EE277AF7EEB6
:10C47800006AF4EEE67AF1EE10FA93ED007A88BFDE
:10C48800F0EE667A67EE877A27EE888AFFF77CB83F
:10C49800AC4BDFF8EC921A78D5075CBFB9F81820D6
:10C4A800A4F88C21A84AA94D1288D5ED037A07EE85
:10C4B800102AB8EEC77AF4EEC77AF1EE10FA41F214
:10C4C800C587A34D2B8807EE103AB8EEC77AF4EE6D
:10C4D800C77AF1EE10FAC1F277809E4A9E4D92ED2E
:10C4E800006AD5ED006A94F99821C4ED646A76EE85
:10C4F800665A012AC4ED626AC4ED615A84ED656A20
:10C5080001F0EE85079BC4F89C31002537EEC77A09
:10C51800FCEEE77A914E84ED687A17EE902AA4F83B
:10C528008C21012296ED005A84F898218C4A954274
:10C5380041F279878B4BD3ED007AD3ED013AD3EDF5
:10C54800024AFFF7C9B87A4B93ED005AB5EEC05AC4
:10C55800F1EE10FA40F3CD84834BD3ED004AF5EEAB
:10C56800C04AF1EE10FA40F3C48434EEC77A66EE9E
:10C57800CA5A87EE246AC5EE856AB7EE007AB4EE29
:10C58800C76AF1EE10FA88BFB0EE476AB5EEC06A26
:10C59800F1EE10FA76EE876AB8BFB0EE4C6A66EE36
:10C5A800266A40E7714AD2ED007AB0EEC87AB4EE56
:10C5B800E77AF1EE10FA7FF72BA86D4AD2ED007AF0
:10C5C800B0EEED7AB4EEE77AF1EE10FA7FF720A834
:10C5D800684AD9ED007A92ED007AF0EEE77AF4EE47
:10C5E800C77AF1EE10FA7FF513A801220799C4F86B
:10C5F8006C1184F86821FEF7EEBF07EE102A19784F
:10C60800DFF88081C4F80C71B8EEC77AF7EE006ADB
:10C61800132986EE879AB8F90400B4F810619BEDE7
:10C62800070A01F0E984544A544992ED001AD2ED00
:10C63800053A92ED122A92ED173AD2ED091AD2ED87
:10C648000E4A92ED016A92ED064A92ED0A7AD2ED0F
:10C658000F5AD2ED132AD2ED186A92ED045AD2ED90
:10C66800030A67EE897A69EE288A29EE088AE1EEDC
:10C67800273A01EB86070025A2EE283AC4F80051B4
:10C68800C4F80451E1EE884AA6EE274AE7EE085AB4
:10C6980092ED167A92ED0D6A92ED021AD2ED0C1A0D
:10C6A800C7ED003AE2EEA86A25EE635A27EE437A10
:10C6B80092ED0B2AD2ED152AC7ED204AA0EEE34AE7
:10C6C80026EE646AD2ED143A82ED054AA1EE275AA5
:10C6D800F0EE477AE1EEE45AA2EE086AE2EEC36AA7
:10C6E800E3EEA87A82ED065AC2ED0E5A82ED0F6A81
:10C6F80087ED403AC2ED176AC2ED187AC4F80851BE
:10C70800721C02F01F02A4F81021A8F80400059B6F
:10C71800FEF729BCA4F8E071002A3FF4EDAD0B4DFB
:10C728004FF0020E82E400BFA0380020A838002095
:10C738009C38002098380020C4250020903800201C
:10C748008C3800204D76002078390020984D002044
:10C758007A390020F45F00206439002080390020F5
:10C768008FD0030078470020A4380020D03800205C
:10C77800CC380020D438002040460020D443002084
:10C788001C5D0020144C0020BC4A1178D4F81871A4
:10C79800BB4B9FEDBC7AFE009A1982ED007A002906
:10C7A80079D0B948B0EE476AF0EE476A0022F0EC5B
:10C7B800017A013267EEA77A05EE902AB4EEE77A9D
:10C7C800F1EE10FAF8EEE55AB8BFB0EE677A8A4291
:10C7D80076EEA76AA7EEA56AE9D1F5EEC06A9A19BE
:10C7E800F1EE10FA82ED007A55DDC6EE265AA74A18
:10C7F800A7490988F7EE007A75EEE75AD2ED007A74
:10C8080065EEA77AFDEEE77A17EE902A812A42F3C1
:10C8180053808A42A8BF0A4607EE902AF8EEE77AC4
:10C828009C4AF01902EB800292ED057AD2ED003AAB
:10C8380092ED066A92ED014AD2ED046AD2ED034AFE
:10C8480092ED025AA3EEA77AA4EE276A66EEC76AAB
:10C85800A7EE646ABDEEC77AE5EE276A17EE100AFE
:10C86800812882ED056AC2ED066A42F32280814280
:10C87800A8BF014607EE901AF8EEE77AFCEEE77AD1
:10C88800CDED087ABDF8202099198A801FB9BEF12C
:10C89800130F02F0E786BEF1150F41F0ED801E443C
:10C8A800DFF81082B28828F81720D4F814517A4A91
:10C8B800013582FB05325119EA17C2EBA102C2EB1E
:10C8C800C202AD1AC4F814517448D4F81C11079B5D
:10C8D800734D02682D78C4F81C31591A0A44026055
:10C8E800002D64D107EE901A6E4EDFF8E0916E4F7E
:10C8F800B8EEE78A06F5F07506F51378F6EC017AD6
:10C908009BED070ADBF80832F8EEE77A284627EEAF
:10C91800800A9847A5F1E000DBF828319847A5F18F
:10C928007000DBF898319847D6F8EC00DBF8AC30AB
:10C938009847D7ED007AA9EC010AE0EE087A243589
:10C94800A845E7EC017AD9D1059B1D78FEF749BDCA
:10C95800564B574A19681288564BC96919805A802C
:10C9680017B0BDEC0E8BBDE8F08F534B534E1A78C1
:10C9780012F0010F327840F03983002A00F03E852A
:10C9880092004F494F48DFF848A1DFF8489125F059
:10C998008FFAFFF743BAB4F8E071013F3FB2002FB6
:10C9A800A4F8E0717FF7B8AE474DFFF705BB07EE77
:10C9B800901A3C4D454BDFF8FC80DFF8EC9006946C
:10C9C800F8EEE78A05F5B8760027CDF824801C46EE
:10C9D800059BDBED077A1B78172B00F0A08195EDFE
:10C9E800007AB8EEC78A082B28EE278A07D1B0EE5E
:10C9F800480A089325F030FC089BA8F80000DAF8EC
:10CA0800002092000BD5002F03F01381B0EE480AE6
:10CA1800DBF8083206F170009847B0EE408AB0EEB5
:10CA2800480ADBF82831A6F170009847DBF89831FE
:10CA380030469847059B1B78032BB0EE408A00F0E0
:10CA48007A81D5F8F000DBF8AC30B0EE480A9847A8
:10CA5800D9ED007AA4EC010AE0EE287A0137032F19
:10CA680006F1240608F1020805F10405E9EC017A4B
:10CA7800AED1059B069C1D78FEF7B3BCB6430020DB
:10CA8800AC4600200000000068240020B8430020C5
:10CA9800B4430020D44500209324499268370020ED
:10CAA800AC430020D06C00206C370020587900205F
:10CAB80038560020144C00204D760020F14B002001
:10CAC80010590020CC470020984D0020206F0020EE
:10CAD8002C6F00201C5D0020002F00F09186B8F11B
:10CAE800000F42F0A982089BCD4D002B42F0F68042
:10CAF80095ED006A9DED0E5ACA4825EE866AFDEE50
:10CB0800E44AA5EE076AB0EE675AA6EE265A14EE76
:10CB1800901ABDEEC56A16EE10EA16EE107AE645D2
:10CB2800A8BF67467145C8BF0F4606EE107AB8EE33
:10CB3800C66A012A80ED006A00F0DF8095ED046A7C
:10CB48009DED0F5A25EE866AA5EE076AB0EE675A84
:10CB5800A6EE265ABDEEC56A16EE10EA16EE107A53
:10CB6800E645A8BF67468E45B8BF0F4606EE107A61
:10CB7800B8EEC66A022A80ED016A00F0BE8095ED23
:10CB8800086A9DED105A25EE866AA5EE076AB0EE92
:10CB9800675AA6EE265ABDEEC56A16EE10EA16EEDC
:10CBA800107AE645A8BF67468E45B8BF0F4606EE21
:10CBB800107AB8EEC66A032A80ED026A00F09D80FA
:10CBC80095ED0C6A9DED115A25EE866AA5EE076A69
:10CBD800B0EE675AA6EE265ABDEEC56A16EE10EA02
:10CBE80016EE107AE645A8BF67468E45B8BF0F46D1
:10CBF80006EE107AB8EEC66A042A80ED036A7CD085
:10CC080095ED106A9DED125A25EE866AA5EE076A23
:10CC1800B0EE675AA6EE265ABDEEC56A16EE10EAC1
:10CC280016EE107AE645A8BF67468E45B8BF0F4690
:10CC380006EE107AB8EEC66A052A80ED046A5CD062
:10CC480095ED146A9DED135A25EE866AA5EE076ADE
:10CC5800B0EE675AA6EE265ABDEEC56A16EE10EA81
:10CC680016EE107AE645A8BF67468E45B8BF0F4650
:10CC780006EE107AB8EEC66A062A80ED056A3CD040
:10CC880095ED186A9DED145A25EE866AA5EE076A99
:10CC9800B0EE675AA6EE265ABDEEC56A16EE10EA41
:10CCA80016EE107AE645A8BF67468E45B8BF0F4610
:10CCB80006EE107AB8EEC66A072A80ED066A1CD01E
:10CCC80095ED1C6A9DED155A65EE865AE7EE055AF4
:10CCD800E6EEA57AFDEEE77A17EE905AAC45A8BFC6
:10CCE800AC46A942D8BF614607EE901AF8EEE77A3B
:10CCF800C0ED077A002A3FF491A892004A494948B2
:10CD080025F0D6F8494A1268002A3FF48CA81BF08F
:10CD1800ABF9FFF788B8F0EE676AFFF7A7B995EDAA
:10CD2800007A0BEB4702B8EEC78A128FA8F80020EA
:10CD380028EE278A63E625F08FFAA8F8000080E637
:10CD4800B0EE465AFEF7FFBC39493A4BD1F8EC1021
:10CD58001B6844F620608142A8BF0146B1F57A7F7E
:10CD6800B8BF4FF47A7189B213F0100FA4F8B2115A
:10CD7800DAF8003000F02384DB0441F1A1852E4B62
:10CD8800D3F800E0BEF832707F082C4D2C48D4F858
:10CD9800B431D5ED037AA0FB01018809642191FB28
:10CDA800F0F11429BDEEE77A04EB4305A8BF14217E
:10CDB80001338B42C4F8B43117EE10CAA4BF002364
:10CDC800C4F8B43104EB4303A5F8B8C1B3F9B831DA
:10CDD80007EE103AB8EEC77A77EEC77AFDEEE77A33
:10CDE800CDED067ABDF9181081EAE173A3EBE17382
:10CDF800BB4201F32D8713494FF07E530B60FFF7B9
:10CE08005BB8114B0593114C5EE5DBF80830002B3D
:10CE18003FF42AA80E49A1F14C009847FFF724B81F
:10CE2800E4380020CC47002010590020005D002085
:10CE3800341C0020EC5F0020C44F0020984D0020D7
:10CE4800D34D621004000020104C002068240020FC
:10CE5800F06C00201E21CE48F5F753F800283FF467
:10CE680048AACC4B1B8858063FF543AA94F80432CD
:10CE7800AB4242F01C82C84BD4ED827AD3ED016AF2
:10CE880094ED505ADFEDC55A9FEDC56A27EEC57A75
:10CE980068EE277AA8EE267AE5EE267AB4EEE57AE9
:10CEA800F1EE10FA88BFB0EE657AB4EEC67AF1EE0C
:10CEB80010FAF4EEE57AB8BFB0EE467AF1EE10FA61
:10CEC80088BFF0EE657AF4EEC67AF1EE10FAB8BFD4
:10CED800F0EE467A84ED4E7AC4ED507AFFF709BA3F
:10CEE800FDEEC87AAF4A17EE903A9780D380FFF7E5
:10CEF800FBB9DFEDAD6AFFF7A4BADAF80010490212
:10CF08003EF530AEFEF732BE9FEDA47ADFEDA46A9F
:10CF1800A449F4EEC77AF1EE10FA98BFB0EE677A3A
:10CF2800FDEEE77AB4EEE67AF1EE10FA17EE903AF3
:10CF3800B8BFB0EE667ABEF1010F84ED4F7A4B8030
:10CF48003FF758A9FFF7D0B9B4EEC87AF1EE10FA56
:10CF580098BFB0EE478ABDEEC77AB4EEE68ADFF82E
:10CF680044C2F1EE10FA17EE103AB8BFB0EE668A76
:10CF780084ED4E8AACF80030BEF1000F7FF4D4A8DF
:10CF8800FFF7B2B9BDEEE77A864B17EE102A9A8002
:10CF9800FFF793B9002B3EF43BABFEF718BBF8F74D
:10CFA800DDF9059B7F491A78069B072AA0EB030049
:10CFB80088807EF453AFF8F7D1F90646FEF74FBFE5
:10CFC800F8F7CCF9059BDFF8DC811A780A9B012A6F
:10CFD800A0EB0300A8F8020000F0D482072A7EF430
:10CFE8003FABF8F7BBF90690FEF73CBB002A00F010
:10CFF8000582D4ED583A94ED574AD4ED627A6B49DC
:10D0080094ED617A91ED005AD4ED555A94ED546A35
:10D01800674D6848F4EEC43AF3EE046AF1EE10FA8C
:10D0280077EEA64A00F11E8395ED026A26EE656A40
:10D03800B0EE674AA6EE074AB4EEE44A34EE666AF2
:10D04800F1EE10FA48BFB0EE456A012A80ED006A99
:10D0580000F0D48195ED066A26EE656AB0EE674A5F
:10D06800A6EE074AB4EEE44A34EE666AF1EE10FA28
:10D0780048BFB0EE456A022A80ED016A00F0BE8121
:10D0880095ED0A6A26EE656AB0EE674AA6EE074A8B
:10D09800B4EEE44A34EE666AF1EE10FA48BFB0EE38
:10D0A800456A032A80ED026A00F0A88195ED0E6AB0
:10D0B80026EE656AB0EE674AA6EE074AB4EEE44A81
:10D0C80034EE666AF1EE10FA48BFB0EE456A042AFB
:10D0D80080ED036A00F0928195ED126A26EE656A8A
:10D0E800B0EE674AA6EE074AB4EEE44A34EE666A42
:10D0F800F1EE10FA48BFB0EE456A052A80ED046AE1
:10D1080000F07C8195ED166A26EE656AB0EE674AF6
:10D11800A6EE074AB4EEE44A74EE666AF1EE10FA37
:10D1280048BFF0EE456A062AC0ED056A00F0668140
:10D13800D5ED1A6A66EEE56AB0EE674AA6EE874A4A
:10D14800B3EE046AB4EEE44A74EE466AF1EE10FAFD
:10D1580048BFF0EE456A072AC0ED066A00F04E8126
:10D16800D5ED1E6ADFF850A0DFF8509066EEE55A5C
:10D17800E5EE877AF4EEE74A77EEC67AF1EE10FA32
:10D18800C8BFF0EE457AC0ED077AFEF747BE00BF8C
:10D19800EC5F0020C04F00200400002000C0F944CC
:10D1A80000C0F9C4144C002000000000E038002042
:10D1B800E4380020CC4700202C6F00201C5D0020A4
:10D1C800B8F1000F41F00282DB4D9DED0E5A95ED4E
:10D1D800006ADA4825EE866AA5EE076AB0EE675A55
:10D1E800A6EE265ABDEEC56A16EE10EA16EE107ABD
:10D1F800E645A8BF67467145C8BF0F4606EE107AD8
:10D20800B8EEC66A012A80ED006A3FF476AD95ED66
:10D21800046A9DED0F5A25EE866AA5EE076AB0EE00
:10D22800675AA6EE265ABDEEC56A16EE10EA16EE45
:10D23800107AE645A8BF67467145C8BF0F4606EE97
:10D24800107AB8EEC66A022A80ED016A3FF455AD3D
:10D2580095ED086A9DED105A25EE866AA5EE076AD7
:10D26800B0EE675AA6EE265ABDEEC56A16EE10EA6B
:10D2780016EE107AE645A8BF67467145C8BF0F4647
:10D2880006EE107AB8EEC66A032A80ED026A3FF409
:10D2980034AD95ED0C6A9DED115A25EE866AA5EE22
:10D2A800076AB0EE675AA6EE265ABDEEC56A16EEB4
:10D2B80010EA16EE107AE645A8BF67467145C8BF62
:10D2C8000F4606EE107AB8EEC66A042A80ED036AA5
:10D2D8003FF413AD95ED106A9DED125A25EE866A5E
:10D2E800A5EE076AB0EE675AA6EE265ABDEEC56AE5
:10D2F80016EE10EA16EE107AE645A8BF67467145A5
:10D30800C8BF0F4606EE107AB8EEC66A052A80ED49
:10D31800046A3FF4F2AC95ED146A9DED135A25EEBC
:10D32800866AA5EE076AB0EE675AA6EE265ABDEEE3
:10D33800C56A16EE10EA16EE107AE645A8BF6746EB
:10D348007145C8BF0F4606EE107AB8EEC66A062ABF
:10D3580080ED056A3FF4D1AC95ED186A9DED145A3D
:10D3680025EE866AA5EE076AB0EE675AA6EE265A3B
:10D37800BDEEC56A16EE10EA16EE107AE645A8BFAD
:10D3880067467145C8BF0F4606EE107AB8EEC66A02
:10D39800072A80ED066A3FF4B0AC95ED1C6A9DED56
:10D3A800155A65EE865AE7EE055AE6EEA57AFDEEC1
:10D3B800E77A17EE905AAC45A8BFAC46A942C8BF59
:10D3C8008C4607EE90CAF8EEE77AC0ED077A91E44A
:10D3D800DFED5B6AFEF76CBFB5EEC07AF1EE10FACE
:10D3E80001F15A82B7EE006A36EE477AC6EE076A4E
:10D3F800FEF7E4BEDFED526AFEF779BEDFF878A1EA
:10D40800DFF87891FEF70ABD4E494A79002A3EF4C2
:10D418002BAA4D4A1278002A3EF426AA0B784B49CB
:10D42800DFED4B4A07EE903A0B88B8EE677A07EEC5
:10D43800902A06EE903AF8EEE77AF8EE666A67EE1A
:10D44800277AB7EE007A87EEA63AB4EEE43AF1EE20
:10D4580010FA88BFB0EE643AB4EEC73AF1EE10FAAB
:10D46800B8BFB0EE473AFEF701BA3A4B5988FEF713
:10D4780036BDB4F8B21101F57A7189B2FEF72FBD45
:10D48800354B93ED006AFEF7BEBF344F3B78013B46
:10D498000D2B24D8DFE813F0F506BB07E606CB060C
:10D4A80023002300A4078F0734070E0067075B07D4
:10D4B800860702072A4B1B78002B02F0F5801A20FA
:10D4C8000AF0FCF8002842F0EF80264B1B78002B6E
:10D4D80042F0EA8009233B701DF096FAAA78012AE7
:10D4E80000F063852B79012B01F05985022B7EF41E
:10D4F8000BAF3B78012B7EF407AF1A4B1B78002B40
:10D508007EF402AF1CF034FFFEF7FEBE164B9FED13
:10D51800177AD3ED087AF4EEC77AF1EE10FA00F232
:10D52800F9849FED137A134DD5ED037A77EE877A58
:10D53800C5ED037AFEF7BBBCE4380020CC470020D9
:10D548000000C842544F0020964D0020304D002066
:10D55800713DAA3F0C4B00209C380020623C002003
:10D568000E480020595E0020403700208FC2753CCD
:10D5780000000000984D00202C6F00201C5D00204A
:10D58800DFF87082F7F7EAFE9049D4F87C21096841
:10D598000690821A511AC4F87C01A8F80420A8F849
:10D5A8000610FEF75FB8F7F7D9FE0A90FDF7E3BD5E
:10D5B800874B9B7B002B3EF46DACFEF770BCDD0007
:10D5C8003FF5DAABFEF778BCB4F88C51954240F2DF
:10D5D800028594F8A451002D40F06E877D4A7E4E56
:10D5E80092ED007AD6ED007A94F99821C4ED647A28
:10D5F80077EE676A012AC4ED627AC4ED616A84ED48
:10D60800657A02F03D80079BC4F89C31734A9FED10
:10D61800747A92ED005A84ED687A012284F8982190
:10D62800FEF784BF6F4B1B88002B40F0E8856E4ADD
:10D638006E4B11781868F3F76AFBD4F86C21079BD6
:10D648009A1AFDF74EBE6A4BD9ED007A93ED007A2F
:10D65800F0EEE77AF4EEC77AF1EE10FA7DF7D8AF7C
:10D66800FDF7C8BFD5ED015A65EEC65AB0EE674A58
:10D67800A5EE874AB4EEE44A74EE665AF1EE10FA63
:10D6880048BFF0EE455A012AC0ED005A3FF4B6AE45
:10D69800D5ED055A65EEC65AB0EE674AA5EE874A3B
:10D6A800B4EEE44A74EE665AF1EE10FA48BFF0EEB2
:10D6B800455A022AC0ED015A3FF4A0AED5ED095AE9
:10D6C80065EEC65AB0EE674AA5EE874AB4EEE44A5C
:10D6D80074EE665AF1EE10FA48BFF0EE455A032A86
:10D6E800C0ED025A3FF48AAED5ED0D5A65EEC65A22
:10D6F800B0EE674AA5EE874AB4EEE44A74EE665A7D
:10D70800F1EE10FA48BFF0EE455A042AC0ED035A6C
:10D718003FF474AED5ED115A65EEC65AB0EE674ABD
:10D72800A5EE874AB4EEE44A74EE665AF1EE10FAB2
:10D7380048BFF0EE455A052AC0ED045A3FF45EAEE4
:10D74800D5ED155A65EEC65AB0EE674AA5EE874A7A
:10D75800B4EEE44A74EE666AF1EE10FA48BFF0EEF1
:10D76800456A062AC0ED056A3FF448AED5ED196A48
:10D7780066EEC66AB0EE674AA6EE874AF3EE045A2A
:10D78800B4EEE44A74EE656AF1EE10FA48BFF0EEC2
:10D79800456A072AC0ED066A3FF430AED5ED1D6A2A
:10D7A800DFF854A0DFF8549026EEC66AE6EE077A52
:10D7B800F4EEE47A77EEE57AF1EE10FAB8BFF0EE1F
:10D7C800457AC0ED077AFEF729BB00BFF047002075
:10D7D800886A0020F45F0020643900208039002026
:10D7E80000000000C8750020CA750020CC75002014
:10D7F800D4380020144C00202C6F00201C5D002021
:10D80800089BD94D002B41F08D8095ED006A9DED68
:10D818000E5AD64825EE866AFDEEE44AA5EE076A5A
:10D82800B0EE675AA6EE265A14EE901ABDEEC56AF7
:10D8380016EE10EA16EE107AE645A8BF674671455F
:10D84800C8BF0F4606EE107AB8EEC66A012A80ED08
:10D85800006A3EF4DFAA95ED046A9DED0F5A25EEA5
:10D86800866AA5EE076AB0EE675AA6EE265ABDEE9E
:10D87800C56A16EE10EA16EE107AE645A8BF6746A6
:10D888008E45B8BF0F4606EE107AB8EEC66A022A71
:10D8980080ED016A3EF4BEAA95ED086A9DED105A26
:10D8A80025EE866AA5EE076AB0EE675AA6EE265AF6
:10D8B800BDEEC56A16EE10EA16EE107AE645A8BF68
:10D8C80067468E45B8BF0F4606EE107AB8EEC66AB0
:10D8D800032A80ED026A3EF49DAA95ED0C6A9DED3F
:10D8E800115A25EE866AA5EE076AB0EE675AA6EECB
:10D8F800265ABDEEC56A16EE10EA16EE107AE6450F
:10D90800A8BF67468E45B8BF0F4606EE107AB8EE38
:10D91800C66A042A80ED036A3EF47CAA95ED106A73
:10D928009DED125A25EE866AA5EE076AB0EE675A93
:10D93800A6EE265ABDEEC56A16EE10EA16EE107A65
:10D94800E645A8BF67468E45B8BF0F4606EE107A73
:10D95800B8EEC66A052A80ED046A3EF45BAA95ED26
:10D96800146A9DED135A25EE866AA5EE076AB0EE95
:10D97800675AA6EE265ABDEEC56A16EE10EA16EEEE
:10D98800107AE645A8BF67468E45B8BF0F4606EE33
:10D99800107AB8EEC66A062A80ED056A3EF43AAAFD
:10D9A80095ED186A9DED145A25EE866AA5EE076A6C
:10D9B800B0EE675AA6EE265ABDEEC56A16EE10EA14
:10D9C80016EE107AE645A8BF67468E45B8BF0F46E3
:10D9D800FEF7FEB9664ED4ED017A94ED006A3188FF
:10D9E800726977EEA77AF0EE006AB0EE677AA6EE73
:10D9F800267A4E1E04EBC601D6EE267A0839103276
:10DA0800F6EE003A27EE237A67EEA37A84ED207AC1
:10DA1800C4ED217A574C274604F1800091ED027A33
:10DA280091ED036AD7ED036AD7ED027A52ED014A08
:10DA380012ED025A37EE674A76EEC65A77EE277A23
:10DA4800E4EE845A013EA1F10801E5EE047A07F1FB
:10DA5800080702F1080236EE267A00F10800E4EE23
:10DA6800877AE5EE475A67EEA37A25EEA37AC0EDEA
:10DA7800007A80ED017AD1D1BEF1140F7EF417AF90
:10DA8800F7F76CFC069BDFF80081C01AA8F80200C3
:10DA9800D4F81451FEF70BBFD4F81831B4F810C1FC
:10DAA800354ACCF120095FFA89F90CEB431702EBF0
:10DAB80087075FEA990201F0F285013216012F48C3
:10DAC8002F4907EB060807F1100212ED024A12ED82
:10DAD800035A12ED016A12ED047A50ED024A50ED34
:10DAE800035A50ED016A50ED047A64EE244A65EE5B
:10DAF800255A66EE266A67EE277A1032904541ED80
:10DB0800024A41ED035A41ED016A41ED047A00F100
:10DB1800100001F11001D8D11A48A6F110010F44E4
:10DB280000EB0108214419F0030209D0B7EC017A8F
:10DB3800F8EC017A67EE277A013AE1EC017AF5D13F
:10DB4800BCF1000F41F03180BEF1140F7EF4AFAE8E
:10DB5800F7F704FC069BDFF83080D4F81451C01A9C
:10DB6800A8F80200FEF7A3BEE4380020CC47002046
:10DB7800BC43002068240020D443002064450020D2
:10DB88007824002054450020144C0020D04E3188C1
:10DB980073684FEA51094FEA89005FEAD10C04EB38
:10DBA800000204EB810500F0A18000F110010CF1E6
:10DBB800010CC84F02EB0C1C2944103203F1100E63
:10DBC80005F1100050ED032A50ED043A17ED043A20
:10DBD80017ED032A50ED026A10ED016A17ED021ADB
:10DBE80057ED010A11ED044A11ED035A52ED044AAA
:10DBF80052ED035A12ED027A52ED017A51ED021AF2
:10DC080011ED010A73EE238A32EE228A47ED048A67
:10DC180007ED038A71EE268A30EE868A47ED028A7E
:10DC280007ED018A74EE848A35EE858A42ED048A0E
:10DC380002ED038A77EE218A37EE808A42ED028A66
:10DC480002ED018A73EE633A75EE655A1EED035ACA
:10DC580032EE623A74EE644A25EE638A1EED044A97
:10DC680023EE052A64EE652AA3EE048A1032944551
:10DC780024EE843AA3EE842A07F110070EF1100E61
:10DC8800A5EE853A00F1100001F11001E4EE852AB5
:10DC980000ED078A00ED082A01ED073A41ED082A50
:10DCA8005EED055A1EED065A71EE666A30EEC66ADA
:10DCB80031EEC77A70EE677A26EE253A65EEE63AD7
:10DCC80025EE674A67EE054AE6EE053AA6EE853A7E
:10DCD800A7EE254AE7EEA54A00ED063A40ED053ADB
:10DCE80001ED064A41ED054A7FF46CAF1FFA89F948
:10DCF8001A46494678481BF049F972684946284649
:10DD08001BF044F9059B1A78142A7FF4C1AEB7E6D4
:10DD1800D4F8185171497248724BEA0011441544FD
:10DD28008A88196800EE102A643AC82AA8BFC8224F
:10DD3800782AB8BF782207EE902AB8EEC07AF8EEB3
:10DD4800E77A00EB850577EE670A77EE876A67EE74
:10DD5800877A20EEA67AB8EE400AC7EE870A2846E8
:10DD6800D5F81490D5F81880EF692E6A1BF048FD95
:10DD7800059BC5F8149093F800E0C5F81880BEF12B
:10DD8800140FEF612E6201F0A484D4F81821564BC9
:10DD9800D4F81451013283FB0213A3EBE27303EBB3
:10DDA8004303D31A0135C4F81831C4F8145175E681
:10DDB800474E4948B268B18923F022F9059B93F888
:10DDC80000E0BEF1140F01F09184D4F8145101352C
:10DDD800C4F81451FFE5454E31785FEA910C01F023
:10DDE800AC85434F0CF101094FEA491907EB0908C3
:10DDF80007F12002A7F1700012ED076A52ED056ADB
:10DE080012ED037A52ED017A52ED025A12ED084AE8
:10DE180052ED064A12ED045A26EE066A66EEA66A26
:10DE280027EE077A67EEA77AA4EE046A20329045B7
:10DE3800E4EEA46A00F11000A5EE057AE5EEA57AF5
:10DE4800F1EEC65AB1EEE66AF1EEC76AB1EEE77ACC
:10DE580040ED085A00ED076A40ED066A00ED057AC4
:10DE6800CAD1A9F120023A4404EB0C1711F00300BF
:10DE780018BF08320FD052ED017A12ED027A67EE20
:10DE8800A77A0138E7EE077A02F10802B1EEE77ADD
:10DE9800A7EC017AEFD1BEF1140F01F00A84013525
:10DEA800C4F81451FEF772BCF7F758FA059B0690B0
:10DEB80093F800E0BEF1140F05BFDFF83880D4F8FE
:10DEC8001451D4F81451A8F80050FDF756B800BF03
:10DED800BC4300207824002068240020AC460020A1
:10DEE800B06E00201C6F002056555555B6430020D3
:10DEF800E8240020144C0020306E99BC2716983D69
:10DF0800A40DC93F843459BEDB0F4940D06D393A5E
:10DF180000000000F0EEE76AB7EE005A35EE665AE8
:10DF28001FED0B4A5FED0B5A1FED0A6A1FED0C7AC5
:10DF380094ED6B0AF1EEC54AE6EE845AF5EEC07A26
:10DF4800A6EEA56AF1EE10FAA6EE867A48BF5FED56
:10DF5800127A27EE247A48BF37EEC77A27EE000AEE
:10DF680024F07AF9B0F5617F00F38D8607EE900A08
:10DF7800F8EEE76A5FED1B7A66EEA76A07EE905A3D
:10DF8800BDEEE67AF8EEE77A17EE103A2033402B2A
:10DF980041F281841FED220A24F05EF900B207EEF7
:10DFA800900AB8EEE77AFFF7BEBAC249C24B896851
:10DFB8001B6899423FF696AA3B780C3B022B7EF6EB
:10DFC800A3A9BE4C3A702378002B3EF49DA90023E8
:10DFD8002370FEF799B9BA4A02F1500503E00432FA
:10DFE800954200F069821378262BF8D19678D37879
:10DFF8009E42F4D2FFF7EDBAB24DB34F95ED004A09
:10E0080095ED057AD5ED014A95ED066AD5ED046AD8
:10E0180095ED035AD5ED025A67EE897A07EB860229
:10E02800A4EE277AA4EEA76A66EEC76AA5EE476A49
:10E03800E5EEA76A20EE070A85ED056AC5ED066AD2
:10E0480082ED007A29EE088A24F006F969EE288A1A
:10E05800D5ED0E5AD5ED176A95ED091AD5ED121AB8
:10E0680095ED0F5A95ED187A95ED0A2AD5ED132AF4
:10E0780095ED0D6AD5ED167A95ED0C3AD5ED0B3A7E
:10E0880095ED154AD5ED144AE1EE085A002207EB42
:10E098008601E8EEA16A00B2C4F80021A2EE085A8F
:10E0A800C4F80421C4F80821A8EEA27A26EE656A0D
:10E0B80067EEE67AA3EE655AA3EE886AA6EEC47AFE
:10E0C800E8EEA47A85ED0E5AC1ED205A85ED0F6A67
:10E0D800C1ED406A85ED177AC5ED187AFEF710BBD9
:10E0E800D4F89C51079B5D1BFEF710BABBF938208A
:10E0F800CBF8201007EE902A0121F8EEE77ACBF84A
:10E108006020CBF87C100022012FCBED1C7ACBEDE0
:10E118001B7ACBF8742001F09D82B7427CF491AF52
:10E12800BBF93A20CBF8642007EE902A002101229F
:10E13800F8EEE77ACBF82410CBF890200022012FD4
:10E14800CBED217ACBED207ACBF8882001F08682BE
:10E15800B7427CF4AAAFBBF93C20CBF8682007EEA5
:10E16800902A00210122F8EEE77ACBF82810CBF8A4
:10E17800A4200022012FCBED267ACBED257ACBF80F
:10E188009C207CF4C6AF9FED518A032D49D04CB139
:10E1980007EE904AF8EEE77AF4EEC87AF1EE10FA54
:10E1A80001F1D0834A4A4B4C1168DBF86820A8F883
:10E1B800060094F8200102EB560292FBF6F60022C4
:10E1C800CBF828608A620A63CA6228B1424A126898
:10E1D80032F480637CF4A0AF404A126812F4003233
:10E1E80041F030823E481146835C012B02F10C025B
:10E1F80000F0778301311829F6D1FCF78DBF394932
:10E208004B69002B3DF46DA83748384B008893FBC9
:10E21800F0F00B684FF0010E186081F811E0FDF77F
:10E2280060B8B0EE480A24F017F800B2AFE71BF068
:10E23800AFFE2F4A0292A2F10C032621019300910E
:10E24800A2F10A035021163A492010F019FFA8B983
:10E25800284BAA7818604FF0FF31596007233B70AC
:10E26800FFF73DB9DFF88C801BF092FE224AD8F800
:10E278000430126864339342C1F07C83AA78FFF7B4
:10E288002EB91E4B1B78D90701F16A831F2009F0AC
:10E2980015FA0028F2D00C233B70EFE71F200692F6
:10E2A80009F00CFA069A00287FF419A901233B709B
:10E2B800FFF715B94C1A0020F4470020595E0020DA
:10E2C8009440002040460020D44300200000000075
:10E2D8005879002068240020BC4F0020E85700200F
:10E2E8009C540308D0750020E875002020A1070081
:10E2F80032390308F85F0020F07500204D760020C1
:10E308001A2009F0DBF900283FF4E6A89B4B1B888C
:10E31800002B7FF4E1A89A4B4520D3F800801BF02E
:10E32800FBFE0E201BF0F8FE40461BF0EBFFDDF86D
:10E338001C8040461BF0E6FF924A934B12681A6015
:10E3480040460A233B701CF087F8FFF7C5B8012A3E
:10E3580001D1F3F7CDFF0D2313203B7005F00AFD23
:10E36800AA78FFF7BCB8894B89495B680968C83344
:10E378008B4205D31BF034FEAA7800283FF4AFA8DF
:10E38800032A93D1DFF84082D8F8000005F02CF872
:10E39800804B1B780022022BC8F8002001F0118462
:10E3A800AA7883E7012A01F0D4820E2313203B7058
:10E3B80005F0E0FC62E71BF0EBFD1CF05BFB0028BE
:10E3C8003FF45CAF1BF00CFE00283FF457AF6D4ADA
:10E3D8006D4B12681A600A233B70AA78FFF77FB862
:10E3E8001BF0D6FD6C4B002105208DE80300A3F13E
:10E3F80008020291532010F043FE00287FF43EAF3C
:10E40800624BAA78186008233B70FFF768B8604B26
:10E418005E491B684B60614800230B600321036061
:10E428003970FFF75CB8DFED5E7A5E4B94ED687A81
:10E43800C3ED007AC3ED017AC3ED027A5A4BF0EED0
:10E44800674AF0EE673A1968FDF746B9574A584DDA
:10E45800D2ED006A574A95ED006A1278C4ED646AF5
:10E4680084ED656A002A00F01F8276EE665A94F9F8
:10E478009821C4ED615A0132C4ED626A00F08985C1
:10E48800079BC4F89C31002537EE677AFCEEE77AE3
:10E49800494E84ED687A17EE902AA4F88C21FF2261
:10E4A80096ED005A84F89821FEF740B8434B1D7842
:10E4B80005F00108FDF7AEBC3C4A3D4DD2ED007AAF
:10E4C8003C4A95ED007A1278C4ED647A84ED657A59
:10E4D800002A00F0658377EE676A94F99821C4ED05
:10E4E800616A0132C4ED627A00F0DB86079BC4F8EA
:10E4F8009C3100259FED2A7A2F4E84ED687AFF2201
:10E5080096ED005A84F89821FEF710B82C49DFEDF3
:10E518002D7A0968C4ED4C7A11F080530A9340F0C3
:10E52800A683DAF8001011F480030A9300F0CF8173
:10E5380000230A93B6EE007A67EE877AF4EEE57A5E
:10E54800F1EE10FAC8BFF0EE675A40F39083C4EDBD
:10E55800685AFDF70BBB73EEE77AB7EE007AF4EE74
:10E56800C77AF1EE10FAC4ED4C7A41F38F8084EE4D
:10E57800A77A8DED0E7AFDF7EEBA00BF605E002037
:10E588005C5E0020705E0020685E0020F85F00205E
:10E59800F0750020EC470020EC3A03081C3D0020F1
:10E5A8000000000078470020C44F0020885E00204B
:10E5B80068390020507100207C3900204D760020F9
:10E5C800EC5F002000000080203D0020D14D0D9B15
:10E5D8009DED0E5A95ED006A002B00F01B8725EE85
:10E5E800866ACD48A5EE076AB0EE675AA6EE265AA7
:10E5F800BDEEC56A16EE10EA16EE107AE645A8BF1B
:10E6080067467145C8BF0F4606EE107AB8EEC66A6F
:10E61800012A80ED006A3DF401AC95ED046A9DED98
:10E628000F5A25EE866AA5EE076AB0EE675AA6EE7F
:10E63800265ABDEEC56A16EE10EA16EE107AE645C1
:10E64800A8BF67467145C8BF0F4606EE107AB8EEF8
:10E65800C66A022A80ED016A3DF4E0AB95ED086ACE
:10E668009DED105A25EE866AA5EE076AB0EE675A48
:10E67800A6EE265ABDEEC56A16EE10EA16EE107A18
:10E68800E645A8BF67467145C8BF0F4606EE107A33
:10E69800B8EEC66A032A80ED026A3DF4BFAB95ED79
:10E6A8000C6A9DED115A25EE866AA5EE076AB0EE52
:10E6B800675AA6EE265ABDEEC56A16EE10EA16EEA1
:10E6C800107AE645A8BF67467145C8BF0F4606EEF3
:10E6D800107AB8EEC66A042A80ED036A3DF49EAB50
:10E6E80095ED106A9DED125A25EE866AA5EE076A29
:10E6F800B0EE675AA6EE265ABDEEC56A16EE10EAC7
:10E7080016EE107AE645A8BF67467145C8BF0F46A2
:10E7180006EE107AB8EEC66A052A80ED046A3DF462
:10E728007DAB95ED146A9DED135A25EE866AA5EE2C
:10E73800076AB0EE675AA6EE265ABDEEC56A16EE0F
:10E7480010EA16EE107AE645A8BF67467145C8BFBD
:10E758000F4606EE107AB8EEC66A062A80ED056AFC
:10E768003DF45CAB95ED186A9DED145A25EE866A6A
:10E77800A5EE076AB0EE675AA6EE265ABDEEC56A40
:10E7880016EE10EA16EE107AE645A8BF6746714500
:10E79800C8BF0F4606EE107AB8EEC66A072A80EDA3
:10E7A800066A3DF43BAB95ED1C6A9DED155A65EE86
:10E7B800865AE5EE075AE6EEA57AFDEEE77A17EEF9
:10E7C800902A9445A8BF94468A42A8BF614607EE9E
:10E7D800901AF8EEE77AC0ED077AFDF71FBBBEF195
:10E7E800010F7FF7D0AC07EE103AB8EEC77AC7EE44
:10E7F800876AB1EEE68AC8E4BEF1010F40F32E87BE
:10E8080007EE103AB8EEC77AC7EE876AB1EEE68A25
:10E81800032D13D04CB107EE904AF8EEE77AF4EEE8
:10E82800C87AF1EE10FA01F18D80DBF8642002EB72
:10E83800560292FBF6F2CBF8242089E4B0EE480A9F
:10E8480023F00AFD00B2E5E7BEF1010F40F30287AD
:10E8580007EE103AB8EEC77AC7EE876AB1EEE68AD5
:10E86800032D13D04CB107EE904AF8EEE77AF4EE98
:10E87800C87AF1EE10FA01F16580DBF8602002EB4E
:10E88800560292FBF6F2CBF8202046E4B0EE480A96
:10E8980023F0E2FC00B2E5E7F7EE006AFDF78EBC74
:10E8A800F7EE006AFDF704BD76EEC65AF0EE466A4A
:10E8B800DDE58222FDF7E8BFDFED187AFDF7B0BF8E
:10E8C800174BD3F800E0BEF93270FEF75EBAB6EE29
:10E8D800007AF4EEC75AF1EE10FA3FF72BAEFDF7C7
:10E8E80045B9D4F824614A003EB1551800EB8505B6
:10E8F80076786D78B542BCF40FAC0A4400EB820020
:10E908000022C4F82401A4F81022C4F81422FCF749
:10E9180003BC00BFE4380020CC47002000000243BD
:10E92800C44F002095ED006A9DED0E4AE34825EEA0
:10E93800866AFDEEE43AA4EE076AB0EE674AA6EEF0
:10E94800264A13EE901AB4EEC45AF1EE10FAB0EE5D
:10E95800446A88BFB0EE646ABDEEC66A16EE10EA75
:10E9680016EE107AE645A8BF67467145C8BF0F4640
:10E9780006EE107AB8EEC66A012A80ED006A3DF408
:10E9880049AA95ED046A9DED0F4A25EE866AA4EE24
:10E99800076AB0EE674AA6EE264AB4EEC45AF1EE0C
:10E9A80010FAB0EE446A88BFB0EE646ABDEEC66A7B
:10E9B80016EE10EA16EE107AE645A8BF67468E45B1
:10E9C800B8BF0F4606EE107AB8EEC66A022A80ED86
:10E9D800016A3DF41FAA95ED086A9DED104A25EEDF
:10E9E800866AA4EE076AB0EE674AA6EE264AB4EE37
:10E9F800C45AF1EE10FAB0EE446A88BFB0EE646A09
:10EA0800BDEEC66A16EE10EA16EE107AE645A8BF05
:10EA180067468E45B8BF0F4606EE107AB8EEC66A4E
:10EA2800032A80ED026A3DF4F5A995ED0C6A9DED87
:10EA3800114A25EE866AA4EE076AB0EE674AA6EE8A
:10EA4800264AB4EEC45AF1EE10FAB0EE446A88BF12
:10EA5800B0EE646ABDEEC66A16EE10EA16EE107ADB
:10EA6800E645A8BF67468E45B8BF0F4606EE107A42
:10EA7800B8EEC66A042A80ED036A3DF4CBA995ED89
:10EA8800106A9DED124A25EE866AA4EE076AB0EE7A
:10EA9800674AA6EE264AB4EEC45AF1EE10FAB0EE72
:10EAA800446A88BFB0EE646ABDEEC66A16EE10EA24
:10EAB80016EE107AE645A8BF67468E45B8BF0F46E2
:10EAC80006EE107AB8EEC66A052A80ED046A3DF4AF
:10EAD800A1A995ED146A9DED134A25EE866AA4EE68
:10EAE800076AB0EE674AA6EE264AB4EEC45AF1EEBB
:10EAF80010FAB0EE446A88BFB0EE646ABDEEC66A2A
:10EB080016EE10EA16EE107AE645A8BF67468E455F
:10EB1800B8BF0F4606EE107AB8EEC66A062A80ED30
:10EB2800056A3DF477A995ED186A9DED144A25EE1E
:10EB3800866AA4EE076AB0EE674AA6EE264AB4EEE5
:10EB4800C45AF1EE10FAB0EE446A88BFB0EE646AB7
:10EB5800BDEEC66A16EE10EA16EE107AE645A8BFB4
:10EB680067468E45B8BF0F4606EE107AB8EEC66AFD
:10EB7800072A80ED066A3DF44DA995ED1C6A9DEDC6
:10EB8800154A65EE865AE7EE045AE6EEA57AB4EE23
:10EB9800E75AF1EE10FAC8BFF0EE647AFDF72AB929
:10EBA80077EEC76AF0EE477A97E4454A4FEA890755
:10EBB8005FEA9C09384402EBC313274437D009F1B4
:10EBC80001094FEA091903EB090803F1100200F1E2
:10EBD800100607F1100112ED024A12ED035A12ED68
:10EBE800016A12ED047A56ED024A56ED035A56EDC3
:10EBF800016A56ED047A64EE244A65EE255A66EEFB
:10EC0800266A67EE277A1032904541ED024A41EDB7
:10EC1800035A41ED016A41ED047A06F1100601F14B
:10EC28001001D8D1A9F110094B4448444F441CF0B5
:10EC3800030C3EF489AFB3EC017AF0EC017A67EE8D
:10EC4800277ABCF1010CE7EC017AF4D1FEF77CBF1E
:10EC5800BEF834309FED1B7A07EE903AF8EEE77A6B
:10EC6800194B67EE877AC3ED007AFDF725B9B7EE41
:10EC7800007A77EE677AF4EEE75AF1EE10FA88BF79
:10EC8800F0EE675A63E407EE905ADFED106AF8EE8B
:10EC9800E77A66EEA65A9FED0E5A9FED0E6A9FED33
:10ECA8000E7AA5EE856A26EEA55AA5EE867AE5EED9
:10ECB800076A26EEA70AFFF76FB900BFCC47002006
:10ECC800D44300206F12833A0400002084F9223FC5
:10ECD80092E741B99730083C15A82ABE95ED006A1D
:10ECE8009DED0E4ACC4825EE866AFDEEE43AA4EE88
:10ECF800076AB0EE674AA6EE264A13EE907AB4EE9B
:10ED0800C45AF1EE10FAB0EE446A88BFB0EE646AF5
:10ED1800BDEEC66A16EE10EA16EE101AE645A8BF52
:10ED280061467745C8BF394606EE101AB8EEC66A7E
:10ED3800012A80ED006A3DF4E0AF95ED046A9DED8F
:10ED48000F4A25EE866AA4EE076AB0EE674AA6EE79
:10ED5800264AB4EEC45AF1EE10FAB0EE446A88BFFF
:10ED6800B0EE646ABDEEC66A16EE10EA16EE101A28
:10ED7800E645A8BF6146BE45B8BF394606EE101A3B
:10ED8800B8EEC66A022A80ED016A3DF4B6AF95ED89
:10ED9800086A9DED104A25EE866AA4EE076AB0EE71
:10EDA800674AA6EE264AB4EEC45AF1EE10FAB0EE5F
:10EDB800446A88BFB0EE646ABDEEC66A16EE10EA11
:10EDC80016EE101AE645A8BF6146BE45B8BF3946DB
:10EDD80006EE101AB8EEC66A032A80ED026A3DF400
:10EDE8008CAF95ED0C6A9DED114A25EE866AA4EE6E
:10EDF800076AB0EE674AA6EE264AB4EEC45AF1EEA8
:10EE080010FAB0EE446A88BFB0EE646ABDEEC66A16
:10EE180016EE10EA16EE101AE645A8BF6146BE4582
:10EE2800B8BF394606EE101AB8EEC66A042A80ED55
:10EE3800036A3DF462AF95ED106A9DED124A25EE26
:10EE4800866AA4EE076AB0EE674AA6EE264AB4EED2
:10EE5800C45AF1EE10FAB0EE446A88BFB0EE646AA4
:10EE6800BDEEC66A16EE10EA16EE101AE645A8BF01
:10EE78006146BE45B8BF394606EE101AB8EEC66AF6
:10EE8800052A80ED046A3DF438AF95ED146A9DEDCE
:10EE9800134A25EE866AA4EE076AB0EE674AA6EE24
:10EEA800264AB4EEC45AF1EE10FAB0EE446A88BFAE
:10EEB800B0EE646ABDEEC66A16EE10EA16EE101AD7
:10EEC800E645A8BF6146BE45B8BF394606EE101AEA
:10EED800B8EEC66A062A80ED056A3DF40EAF95EDD8
:10EEE800186A9DED144A25EE866AA4EE076AB0EE0C
:10EEF800674AA6EE264AB4EEC45AF1EE10FAB0EE0E
:10EF0800446A88BFB0EE646ABDEEC66A16EE10EABF
:10EF180016EE101AE645A8BF6146BE45B8BF394689
:10EF280006EE101AB8EEC66A072A80ED066A3DF4A6
:10EF3800E4AE95ED1C6A9DED154A65EE865AE7EE3E
:10EF4800045AE6EEA57AB4EEE75AF1EE10FAC8BF15
:10EF5800F0EE647AFDEEE77A17EE901A8C45A8BFBA
:10EF68008C468F42D8BF674607EE907AF8EEE77A6C
:10EF7800C0ED077AFDF7BEBE28494A69002A3CF46D
:10EF880099AA0A6813604B74FCF794BA244DFDF7EC
:10EF98000BB8D4F89C51079B5D1BFFF775BA214B42
:10EFA8001B78DA0704D408F013FA002840F06885C3
:10EFB8001D4DD4F80C222B689A423EF69AAA3B784B
:10EFC800012B3DF4A1A9194C2278002A3DF49CA9F3
:10EFD8000B2B19D801229A4040F6030112EA0108C6
:10EFE8007EF4F5AF12F4C06F0ED0093B012B0BD89D
:10EFF80045201BF091F8FF201BF08EF80C481BF001
:10F0080001F840461BF088F80A4B2A685A600B231F
:10F018003B70FEF7DCBF00BFCC470020D075002056
:10F02800984D00204D760020F0750020595E002094
:10F03800D4640308F85F00200D9B002B00F0718357
:10F04800E34D9DED0E4A95ED006A089B25EE866A14
:10F05800A4EE076AB0EE674AA6EE264AB0EE446A06
:10F0680033B1B4EE445AF1EE10FAC8BFB0EE646A98
:10F07800FDEEE44ABDEEC66A14EE907A16EE101A5A
:10F088008F4214EE90EA00F3F3846145A8BF61460D
:10F0980006EE101ACF48B8EEC66A012A80ED006A5B
:10F0A8003CF4BCAE95ED046ADDED0F4A089B25EEF5
:10F0B800866AA4EE876AF0EE674AE6EE264AB0EE64
:10F0C800646A002B00F0CA84B4EEE45AF1EE10FA38
:10F0D80040F3C48439466145A8BF614606EE101A5C
:10F0E800B8EEC66A022A80ED016A3CF497AE95ED47
:10F0F800086ADDED104A089B25EE866AA4EE876A49
:10F10800F0EE674AE6EE264AB0EE646A002B00F09D
:10F118009B84B4EEE45AF1EE10FA40F39584394634
:10F128006145A8BF614606EE101AB8EEC66A032A02
:10F1380080ED026A3CF472AE95ED0C6ADDED114A81
:10F14800089B25EE866AA4EE876AF0EE674AE6EE2B
:10F15800264AB0EE646A002B00F06C84B4EEE45AE0
:10F16800F1EE10FA40F3668439466145A8BF61465E
:10F1780006EE101AB8EEC66A042A80ED036A3CF45B
:10F188004DAE95ED106ADDED124A089B25EE866AB4
:10F19800A4EE876AF0EE674AE6EE264AB0EE646AA5
:10F1A800002B00F03D84B4EEE45AF1EE10FA40F37F
:10F1B800378439466145A8BF614606EE101AB8EE95
:10F1C800C66A052A80ED046A3CF428AE95ED146AF7
:10F1D800DDED134A089B25EE866AA4EE876AF0EEF9
:10F1E800674AE6EE264AB0EE646A002B00F00E8409
:10F1F800B4EEE45AF1EE10FA40F30884394661455A
:10F20800A8BF614606EE101AB8EEC66A062A80ED57
:10F21800056A3CF403AE95ED186ADDED144A089BC7
:10F2280025EE866AA4EE876AF0EE674AE6EE264A7D
:10F23800B0EE646A002B00F0E083B4EEE45AF1EE1D
:10F2480010FA40F3DA8339466145A8BF614606EEF5
:10F25800101AB8EEC66A072A80ED066A3CF4DEADDD
:10F2680095ED1C6ADDED154A089B65EE865AE4EEBD
:10F27800875AE5EEA67A002B00F0B783F4EEC57A3C
:10F28800F1EE10FA40F1B1833A466245A8BF6246F2
:10F29800964607EE90EAF8EEE77AC0ED077AFCF7B3
:10F2A800BDBDD4F89C51079B5D1BFFF723B907EE42
:10F2B800905ADFED496A9FED497A84F80452F8EED6
:10F2C800E77A67EEA67A77EE876ABDEEE66A16EE0B
:10F2D800103A2033402B40F29782DFED416A414BD0
:10F2E800BDEEE77AC3ED016A17EE103A2033402BE2
:10F2F80000F260829FED3C7AF4EEC77AF1EE10FAE4
:10F3080040F3CA83DFED395A9FED396A01E0F0EE28
:10F31800477AF4EEC67AF1EE10FA37EEE57AF6DCC3
:10F32800DFED347AB4EEE77AF1EE10FA40F1B1830A
:10F33800DFED2E5A9FED306A01E0B0EE677AB4EE49
:10F34800C67AF1EE10FA77EE257AF6D49FED237A95
:10F35800F4EEC77AF1EE10FA40F3E3829FED227AD9
:10F3680077EE677A67EEA75A9FED245A9FED246AD5
:10F378009FED247AA5EE856A27EEA55AA5EE867A32
:10F38800E5EE077AC4ED827AFDF77ABD95ED000ABD
:10F398000893069222F060FF1B49DFF870E0D1F86D
:10F3A800EC10DFF86CC0069AACF800008EFB013E4A
:10F3B800C917C1EBAE1107EE901AF8EEE77A089B71
:10F3C800FDEEE77A17EE901AACF80210FCF7F1BDE3
:10F3D800E4380020CC47002035FA8E3CDB0FC93FCB
:10F3E8000000000004000020DB0F4940DB0FC9408B
:10F3F800E4CB1641DB0F49C0E4CB16C192E741B913
:10F408009730083C15A82ABE341C0020D34D621042
:10F41800144C002025EE866AA5EE076AB0EE675AFE
:10F42800A6EE265ABDEEC56A16EE100A814200F312
:10F438006C816045A8BF604606EE100A0A9BB8EECC
:10F44800C66A002B00F01084DC48012A80ED006AAF
:10F458003CF4E4AC95ED046A9DED0F5A25EE866AFE
:10F46800A5EE076AB0EE675AA6EE265ABDEEC56A43
:10F4780016EE107AB94200F346816745A8BF674681
:10F4880006EE107A0A9BB8EEC66A002B00F0A98334
:10F49800022A80ED016A3CF4C1AC95ED086A9DED45
:10F4A800105A25EE866AA5EE076AB0EE675AA6EEF0
:10F4B800265ABDEEC56A16EE107AB94200F32D81C0
:10F4C8006745A8BF674606EE107A0A9BB8EEC66A7B
:10F4D800002B00F0A483032A80ED026A3CF49EAC62
:10F4E80095ED0C6A9DED115A25EE866AA5EE076A20
:10F4F800B0EE675AA6EE265ABDEEC56A16EE107A29
:10F50800B94200F308816745A8BF674606EE107A3E
:10F518000A9BB8EEC66A002B00F07783042A80EDB8
:10F52800036A3CF47BAC95ED106A9DED125A25EE0A
:10F53800866AA5EE076AB0EE675AA6EE265ABDEEB1
:10F54800C56A16EE107AB94200F3E3806745A8BF92
:10F55800674606EE107A0A9BB8EEC66A002B00F0E2
:10F56800B182052A80ED046A3CF458AC95ED146A22
:10F578009DED135A25EE866AA5EE076AB0EE675A26
:10F58800A6EE265ABDEEC56A16EE107AB94200F309
:10F59800BE806745A8BF674606EE107A0A9BB8EE9C
:10F5A800C66A002B00F02783062A80ED056A3CF422
:10F5B80035AC95ED186A9DED145A25EE866AA5EED0
:10F5C800076AB0EE675AA6EE265ABDEEC56A16EE71
:10F5D800107AB94200F3A3806745A8BF674606EED4
:10F5E800107A0A9BB8EEC66A002B00F07582072ACB
:10F5F80080ED066A3CF412AC95ED1C6A9DED155A37
:10F6080065EE865AE7EE055AE5EEA67AFDEEE77A4C
:10F6180017EE902A914203DC6245A8BF6246114664
:10F6280007EE901A0A9BF8EEE77A002B7FF435AEC6
:10F638000C9B002B7FF431AE0B9B9E45B8BFF0EEC0
:10F64800647A2AE65E4A1278032A00F015820022BC
:10F65800FEF7C8BD9FED5B8AFFF702B99FED598A97
:10F66800FFF7D6B89FED580ADFF8708125EE800ABB
:10F6780022F0F2FDD4F81451A8F80600FDF717B9E6
:10F68800D4F89C51079B5D1BFDF7C0BF4F49096823
:10F6980011F080530A937EF44DAFFEF742BF4C48F9
:10F6A8004C498046FEF73FBA07981AF0D5FEFDF799
:10F6B80013BFF5F753FE059BDFF8208193F800E0B0
:10F6C800069B3178D4F81451C01AA8F80400FEF744
:10F6D800E6BBF5F743FE059BDFF8008193F800E0F1
:10F6E800069BC01AA8F80200FEF74FBBF5F736FED6
:10F6F800059BDFF8E88093F800E0069BC01AA8F89D
:10F708000200FEF762BB0F46BAE6084694E60F46CB
:10F7180042E70F461DE70F46F8E60F46D3E60F46C9
:10F728005DE70EA9BDEEE46A01EB820290462A4825
:10F73800089A224D0A9B089416EE107A05E0414576
:10F74800A5EC016A00F1100031D090ED006AB1EC2F
:10F75800014A25EE866AA7EE046AB0EE674AA6EE6D
:10F76800864AB0EE446A32B1B4EE445AF1EE10FA69
:10F77800C8BFB0EE646ABDEEC64A06EE107A14EE53
:10F78800104AA74206DC14EE104A6445A8BF644636
:10F7980006EE104AB8EEC66A002BD0D10C9C002C9D
:10F7A800CDD10B9CA645B8BFB0EE646AC7E7089CEC
:10F7B800FCF734BBDFED037AE4E500BFCC4700205B
:10F7C8009C770020000000000000C842EC5F002089
:10F7D8005445002068240020E4380020144C002000
:10F7E80092E741B99730083C15A82ABEE4CB1641E8
:10F7F800DB0FC940E4CB16C1DB0FC93FDB0F494023
:10F80800DB0FC9BFDB0F49C0F4EEC77AF1EE10FA7F
:10F8180040F355815FED0A5A1FED0C6A01E0F0EEE6
:10F82800476AF4EEC66AF1EE10FA36EEE57AF6DCCF
:10F838005FED0C6AB4EEE67AF1EE10FA40F12F8132
:10F848005FED155A1FED156A01E0B0EE667AB4EE69
:10F85800C67AF1EE10FA77EE256AF6D41FED1A7A19
:10F86800F4EEC76AF1EE10FA40F3B3801FED1D7A8B
:10F8780077EE666A66EEA65A1FED275A1FED276ACD
:10F888001FED277AA5EE856A26EEA55AA5EE867A9B
:10F89800E5EE076A23E51FED277AF4EEC76AF1EE75
:10F8A80010FA40F39B815FED2E5A1FED306A01E09C
:10F8B800F0EE476AF4EEC66AF1EE10FA36EEE57A33
:10F8C800F6DC5FED306AB4EEE67AF1EE10FA40F15C
:10F8D80082815FED395A1FED396A01E0B0EE667A30
:10F8E800B4EEC67AF1EE10FA77EE256AF6D41FED7B
:10F8F8003E7AF4EEC76AF1EE10FA05DD1FED417AA3
:10F9080077EE666AFFF7C5B91FED437AF4EEC76A6A
:10F91800F1EE10FA44BF1FED457A77EE666AFFF7FD
:10F92800B8B91FED497AF4EEC77AF1EE10FA44BF80
:10F938001FED4C7A77EE677A14E5D14F07F1800214
:10F94800FEF794BAA8F80600ABF8A860CC4CFBF711
:10F95800EABBF2F748FB00283EF490ACFEF725BD61
:10F9680080201CF0E9F808B103F066FD0FF0E4FC14
:10F97800FEF78CBC40200AF07FFE00287EF47EACA7
:10F98800D8F80030DFF844A3DFF844B34FF040095B
:10F998000EE01AF0C1FBDBF80020D8F80030013A7D
:10F9A8000133B9F10109CBF80020C8F8003079D04B
:10F9B8001AF803301846002BEBD100234FF0FF3222
:10F9C800C8F800300423C8F804203B70AA78FDF773
:10F9D80086BD9FEDAC7AF4EEC76AF1EE10FA44BF2B
:10F9E8009FEDA97A77EE666A44E7FDEEE77A17EEAF
:10F9F800902ABA42FFF64DAC47E4BDEEC66A16EE51
:10FA0800101AB942BFF620AC394620E4BDEEC66AEA
:10FA180016EE101AB942BFF6F2AB3946FFF7F2BB41
:10FA2800BDEEC66A16EE101AB942BFF6C3AB394628
:10FA3800FFF7C3BBBDEEC66A16EE101AB942BFF691
:10FA480094AB3946FFF794BBBDEEC66A16EE101AA2
:10FA5800B942BFF665AB3946FFF765BBBDEEC66A6E
:10FA680016EE101AB942BFF636AB3946FFF736BB69
:10FA780014EE901AFFF70CBB04F060F9FBF74CBBCF
:10FA8800824B1B6803F59C530833C4F80C32FDF70E
:10FA980030BDF0EE477A59E4B0EE677A40E4F0EE14
:10FAA800476ADBE61AF80330002B7EF4E7AB84E7FD
:10FAB80094F87831002B7BF4CBADFBF7B6BDB0EEF4
:10FAC800667AB5E60C9B002B7FF44BAD0B9B9E45ED
:10FAD800B8BFB0EE646A44E50C9B002B7FF487AD99
:10FAE8000B9B9E45B8BFB0EE646A80E5684A694BD7
:10FAF80010681B689847684BD7ED006A93ED007A49
:10FB0800664BD3ED007A664B83ED020A654B67EED0
:10FB1800277A2B4427EEAC7AD3ED007A624B67EE56
:10FB2800277AF0EE665AEDEEA75A93ED006AB1EE29
:10FB3800467AB4EEE57AF1EE10FA08DCF4EEC65A2D
:10FB4800F1EE10FA8CBFB0EE467AB0EE657A574BFC
:10FB58001B78012B02D0192B7BF4E4ACDFED547A2F
:10FB6800F4EEE7DAF1EE10FACCBF01230023FBF73D
:10FB7800E4BCDFED507AB4EEE7EAF1EE10FA27DCE8
:10FB8800DFED4D7AB4EEE7EAF1EE10FA20D44B4BF4
:10FB9800D3ED007AB1EE677AF4EEC7DAF1EE10FA37
:10FBA80013D4F4EEE7DAF1EE10FA88BFF0EE67DA74
:10FBB800434B87ED00CA1B689342BBF6A1ABFBF72A
:10FBC80005BC04F015F8FEF7EBBBF0EE47DAEFE7FB
:10FBD800DFED3CDAECE7F0EE476A88E6B0EE667AED
:10FBE8006FE60C9B002B7FF453AC0B9B9E45B8BF74
:10FBF800B0EE646A4CE40C9B002B7FF4D5AC0B9BF5
:10FC08009E45B8BFB0EE646ACEE40C9B002B7FF42F
:10FC180085AC0B9B9E45B8BFB0EE646A7EE40C9B36
:10FC2800002B7FF458AC0B9B9E45B8BFB0EE646ABE
:10FC380051E4132B05D1B0EE480A22F00DFB099BC5
:10FC48001880B0EE480ADBF808321F489847059B31
:10FC58001B78132BB0EE408A7CF4E1AE22F0FCFA5C
:10FC6800099B5880FCF7DBBE0C9B002B7FF4ECABA8
:10FC78000B9B9E45B8BFB0EE646AFFF7E5BB00BFBB
:10FC880068240020DB0FC9BFDB0F49C0F0750020D6
:10FC9800503800206438002004000020A4370020D9
:10FCA8006C47002074380020DC380020685C002095
:10FCB8000000964200C0F84400C0F8C4D8380020BC
:10FCC800BC38002000000000B06E0020CC380308CB
:10FCD8001C3D00202DE9F04F2DED028B93B0054619
:10FCE80020F0F8F8B64B1E7826B113B0BDEC028BA5
:10FCF800BDE8F08FB34B1B685A05F6D5DFF82483AF
:10FD0800D8F80020002A00F02381AF4CD4F828311D
:10FD180003F5F43348339D42C0F01A81DFF808B385
:10FD280094F82C31DBF80010C4F82851013384F81A
:10FD38002C318B0701F17E8011F0140F41F06180A6
:10FD480094F82C3113F0070701F0D880282B9F4B2B
:10FD5800029301F0D8815E2090479D4B1B78002BC1
:10FD68006BD0994C9B4AD4F83031EB1A934200F28D
:10FD7800D187DFF8B8A29AF80080B8F1000F33D124
:10FD8800DFF86092D9F80000F5F798FDC0B20128B5
:10FD98000ED90228904F41F0B9823B78002B41F0F0
:10FDA8004E84D4F83831EB1AB3F57A6F81F0DA84DF
:10FDB8008A480768002F40D09AF80030BBB9884BB2
:10FDC800D9F800001B689B781E3B012B4FF00201FD
:10FDD80041F24084043012F01FF9012200238AF80E
:10FDE800002084F8443126E07C4807682FB3D4F813
:10FDF800403140F6B732EB1A93421ED994F83C31A1
:10FE0800002B01F07A82013BDBB284F83C31002BF5
:10FE180001F05E8117F8011B94F84421076094F8FB
:10FE2800453170480A440133006884F8442184F855
:10FE38004531F5F747FDC4F840516B4A029B1278EB
:10FE48001B68012A03F101030A9300F0B486674B8B
:10FE58001B786BB1664F3B6853B1029B5A4CD3F881
:10FE680000B0D4F85831ABEB0303632B00F258868B
:10FE7800DFF8BC8198F800A0BAF1020F01F0048104
:10FE8800554F97F87430032B00F0A587594B1B7812
:10FE980073B1594E33685BB14B4CF5F75FFAD4F840
:10FEA800643144F61F62C31A9342834600F2D48039
:10FEB800524B1B78002B4ED1514B1B7843B1424C0F
:10FEC800D4F8B43203F50043E8339D4280F0E98664
:10FED8004C4B1B78002B3FF408AF3B4E4A4C4B4D24
:10FEE80006F2BD272068F5F7E9FC00283FF4FDAECF
:10FEF8002068F5F7DBFC2B7880465A1E33B1206862
:10FF08002A70F5F7DBFC0028F2D1EEE60322394629
:10FF1800781E23F044F996F8BC3296F8BD2286F88C
:10FF2800BF8283F47F4383F0FF039B1A1FFA88F88C
:10FF38009BB2B8EB132FD5D196F8BE22DBB29A420A
:10FF4800D0D1781E11F07AFB2B7818442870C9E7B5
:10FF58001E4B029301E72E4C2278002A40F022869D
:10FF6800DFF8D09099F80040002C65D1294E307800
:10FF7800002841F0EF82144C274ED4F8AC22317897
:10FF8800264B93FBF1F313449D4295D3244A94F8EE
:10FF9800B032C4F8AC52D75CF90701F16984BA07EA
:10FFA80001F1FE837B0701F18C8394F8B03231783C
:10FFB800013393FBF1F201FB123384F8B0327BE793
:10FFC800CC4A00202C6F002084260020F0750020E9
:10FFD800EE7700203F0D03000C000020D84F0020D2
:10FFE800D44F0020D04F0020EF770020FC7700206E
:08FFF800A8600020047800203D
:020000040801F1
:100000000878002048780020597800200E780020D9
:100010001478002018780020E07700205078002025
:1000200058780020A086010054780020E04F00207E
:10003000644F0020DC4F0020385A00205178002007
:10004000054E376E002F41F09D80044B89F80070FB
:10005000C3F8AC5234E700BF60780020842600204B
:1000600094F86A31002B41F03F80E04B1B6803F0AD
:100070000802002A48F603414AF60B404BF60F42AD
:1000800049F6074704BF02460F4613F0040F4FF02E
:10009000190118BF17469A0684F86A1103D547F468
:1000A000804747F0200704F037FDC7F30908002810
:1000B00041F0EB84CE4B9B79002B41F03D859A4675
:1000C00064204FF0FF394FF0000C0A970B97ADF802
:1000D00034C0CDF83AC0CDF83EC0CDF842C0CDF81E
:1000E0003080ADF836A0ADF838908DF846000AAFF4
:1000F0000FCFDFF80CE384F805C0AEE80F0097E8F7
:100100000F00AEE807002EF8023B71464FF0010CDD
:100110001B0CFE271F20C82201F81E39A770A271F0
:1001200084F807C0E07094F87A01207180F0F10340
:1001300083EA0313DAB2130983F0E70343EA0223E5
:1001400083EAC2031BB283EA0312D2B2C3F30723CA
:1001500083EA121343EA022383EAC2031BB283F049
:10016000C80282EA0212D2B2C3F3072383EA12134F
:1001700043EA022383EAC2031BB283EA0C0787EA3D
:100180000717FFB2C3F3072282EA171242EA0722D7
:1001900000EB0C0382EAC7070EEB0C0084F87A31FF
:1001A000278011F8013B7B4083EA0313DBB21A0975
:1001B00082EA172242EA032282EAC3031BB29FB2F9
:1001C00081422780EDD183F07C0383EA0313DBB205
:1001D0004FEA131E8EEA172E8EEA032E8EEAC30E06
:1001E0000FFA8EFE1FFA8EF9DFF818C2A4F80090FD
:1001F0005FFA8EFE4FEA192984F8289084F827E0E8
:100200000CF5D17804F1220ADCF80000DCF80410C7
:10021000DCF80820DCF80C3047460FC70CF1100C56
:10022000D445B846F0D1DCF800003860714F9CF836
:10023000043088F8043007F1270884F8C9E184F80D
:10024000CA9117F8011F3068F5F740FBB845F8D19F
:1002500094F86B21002A40F04C876749029B08788C
:100260001B680A2184F86B11002801F00181DFF876
:1002700098E10128BEF80010059141F2648402283B
:10028000BEF8028001F01A84BEF80410049103281D
:1002900001F014850428BEF806A001F00A85BEF816
:1002A00008100391052801F000850628BEF80AC051
:1002B00001F0F8840728BEF80C1001D0BEF80E201B
:1002C00094F87A010A93074687F0300383EA031310
:1002D000DBB24FEA131E494806978EF07A0E4EEABB
:1002E000032E008827718EEAC303DFF820E1C0EBFC
:1002F00000208EFB007E8644C017C0EB6E27079758
:10030000059F4FF0000967F30F09049F68F31F4929
:100310004FF0000867F30F08039FCDF82C901BB235
:100320004FF0000E83EA031067F30F0E0027C0B2F0
:1003300061F30F07C3F307236CF31F4E62F31F47EC
:100340004FF0000C9DF81C20CDF834E083EA101328
:100350006AF31F48CDF830800E978DF83CC08DF8B9
:100360003D2043EA00230DF1280883EAC007B8E8DE
:100370000F003FB287F0C80989EA0919DFF880E069
:1003800084F805C05FFA89F9C7F30727AEE80F00C4
:1003900087EA191747EA092398E8030083EAC903A3
:1003A0001BB283F023074EF8040B87EA0717FFB24E
:1003B000C3F3072282EA1712069B704642EA07221D
:1003C00003F1010882EAC70720F814194FF0230C43
:1003D000FE211622C82384F87A8127800EF1020EAE
:1003E00084F807C0A170E270A37111E0644F00208F
:1003F000544F0020272800200C4B00208477002039
:100400008C260020862600203E61002003082080E4
:1004100010F8013B7B4083EA0313DBB21A0982EA3E
:10042000172242EA032282EAC3031BB29FB270453D
:100430002780EDD183F0F40383EA0313DBB24FEAA4
:10044000131E8EEA172E8EEA032E8EEAC30E0FFAC3
:100450008EFE1FFA8EFCD54FA4F800C04FEA1C296F
:100460005FFA8EFE84F81EE084F81F907968BA68FF
:100470003868FB6807F5D17CACE80F00386979690A
:10048000BA6904F2C118ACE8070004F2A31784F8B3
:10049000C19184F8C0E117F8011F3068F5F716FA2A
:1004A000B845F8D194F87271002F40F02B86C04BFC
:1004B00094F87AC1B3F90010B3F90220B3F904300B
:1004C0009FEDBC6A677107EE103A029B1B680A93A6
:1004D0008CF06A0383EA031306EE901AD9B20B0973
:1004E00083F0D50343EA012383EAC1031BB283EA05
:1004F00003115242C9B207EE902AC3F3072383EADD
:10050000111343EA0123F8EEE77AF8EEE66AB8EE53
:10051000C77A83EAC1031BB267EE867A66EE866A03
:1005200027EE067A002083F0C80ECDED0C7ACDEDD3
:100530000B6A8DED0D7A0E900F9010908EEA0E18CA
:100540000DF128095FFA88F8C3F3072EB9E80F0008
:100550008EEA181E4EEA082E8EEAC80EDFF8708268
:100560000FFA8EFEA8E80F008EF01E0799E807002C
:1005700087EA071A5FFA8AFACEF3072787EA1A177B
:1005800047EA0A2788E8070087EACA071C214FF0D4
:10059000050A4FF01E094FF0FE0EC8220CF10103B0
:1005A000E17084F872A184F8079084F802E0A8F161
:1005B0001001A27108F10C0084F804C0278084F8AF
:1005C0007A3111F8013B7B4083EA0313DBB21A094D
:1005D00082EA172242EA032282EAC3031BB29FB2D5
:1005E00081422780EDD183F0270383EA0313DBB236
:1005F0001A0982EA172282EA032282EAC3031BB2A3
:100600001FFA83FCDFF8A481A4F800C05FFA83FE20
:100610004FEA1C2C84F825C084F824E008F5D17931
:1006200004F1220AD8F80000D8F80410D8F80820FD
:10063000D8F80C304F460FC708F11008D045B9461E
:10064000F0D15D4FB8F80030A9F8003007F1240868
:1006500084F8C6E184F8C7C117F8011F3068F5F7C0
:1006600035F9B845F8D194F873310293002B40F076
:100670004585524B1B68052213F0140F84F8732133
:1006800040F0EB86DFED4E7A94F87AC1484B4D4A44
:10069000B3F90410B2F906204B4F4C48CDED0C7A5B
:1006A0008CF0220383EA03135FFA83FE4FEA1E13E2
:1006B00083F0590343EA0E23B2F5FA6F83EACE03BF
:1006C0001BB2A8BF4FF4FA6283EA031EB2F57A7F29
:1006D0005FFA8EFEB8BF4FF47A72C3F307234FF070
:1006E000640883EA1E13A2F57A7208FB02F243EA59
:1006F0000E2387FB028783EACE0ED2174FF0000944
:1007000080FB0180C2EBA712C9170FFA8EF7CDF854
:100710002890CDF82C90CDF83490C1EBA00387F051
:10072000C8090DF12808ADF83A20ADF83830C646B2
:1007300089EA0919BEE80F005FFA89F9C7F30727AC
:1007400087EA191747EA092787EAC909204FDEF81F
:1007500000E084F804C00FC70FFA89F989F04A0352
:1007600083EA0310C0B2C9F3072383EA10133A46A1
:100770000CF1010143EA002383EAC00342F810E9C7
:1007800000204FF04A094FF0FE0C4FF0140E84F891
:100790007A11C82160712380043784F8079084F8A7
:1007A00002C084F803E0A171184613E086260020F9
:1007B000704F002088C3E43A27280020644F0020AF
:1007C000000000003E610020D34D6210676666663F
:1007D0008C26002012F8011B414081EA0111C9B2A8
:1007E0000B0983EA102343EA012383EAC10109B21A
:1007F00088B2BA422080EDD181F0140181EA011162
:10080000C9B24FEA111E8EEA102E8EEA012E8EEA30
:10081000C10E0FFA8EFE1FFA8EF94FEA192CBC4B4F
:10082000BB4884F81DC05FFA8EFE84F81CE0B84F08
:1008300059689A680068DB68A4F8009007F5D179D8
:10084000A9E80F0038697969B7F818A0A9E803008A
:1008500004F2A317A9F800A0BA4684F8BFC184F82F
:10086000BEE104F2BF191AF8011F3068F5F72EF83F
:10087000D145F8D1A74BA84A1B781278013B12F05A
:100880000100DBB214BFC0214021172B03D8A34ABB
:1008900013441B7B0293A24B1A8893071ABF0023B1
:1008A00041F01001012312F4027F18BF022312F05D
:1008B000100F18BF062312F0200F18BF10230028B6
:1008C00040F04A874FF0030994F87AC10A938CF0FC
:1008D000460383EA0313DAB2130983F0920343EA6F
:1008E000022383EAC2031BB283EA0310C0B2C3F33C
:1008F000072282EA101242EA002282EAC00212B201
:1009000082F0C80E8EEA0E1E00235FFA8EFE9DF85E
:1009100008A08DF82CA00320C2F307228DF82F9099
:1009200082EA1E128DF82D308DF82E108DF83000D1
:1009300042EA0E2998E8070089EACE0E0FFA8EF8EF
:10094000DFF8E0E1E37188EA0819AEE803005FFA36
:1009500089F9C8F3072888EA191848EA092181EAC1
:10096000C90994F808808EF800200FFA89F988EAFE
:10097000090282EA02185FFA88F8C9F3072282EABC
:10098000181242EA0822607AA17A94F80B906371F7
:1009900082EAC80212B2504080EA0010C0B2C2F32C
:1009A000072282EA101242EA002282EAC00212B250
:1009B000514081EA0111C9B2C2F3072282EA111241
:1009C00042EA012282EAC10212B289EA020989EAF4
:1009D00009195FFA89F9C2F3072282EA191242EA79
:1009E000092294F80C80607BA17B84F804C082EA21
:1009F000C90212B288EA020888EA08185FFA88F881
:100A0000C2F3072282EA181242EA082282EAC802E6
:100A100012B2504080EA0010C0B2C2F3072282EA4C
:100A2000101242EA002282EAC00212B2514081EA68
:100A30000111C9B2C2F3072282EA111242EA01226D
:100A400082EAC102E17B94F8109013B281EA0302BA
:100A500082EA0212D2B2C3F3072383EA121343EAF3
:100A6000022383EAC2031BB289EA030282EA02126A
:100A7000D2B2C3F3072383EA121343EA022383EAC1
:100A8000C2031BB283F0320282EA0212D2B2C3F373
:100A9000072383EA121343EA022383EAC2031BB249
:100AA0009AB24FF0FE08DBB222800920C8210CF177
:100AB000010C84F802804FEA1228AEF10E02E070B9
:100AC000A17184F87AC184F812800293637451682A
:100AD0005EF80E0C92683EF8023C0EF5CA7CACE85B
:100AE0000700ACF800309DF808308CF802900EF545
:100AF000D27A84F8B48184F8B33117F8011F3068D2
:100B0000F4F7E4FEBA45F8D1C4F864B1FFF7D4B9FC
:100B1000862600200C4800204D7600200C3B030860
:100B2000C04F00208C260020DFF8BCA3DFF8BC8378
:100B3000DFF8BC93412010F0CBFFBAF9023088FBFC
:100B40000320DB17C3EBA00080B210F0A7FFBAF9B7
:100B5000003088FB0320DB17C3EBA00080B210F04D
:100B60009DFFBAF9043088FB0320DB17C3EBA0001C
:100B700080B210F093FF99F800103868F4F7A6FEE1
:100B800094F85C3113F0010800F0D583C44AC4F82E
:100B900058B10133DBB2A2FB0312D20802EB82028E
:100BA000A3EB420384F85C31FFF766B9BD4BBE4945
:100BB0001868F4F757FE00232370FFF7D5B9BB4F31
:100BC000386800283FF447A94FF0000ADFF8248373
:100BD000B74CAB465546F4F775FEF8B1F5B94FF092
:100BE0000109AA463868F4F765FE83B27E2B00F04F
:100BF000648298F80120002A49D194F84811B1B1D3
:100C00001B2B84F8482100F032820D2B45D0386828
:100C100088F80190F4F756FE0028E3D1AA46504622
:100C20000AAAA4495D4610F06BFFFFF714B97D2BAB
:100C300000F0288494F84C2122B180F02003DBB22C
:100C400084F84C1194F84721062A10D8B4F84A11B8
:100C500038681944A4F84A11A118013281F85031BA
:100C600084F84721F4F72EFE0028BBD1D6E7B4F86C
:100C70004A2188F8019013449BB21A0A52FA83F36E
:100C8000FF2BA4F84A31386802D18B4DA3E73868AE
:100C9000F4F718FE0028A5D1C0E73868A4F84A2167
:100CA000F4F710FE00289DD1B8E794F8B832C4F8E4
:100CB000B452012B40F2298394F8B9227F49981845
:100CC00001EB8001013202F001024E6A84F8B92280
:100CD000BEB17B4F0B970DF14808123FA52348F892
:100CE000207D802284F8103115232946404684F85F
:100CF000112184F81231B047002840F0688294F83E
:100D0000B832704A013382FB0312A2EBE37202EBAA
:100D100042029B1A84F8B832FFF7DEB86A4A6B4B7E
:100D200092F80BE0029AD4F8341110681B88684AD4
:100D3000401A4FF47A71DFB201FB0EF11B0A97776C
:100D4000177588424FF00007D37753759770177166
:100D500080F0C8825F4B6049DFF89CE11B68DFF8D8
:100D60007CC10F688868DCF80010C4F830518EFB35
:100D7000038CDB17C3EB6C13DFF870C18EFB018EA5
:100D80008CFB07988CFB009CC017C0EBAC0003F5F4
:100D9000FA734FEAE17C9BB2CCEB6E1CFF1701F5B6
:100DA000EA4EC7EBA8070EF1300E93761B0A0CF142
:100DB000780C4FEA2E2E3031D3764FEA27280312D3
:100DC000177782F81D8082F8200082F8213082F89F
:100DD00024C082F823E082F82210FEF7CEBFDFF8AD
:100DE0001C91D9F80000F4F761FD00283FF452A8E7
:100DF000D9F800000121F4F755FD0222002387F8FD
:100E0000742088F80030FFF745B85E209047D8F886
:100E1000003030209847314B1F68F8B211F054F978
:100E2000C7F3072011F050F994F82C3113F00302A6
:100E300000F03283D8F80020FEF788BFDFF8C090BA
:100E40009FED278A4FF0240A5E2090475046D8F83D
:100E500000309847234BF9EC016A9B8A07EE103A61
:100E6000F8EEE66AB8EEC77A0AF1010AC6EE877AAA
:100E70005FFA8AFA67EE887AFDEEE77ACDED027ABC
:100E8000BDF90870F8B211F01FF9C7F3072011F08F
:100E90001BF9BAF1270F00F0E480D8F80020D3E75F
:100EA000CDCCCCCC4C780020A0770020CC4F0020BB
:100EB00084260020CA270020D42700200C3B0308EA
:100EC000A927002056555555884D0020304D00204B
:100ED0001C780020684F00201C4D00206C4F002023
:100EE00000007A44784F0020704F002067666666E5
:100EF000846A00200C0000201F85EB513441002043
:100F0000A84F00205E209047D8F800300220984774
:100F1000FF2010F01DFB0378FF2B00F09D8390F95C
:100F20000130DF17FFB2D8B211F0CEF8384611F019
:100F3000CBF8D8F800305E209847D8F8003003206E
:100F40009847FF2010F004FB0378FF2B00F081830B
:100F5000B0F90830D8B2C3F3072711F0B5F8384616
:100F600011F0B2F8CE4B1B78042B74D0DFF864A3D9
:100F7000B4F82E219AF80010DFF85C9392FBF1F39D
:100F800001FB13239BB2B9F80020A4F82E311F01F6
:100F9000BFB2642303FB02134900B3FBF1F347EA3A
:100FA0000327C3F303225E20D8F80030BFB21743F3
:100FB0009847D8F8003006209847F8B211F084F826
:100FC000380A11F081F8B74AB4F82E31517AB9F8DD
:100FD000009001330129A4F82E3100F08685537B5F
:100FE00009EB89091FFA89F9002B40F0B083D8F882
:100FF0000030AD4F5E209847D8F800303A2098472F
:10100000A7FB09377F091FFA87FA5FFA8AF011F008
:101010005BF84FEA1A2011F057F8D8F800305E203C
:101020009847D8F800303B209847642303FB179378
:101030009BB29E48053380FB0320DB17C3EBA00067
:10104000C0B211F041F8002011F03EF8984FBB7982
:10105000002B40F0078394F82C31D8F80020FEF7DD
:1010600079BEDBF80010D8F80020FEF769BE3868BA
:10107000F4F728FC00287FF4CAAD386884F846915C
:1010800088F80190F4F71EFC00287FF4ABADC5E5AD
:10109000F4F768F9874B1B68A0EB030B40F6B833F5
:1010A0009B4500F23D81844B1A793A2A00F0308446
:1010B000002388F80030FEF7EDBE386884F846A1BA
:1010C00084F847A184F8489188F801A0F4F7FAFB66
:1010D00000287FF487ADA1E594F8441194F84531D8
:1010E00076484A1CFEF7A3BE013B84F86A31FFF73D
:1010F000AFB8013A84F86B21FFF7D4B9013B84F80B
:10110000733101E5013F84F87271FFF7ACBA4FF01B
:10111000000A5E201F6884F82CA19047D8F80030A0
:10112000DFF8B89117209847504610F0CDFF644B78
:10113000A3FB07239B0BA9FB03125209C2EB02126C
:10114000A3EB8203D8B210F0BFFFD8F800305E20C6
:101150009847D8F80030182098475A4BA3FB07232C
:101160009B09A9FB03125209C2EB0212A3EB8203F3
:10117000D8B210F0A9FF504610F0A6FFD8F8002012
:10118000FEF7EDBD0024DFF8588127464FF0500AE6
:1011900002E0DBB283F3118816F804B0601C5946F4
:1011A000304410F079FB002840F0B5810BF10103C9
:1011B0001C44EFF311838AF31288326E9442E8DB09
:1011C0000022DBB2326683F31188FEF73EBF0A9E2F
:1011D000BE4240F29F843D46002141F2210015F8B5
:1011E000013B81EA03235A0013F4004F80EA020115
:1011F00092B289B208BF11464A0080EA020311F494
:10120000004F99B293B218BF0B46590080EA010211
:1012100013F4004F89B293B208BF0B46590013F480
:10122000004F80EA010289B292B208BF0A46530019
:1012300012F4004F80EA03019BB289B208BF19463D
:101240004A0080EA020311F4004F99B293B218BF2A
:101250000B46590013F4004F80EA010289B292B2A2
:1012600008BF0A46530080EA030112F4004F9BB204
:1012700089B208BF1946B542B1D14046F0F7C2FA6B
:1012800011490A9D11486D1A152DA8BF15252A462A
:1012900020F012FE0E4A94F8B832157031E500BF06
:1012A0009C770020884D00201F85EB51676666669D
:1012B000544F0020405A0020285A0020D04F0020D0
:1012C00073B2E745D34D621094270020E43E00201E
:1012D000F93E0020964D0020304D002089888888F6
:1012E000891302088F4B02991B780968C4F83411DE
:1012F000013B012B3FF62EAD10210223917013719B
:1013000028E510F0C3FEFEF79ABD874A02EB830280
:10131000566ADDE410F0AAFE01233B70FEF74CBDD7
:10132000824AB2F85E3100210133A2F85E3188F8BA
:101330000010FEF7AFBD7E4B1B88D90515D4DA0629
:1013400000F1B983980600F1E283590600F1E883C1
:101350001A0700F1E883D80700F1E88313F0020FC1
:101360000CBF4FF004084FF00C08724B724A1B7808
:10137000D27803F001030AB143F002035320039330
:1013800010F0A6FB6D4A128802EB820202EB820289
:10139000900080B210F082FB002010F07FFB684AC2
:1013A000684912883868C2EBC212520081FB0231D0
:1013B00011444FEAE27ACAEB612A5FFA8AFA51468F
:1013C000F4F784FA99F80020039B386848EA030888
:1013D0008AEA020A002189F800A0F4F777FA414668
:1013E0003868F4F773FA99F80030386888EA03032C
:1013F000DBB2194689F80030F4F768FA94F85C31EA
:10140000002B7FF4C3AB4F2010F062FB1AF0E8FB17
:101410001AF0E6FB1AF0E4FB01213868F4F756FAFB
:10142000494A99F8003092F80080386808F00108BD
:10143000414683F0010389F80030F4F747FA99F840
:101440000030386888EA0308414689F80080F4F7DC
:101450003DFA94F85C31FFF799BB3C4B9FED3C7A29
:10146000D3ED007AF8EEE77A67EE877AFFF70CB9EA
:1014700001468446039082460490804605900246C9
:10148000FEF71EBF386884F84C91F4F71BFA002869
:101490007FF4A8ABFFF7C2BB2E49D4F828012B4B31
:1014A00088421F6840F24E8187EAE773A3EBE77337
:1014B000294A1BB282FB0312DF17C7EB62176422B3
:1014C00002FB17331AB23FB25FFA87FB5FFA82FA68
:1014D000C2F30729C7F30727D8F800305E209847E2
:1014E000D8F8003010209847584610F0EDFD3846E7
:1014F00010F0EAFDD8F800305E209847D8F80030A8
:1015000021209847504610F0DFFD484610F0DCFDE2
:1015100094F82C318EE441463A2010F019F9074333
:10152000FFB243E69C7700200C3B03088426002092
:10153000C04F00204D760020244B0020304D00206D
:1015400084770020030820807C770020684F0020EB
:101550000AD7233C3F4B4C001F85EB51B449B54B98
:101560000093A1F13F07B44BB44A099101F8404CF4
:101570000AA8B3490897F0F71CFA089F7B1C089348
:101580003C70089B2922591C08911A70089BEA227A
:10159000591C08911A70089BC822591C08910AA866
:1015A0001A701FF091FD00F101080AA9424608983F
:1015B00020F082FC089A02EB08030133089302F83A
:1015C0000840089B5A1C08921C70089B5A1C0892E1
:1015D0001C70089B5A1C08921C70089B5A1C08928D
:1015E0001C70089B5A1C08921C70089B5A1C08927D
:1015F0001C70089B5A1C08921C70089B5A1C08926D
:101600001C70089B5A1C08921C70089B5A1C08925C
:101610001C70089B5A1C08921C70089B5A1C08924C
:101620001C70089B0122991812A808911A7050F892
:10163000283DDB1B3B701EF01BFC824B3470C3F853
:10164000AC52FEF73DBCC4F8385187F80080FEF775
:10165000B3BB0027384680E4384665E4F4F722F946
:10166000FEF7BFBBD8F80030DFF808A2DFF8009221
:101670005E209847D8F8003028209847DAF80030E4
:1016800089FB0329DB17C3EBA9095FFA89F010F086
:101690001BFDC9F3072010F017FDD8F800305E20BD
:1016A0009847D8F80030042098473B89002B40F039
:1016B0000C82DAF8087087F31007F8B210F004FD16
:1016C000C7F3072010F000FDC5E4594B0B93A3F1BD
:1016D000400800222121A3F13D0903F8402C88F89D
:1016E000021088F80120CDF8289005F0DDFF564B58
:1016F000564A1B88564900280ABF1146032704276B
:10170000580500F1EF81DA0700F1078203F00203C8
:10171000504A002B1CBF032711463A464E4820F082
:10172000CBFB09EB070312A84C4A013340F8203DDC
:101730009B1A002209F8072088F801301EF098FB58
:10174000FEF737BC9146924617469346C4E69AF890
:10175000003099FBF3F94AE4414AD278002A0CBFE1
:101760004FF004094FF00509FFF7AEB80123D9F88F
:1017700000003B70F4F79EF80746D9F80000F4F734
:1017800099F87F067EF418AB8E287EF415AB9AF894
:101790000030002B7EF42CAB324B334A1A602D23E1
:1017A00084F83C31FEF70FBB214A304B0B920DF110
:1017B0004808A2F13D0048F8200D1988DFF8B490E0
:1017C000A2F1400300204FF00A0E02F8400C08225C
:1017D00083F801E040469A70EFF7F0FFD9F8003047
:1017E0002349DA1781FB0313C2EBA30399B24046E6
:1017F000EFF7E4FF03F09EF9D9F808900A9B4FEA4F
:101800001942591C0A911A700A9B4FEA1922591C55
:101810000A911A700A9B5A1C0A9283F800900A9B3C
:101820005A1C0A92187040461EF022FBFEF7BEBBFF
:10183000784D002005550020D8650308E0650308B1
:10184000EC65030884260020C04F0020BC65030817
:10185000C4650308D46503083B4D0020394D0020C2
:10186000244B0020D84F00201C780020304D002051
:10187000676666661C4D0020DFF808939FEDB68A08
:10188000B9F90230B54A0B9207EE903AF8EEE77AD2
:101890000DF1480867EE887AA2F14003FDEEE77A81
:1018A000A2F13D0148F8201D02F8400C0822CDEDC0
:1018B000027A5A701E229A70BDF808104046EFF75F
:1018C0007DFFB9F9003007EE903AF8EEE77A40462E
:1018D00067EE887AFDEEE77ACDED027ABDF8081062
:1018E000EFF76CFFB9F9043007EE903AF8EEE77ABB
:1018F000404667EE887AFDEEE77ACDED027ABDF8D4
:101900000810EFF75BFF40461EF0B2FAFEF74BBB44
:1019100099780393184614F057F800287FF4C8AB61
:101920008F49904F904A09889048914CF961DFF8AF
:101930005892116803689268F962B4F85E11C7F8AA
:101940006CB0FB63FA64D9F80000F965F1F7D6FED4
:10195000834600287EF499AA5146D9F80000F3F78F
:10196000A1FF039B94F86021DB780493642A4FF075
:10197000040387F8743040F00D8194F86131DFF88A
:101980000CA2072B08BF84F861B194F8612106927C
:1019900007EB021BDBF80410059108461FF094FBCF
:1019A000DBF8083003935FFA80FB18461FF08CFBCE
:1019B000C3B20BEB0300069A0599059308308AF829
:1019C000070022F00F008AF80A0002F00F0203EB72
:1019D000CB008AF80D208AF80E005A460AF10F0053
:1019E00020F06AFA059B03990BF109001A460AF1E7
:1019F0000603184420F060FA9AF8073003F1010B4F
:101A0000D3B1013B5FFA83FC0CF1080CDFF880E1F5
:101A1000D4440AF10700002310F8011B59408B0041
:101A2000CA0883EA410302F018024B404EFA02F260
:101A300053408445DBB2EFD14E4A04980BF8023094
:101A400020F01CFA94F861310022013384F86131EE
:101A500084F860219AF802305BB11AF80610D9F8C0
:101A60000000F3F733FF01369AF80230F6B2B342C2
:101A7000F3D894F860310322013384F8603187F899
:101A8000742088F80020FFF7ACB9354B3A4A1B8820
:101A9000927903EB830303EB83039B001FFA83FA22
:101AA000002A46D0304B1A680FFA82F903F042F848
:101AB00040B2FEF708BB4FF0340856E41146944696
:101AC000039292460492FEF7FBBB03F033F810F04A
:101AD000FBFA002010F0F8FA94F82C31D8F8002026
:101AE000FEF738B90327254917E6D8F800305E20FD
:101AF0009847D8F80030392098475FFA89F010F0FD
:101B0000E3FA4FEA192010F0DFFAFFF79FBA4FF01F
:101B100024082AE40021FFF7B0BB19490427FCE59B
:101B20004FF0100821E44FF020081EE44FF00808A1
:101B30001BE44FF0FF32B7E70B4B8246B3F900903E
:101B40006420FEF7C0BA114694460392924604926E
:101B50009046FEF7B5BB00BF58A08B41784D0020E2
:101B6000304D00200C0000201C4D0020684F00204C
:101B70008426002086600020544F0020C86503089A
:101B8000CC650308704F00203441002080600020A5
:101B90000007090E97F87530DFF840A10596190780
:101BA00004BF0133DBB2072B28BF01234FEA031B1D
:101BB00007EB0B024649107C00228AF80A2011F834
:101BC00000C05FFA8BF203920AF10D02039E07EB4D
:101BD0000B013043BCF1010F1070C96802F1010024
:101BE0000ED9ACF10206F6B206F1020E9644024698
:101BF00002F8011B72454FEA1121F9D10136304438
